:100000000C9461100C9492100C9492100C94921019
:100010000C9492100C9492100C9492100C949210D8
:100020000C9492100C9492100C9492100C949210C8
:100030000C9492100C9492100C9492100C949210B8
:100040000C9492100C9492100C9492100C949210A8
:100050000C9492100C9492100C9492100C946CAC22
:100060000C9492100C944F8B0C94258B0C94921042
:100070000C9492100C9492100C9492100C94921078
:100080000C9492100C9492100C9492100C94921068
:100090000C94FB8A0C94D18A0C9492100C94A8298D
:1000A0000C9492100C9492100C9492100C94921048
:1000B0000C9492100C9492100C9492100C94921038
:1000C0000C9492100C9492100C9492100C94A78A99
:1000D0000C947D8A0C9492100C94538A0C94298A67
:1000E0000C94921007634236B79BD8A71A3968560A
:1000F00018AEBAAB558C1D3CB7CC5763BD6DEDFD4A
:10010000753EF6177231BF000000803F0800000006
:10011000BE922449123EABAAAA2ABECDCCCC4C3EFC
:1001200000000080BEABAAAAAA3E00000000BF00EB
:100130000000803F0000000000084178D3BB4387E7
:10014000D1133D190E3CC3BD4282AD2B3E68EC82FB
:1001500076BED98FE1A93E4C80EFFFBE01C4FF7F80
:100160003F00000000000C94FB390C942E150C94F9
:10017000CD7E0C94CA230C94C17D0C949F1E0C94CC
:10018000963C0C944E120C94B4200C94A13A0C940E
:10019000BA140C946E3C0C94E0C10C94523D0C9437
:1001A000005F0C94FEA50C9451120C94B6140C94A0
:1001B000115E0C9431180C941A860C9431630C94D3
:1001C00014160C943A290C941D160C943D280C948A
:1001D0003E5F0C94E0380C94454D0C946E480C94A2
:1001E0004EB80C94CE370C94203C0C947E140C9496
:1001F000CB130C9462140C94EAC20C94B6610C9468
:100200006CC20C940B3D0C948D380C9477280C9494
:100210005C140C940F290C94AE100C9445120C94A1
:100220006A120C94524D0C945F140C94FF390C9488
:10023000F55E0C94623D0C94F5210C9413C30C9460
:100240007F620C9473120C9414490C94157D0C94D9
:10025000B5BD0C94B23B0C94AC190C9457A60C94FD
:10026000633D0C94AA190C946F210C94A6120C9463
:10027000007C0C9431A50C944C260C94AA100C9480
:1002800061310C948DC20C940B130C9481120C945C
:10029000693A0C948A130C94A2690C94D24C0C9475
:1002A000253D0C9451170C946B7C0C9476710C9436
:1002B0007AA60C9419120C94747D0C9484200C94DE
:1002C000BC5E0C94B0360C9473170C945F7E0C9447
:1002D00066620C94A8150C9433400C9427A50C94DA
:1002E000794D0C9439620C946A3C0C94AE190C94C0
:1002F0008F1F0C941F120C94B21D0C94B5740C94A7
:10030000825A0C948A380C9425170C9446120C943B
:10031000C0200C94258D0C9486120C94FA140C9425
:1003200006550C940E8D0C94477C0C9445400C940F
:1003300055A50C944B180C94EB130C94797C0C94ED
:1003400043A50C94C1620C944DA50C9428130C94F5
:10035000708D0C94BF270C943A180C9458A50C94EB
:100360007B7E0C949E140C94EC610C94CD380C9410
:100370000BA60C94B0190C9407B60C9483730C94D0
:100380007F480C947F150C94A6C40C948EA60C94F4
:10039000923D0C94F25E0C94643B0C94D3470C9405
:1003A0006C140C9466180C948E120C94B7380C9440
:1003B0001C180C94F91E0C945A7D0C94C8C40C940F
:1003C00005620C9416120C946D780C9429A60C946A
:1003D000D6140C94B47E0C94AC130C940D7E0C9437
:1003E000035F0C94787F0C94B9490C949C3B0C945B
:1003F000413D0C9458C20C945E3C0C9466A60C943F
:100400002F800C94E93D0C94CF5E0C94413C0C94ED
:10041000D7370C94E65E0C94A8200C94A85E0C943C
:10042000C3350C941DA50C9439A50C9419A50C94F6
:10043000333D0C94FE8E0C94B0630C94E4230C9426
:10044000563A0C9421A50C94E3620C94561A0C9421
:1004500098A60C9406A60C9431390C9483490C94FC
:1004600059A50C94DD690C94FC620C94AF1D0C949E
:1004700098380C9479160C9435A50C9415A60C9408
:1004800039260C94F01B0C94CF100C944DA60C94B0
:10049000847D0C94A8140C94B4190C9459210C94D8
:1004A0008E150C94BE380C94C7150C946F120C94D6
:1004B00072150C947E7D0C94FA4C0C94851E0C9451
:1004C00007120C94F3390C94C4390C944E5E0C94BE
:1004D00043A60C94D9210C9403130C94201E0C9465
:1004E00080610C94B21E0C940B160C942BA50C94EA
:1004F00083120C9432380C94F2130C94D16C0C943B
:10050000CA3C0C94058D0C94F47D0C94E3130C946C
:1005100084A60C94607F0C9413A50C9496120C94F2
:1005200023780C9405C30C94E6480C94E2470C9491
:1005300092120C9437850C94C51E0C9431150C94B2
:10054000BE210C943FA50C9415120C94D71F0C944B
:1005500079390C942A2B0C941A260C94CE7C0C948A
:100560008A7E0C94A8280C94C4100C9477120C94D6
:100570001FA60C942B380C9440120C9460120C940F
:1005800009BD0C944D3D0C9411340C94F3200C9443
:10059000BB8D0C94013A0C9450390C94033A0C9492
:1005A00093730C9449120C94E9390C9451A50C9452
:1005B000577C0C940F5F0C94C93D0C9465140C94FB
:1005C0002B3C0C94013D0C94F1150C94364D0C947D
:1005D0008F3D0C948F2E0C94C47F0C948C630C94E0
:1005E0001D4D0C9490380C94D1370C945F120C94E0
:1005F00031A60C9493380C945D3A0C9434130C94FB
:10060000407F0C947F3B0C94E03C0C9489630C94E9
:10061000143A0C94BC140C940C6D0C94993B0C94EF
:1006200070A60C94BF140C94EC490C94B2190C9461
:10063000C67E0C947B7D0C9463120C9436BB0C9498
:10064000D4130C9454B80C94C4380C9404540C94E3
:10065000828D0C9410330C94EE7B0C940A170C943E
:1006600094100C945EC20C94A63C0C94DC380C9450
:10067000A2410C9447A50C94904C0C947C180C94BB
:10068000AB390C9439A60C94EC160C948F630C9433
:100690001E120C94F48C0C94DF280C94F4470C94E8
:1006A0006D3A0C94017C6364696E6F707375785851
:1006B0005B004E414E494E495459494E46CDCCCC33
:1006C0003D0AD7233C17B7D13877CC2B329595E626
:1006D000241FB14F0A000020410000C84200401C06
:1006E0004620BCBE4CCA1B0E5AAEC59D74556E6BDF
:1006F0006E6F776E207375666669782000556E6B35
:100700006E6F776E20636D642000636C7243747249
:100710003A20002F00496E3A20003D00494E3A0031
:100720003D004C454741435920494E3A00000020C6
:10073000002300260029002C002F003200000100B9
:10074000000301060109012D3E00200023002D3E7B
:1007500000200050656E6465643A20230072617762
:100760000076616C0074656D70007361740068756B
:10077000650066616E0052474200485356006D6F37
:10078000646500536574436D643A0053746F726519
:1007900064204558543A00737566666978436F64FF
:1007A000653A00584F4E0048414C54002074696D22
:1007B000653A004374726C205265733A00205453BA
:1007C0003A0020543A003D0050696E3A004F4E3ACC
:1007D000416C7265616479204163746976650A00D1
:1007E00048414C543A416C726561647920496E61AC
:1007F00063746976650A00584F4E3A416C726561C0
:100800006479204163746976650A00584F46462032
:10081000736B69707065642E205072657620636D0D
:10082000643A005475726E6564206F666620667265
:100830006F6D3A00526573746F7265642066726FF3
:100840006D3A0049676E6F7265642C206368616E53
:100850006E656C20636D643D0020457865633A00E9
:100860004163746976653A0048414C543A416C7270
:100870006561647920496E6163746976650A005820
:100880004F4E3A416C7265616479204163746976B8
:10089000650A00584F464620736B69707065642E78
:1008A000205072657620636D643A005475726E65EF
:1008B00064206F66662066726F6D3A0052657374CD
:1008C0006F7265642066726F6D3A004E6F742065BA
:1008D0006E6F756768206D656D6F727920666F72D7
:1008E0002067726F7570206F7065726174696F6ECA
:1008F00000206D73203A0041726D656420666F724E
:1009000020002044697361726D656400536B6970E7
:1009100070656420686F6D69652073747566660024
:100920004F75744F664D656D6F7279210A00200016
:10093000205375623D00204974656D3D0052414D64
:100940003D00282D292000282B2920002076616CCD
:100950007565206973200020756E6B6E6F776E0A67
:10096000005D3D005B0020696E76616C696400206B
:1009700000206F6B003A00206661696C6564003A84
:10098000005265747279696E67206D6F6462757369
:1009900020434D440A00207365632072656D6169D0
:1009A0006E696E6700537461747573206465666662
:1009B000657265640A002D3E005075623A2000633E
:1009C0006D640046414E5F4F4E4C590044525900F1
:1009D000434F4F4C0048454154004155544F002D62
:1009E0003E005075623A20007365740064656C00C7
:1009F0002D3E005075623A20002D3E005075623A3F
:100A00002000556E6B6E6F776E20636D64200A0058
:100A10004F4646004F4E0020002D3E00436F6E763D
:100A2000657274696E6720002D3E0057726F6E67A5
:100A30002041737369676E6D656E74200052474282
:100A4000783A200020764C6576656C3A0020436F3A
:100A50006E76563A0020436F6E76533A0020486F08
:100A6000743A00436F6C643A0020436F6E7665728F
:100A700074656420563A00436F6E766572746564DF
:100A800020533A002D3E0057726F6E6720417373FA
:100A900069676E6D656E7420002D3E0057726F6E33
:100AA000672041737369676E6D656E7420005361D2
:100AB0007665643A0020537566663A002041543AE0
:100AC00000436F6E666967206368616E67656420C6
:100AD0006C6F63616C6C792C20706F7274616C2028
:100AE00064697361626C6564002F636F6E66696729
:100AF0002E6A736F6E007265626F6F742000436DB3
:100B0000643A20002F636F6D6D616E642F002F7249
:100B1000616D2F002F6974656D2F002F6974656DED
:100B20002F004C6F636174696F6E3A206874747043
:100B30003A2F2F6C617A79686F6D652E72752F7000
:100B40007761003F6D61633D002669703D0026704E
:100B50006F72743D00266E616D653D002F002000B0
:100B6000436F6D706C6574652E2052656D6F766590
:100B700020746F706963200024636F6D6D616E6413
:100B800000536B697070696E672E2E00436C65614F
:100B90006E55702072657461696E656420746F7043
:100BA00069632000220022004F75744F664D656D09
:100BB0006F727921005D20003A5B000A005D0045FC
:100BC0006D7074793A205B000A003A004D41433A57
:100BD00000554450205379736C6F6720696E6974B7
:100BE00069616C697A65642E0A005379736C6F676A
:100BF00020706172616D733A0043757272656E7434
:100C0000204C414E20636F6E6669672869702C64C2
:100C10006E732C67772C7375626E6574293A000ABF
:100C200055736520746865736520636F6D6D616EC3
:100C300064733A202768656C7027202D20746869DA
:100C40007320746578740A276D61632064653A6166
:100C5000643A62653A65663A66653A3030272073D1
:100C6000657420616E642073746F7265204D41431A
:100C70002D6164647265737320696E20454550521E
:100C80004F4D0A276970205B69705B2C646E735B43
:100C90002C67775B2C7375626E65745D5D5D5D2797
:100CA000202D20736574207374617469632049502A
:100CB0000A277361766527202D207361766520638E
:100CC000757272656E7420636F6E66696720696EF7
:100CD000204E5652414D3B204F4E7C4F4646202DD4
:100CE00020656E61626C652F64697361626C65205A
:100CF0006175746F736176650A2767657427205B79
:100D0000636F6E66696720616464725D27202D20C1
:100D100067657420636F6E6669672066726F6D2009
:100D20007072652D636F6E666967757265642055B4
:100D3000524C20616E642073746F7265206164642C
:100D4000722C204F4E7C4F4646202D20656E6162EE
:100D50006C652F64697361626C6520646F776E6C7B
:100D60006F6164206F6E20737461727475700A27EE
:100D70006C6F616427202D206C6F616420636F6E3F
:100D80006669672066726F6D204E5652414D0A2784
:100D900070776427202D20646566696E6520616E1A
:100DA000642073746F7265204D51545420706173C8
:100DB00073776F72640A276F746170776427202DD0
:100DC00020646566696E6520616E642073746F725D
:100DD0006520485454502041504920706173737706
:100DE0006F72640A276C6F67205B73657269616C50
:100DF0005F6C6F676C6576656C5D205B7564705FBA
:100E00006C6F676C6576656C5D27202D2064656668
:100E1000696E65206C6F67206C6576656C20283084
:100E20002E2E37290A276B696C6C27202D207465BC
:100E30007374207761746368646F670A27636C65F5
:100E4000617227202D20636C6561722045455052E8
:100E50004F4D0A277265626F6F7427202D207265CF
:100E6000626F6F7420636F6E74726F6C6C6572006A
:100E7000536F6674207265626F6F74696E672E2E91
:100E80002E0052414D3D000A5379736C6F6720006C
:100E90000A6D71747420000A696E70757473200095
:100EA0000A6974656D7320000A436F6E6669677521
:100EB0007265643A003B003D0050696E3A003B00A9
:100EC0003D4C4F5700546865726D6F3A0041707029
:100ED0006C79696E6720636F6E666967004C6F613D
:100EE00064656420455441473A004E6F2073746F27
:100EF00072656420636F6E666967004C6F6164653C
:100F0000642066726F6D20454550524F4D006C6FE6
:100F10006164206661696C6564004C6F6164696E30
:100F20006720436F6E6669672066726F6D20454566
:100F300050524F4D00436F6E666967206175746F44
:100F4000736176653A000A5379736C6F6720646544
:100F5000627567206C6576656C3A005365726961ED
:100F60006C206465627567206C6576656C3A005329
:100F7000617665640A005365742064796E616D69F9
:100F8000632049500A00454550524F4D20636C651F
:100F9000617265640A004D51545420506173737737
:100FA0006F726420757064617465640A004F544107
:100FB0002050617373776F7264207570646174651B
:100FC000640A00636F756C64206E6F7420706172C8
:100FD00073653A2000557064617465640A004E6F51
:100FE000204950206164726573730052656C6561BD
:100FF00073696E6720736F636B657420616E642024
:10100000726574727900205361766564004C6F617B
:1010100064696E67204854545020636F6E66696738
:10102000206F6E20737461727475703A004F46467B
:10103000004F4E002B002D00455461673A200047B9
:10104000657420455441473A2000485454502F318C
:101050002E312025690025733A2025730D0A0020C2
:10106000485454502F312E310D0A486F73743A2072
:1010700025730D0A4163636570743A202A2F2A0D87
:101080000A436F6E6E656374696F6E3A20636C6FAE
:1010900073650D0A0025730020000D0A00474554B2
:1010A000006661696C656420746F20636F6E6E65A5
:1010B00063740A004552524F523A20536572766566
:1010C000722072657475726E65642000436F6E667F
:1010D0006967206E6F74206368616E6765640A00DB
:1010E000446F6E652E0A00436F6E666967207061FB
:1010F0007273696E67206661696C65640A00676F68
:101100007420436F6E6669670A0066726565200029
:10111000436F6E666967205552493A20687474704F
:101120003A2F2F002044656661756C7420636F6EE2
:101130006669672073657276657220757365643AB7
:1011400020006C617A79686F6D652E7275000A28CF
:101150002B29454C455641544F52000A282B294D06
:10116000554C544956454E54000A282B2950574D8A
:101170005F52454C4159000A282D294D444E5300D9
:101180000A282D2955415254425249444745000AE4
:10119000282B295359534C4F47000A282D295049D1
:1011A00044000A282D294D43503233303137000A8C
:1011B000282D294152544E4554000A282B294F54BA
:1011C00041000A282D29535049204C4544000A2843
:1011D0002D294D4F544F5220435452000A282B2999
:1011E0004143204841494552206F6E205365726942
:1011F000616C33000A282D294343533831312026AE
:101200002048444331303830000A282B29524553B6
:10121000544152545F4C414E5F4F4E5F4D515454B8
:101220005F4552524F5253000A282D2948415244DB
:1012300052455345542C207573696E6720736F6651
:1012400074000A282D29434F554E544552000A2850
:101250002D29444854000A282D294F57495245004A
:101260000A282D294D4F44425553000A282D294460
:101270004D58000A282B2957697A6E6574357830E5
:1012800030000A282B294672656552616D20707204
:10129000696E74696E67000A282B295741544348C8
:1012A000444F47000A4669726D77617265204D416F
:1012B0004320416464726573732064653A30313A47
:1012C00032333A30303A30303A3031006C617A792A
:1012D000686F6D652E7275000A436F6E66696720D0
:1012E0007365727665723A003230313730334C00B4
:1012F00020432B2B2076657273696F6E3A0036346B
:1013000065656130375F323032322D30352D313006
:10131000000A4C617A79686F6D652E7275204C6990
:1013200067687448756220636F6E74726F6C6C6569
:10133000722000204F464600204F4E002042595058
:1013400041535300757074696D6500667265656818
:10135000656170002054696D65723A00204C6F63BE
:101360006B733A002000204C6F636B733A000A5293
:10137000414D3D0020457870697265640A00202D5A
:10138000746172676574207A6F6E652D0020416C00
:1013900061726D20457870697265640A0020636D22
:1013A000643A00204375723A00205365743A005342
:1013B0006176656420746F20454550524F4D00534F
:1013C0006176696E6720636F6E66696720746F204F
:1013D000454550524F4D2E2E002069732000446524
:1013E0006C6574696E6720636F6E662E2052414D86
:1013F000207761733A0053746F70706564005374A2
:101400006F7070696E67206368616E6E656C7320C3
:101410002E2E2E004E6F7420756E6C6F636B65649C
:1014200020696E20313073202D20636F6E74696ED9
:101430007565202E2E2E00556E6C6F636B696E677E
:1014400020636F6E666967202E2E2E00414320496F
:101450006E69740041432044652D496E69740045EE
:101460005252004452590046414E5F4F4E4C590073
:101470004845415400434F4F4C00506F6C6C696EAF
:1014800067004C4F57004D454449554D004849476A
:1014900048004155544F0072617700717565697459
:1014A000007377696E67006C6F636B0044656661FB
:1014B000756C742073657269616C206D6F64652052
:1014C0004E38312075736564003845310026003888
:1014D0004E31000600384532002E00384E32000EE4
:1014E00000384F31003600384F32003E003745316A
:1014F000002400374532002C00374F3100340037CC
:101500004F32003C00374E31000400374E32000CA1
:1015100000203D3E002C002C002C002C00456C656A
:101520007661746F723A20636F6E666967206661D8
:10153000696C65643A00456C657661746F7220630E
:101540006F6E666967206572726F7200456C6576B2
:1015500061746F7220636F6E666967206C6F61647F
:1015600065642000456C657661746F723A204F7532
:1015700074206F66206D656D6F727900456C6576BD
:1015800061746F722044652D496E6974004030307B
:1015900052523030303030313030334630303431E8
:1015A0003043303034322A00403030525230303004
:1015B0003030323030374630303032313030303306
:1015C000302A0040303052523030303030343030F9
:1015D0003346303038343134303033382A003C0030
:1015E0003E00556E6B6E6F776E2073756666697818
:1015F0002000556E6B6E6F776E20636D6420005314
:101600006574206E6F7420696D706C656D656E74A5
:10161000656400466F726365642065786563757400
:10162000696F6E00454C45563A20004D756C7469E3
:1016300056656E7420636F6E666967206661696CBB
:101640006564004D756C746956656E7420696E69C9
:1016500074004D756C746976656E742044652D490F
:101660006E697400204F75743A00206D3300206657
:10167000726F6D2000204D61782072657175657301
:10168000743A002066616E253A00206163746976C1
:101690006520563A00546F74616C20563A002069F8
:1016A0006E69740050574D2D4F75742023002073C0
:1016B000746F700050574D2D4F75742023003D00FE
:1016C00050696E3A0020696E69740052656C6179E8
:1016D0002D4F75742023002073746F700052656C59
:1016E00061792D4F75742023003D3E003A007075DE
:1016F0006220616374696F6E200069646C65006FBD
:1017000066660068656174696E670066616E006494
:101710007279696E6700636F6F6C696E670020692C
:101720007320004F75742000556E6B6E6F776E20BE
:101730007375666669782000556E6B6E6F776E20E4
:10174000636D642000616374696F6E0072656C6123
:10175000794374723A20005B305D3A2000202D20DE
:101760002D202D20EFBBBF003E003E31202D20005C
:1017700020002E00696E00735F6F7574006D7968CC
:101780006F6D6500202D3E2000456D69743A200084
:10179000202D3E20004974656D436D643A20002081
:1017A0002D3E20004974656D3A20003E3E200049E0
:1017B0006E76616C696420636F6D6D616E64003E6E
:1017C0003E3E004E6F204D414320636F6E66696759
:1017D000757265643A20736574206669726D77610D
:1017E00072652773204D41430A004E6F2076616C6D
:1017F000696420454550524F4D20646174612E202C
:10180000496E697469616C697A696E672E00476F09
:101810007420495020616464726573733A002769CB
:1018200070205B69705B2C646E735B2C67775B2C3C
:101830007375626E65745D5D5D5D27202D20736537
:1018400074207374617469632049500A00466169A9
:101850006C656420746F20636F6E6669677572656E
:101860002045746865726E6574207573696E6720B3
:10187000444843502E20596F752063616E20736574
:1018800074206970206D616E75616C6C7921000A3D
:101890007573657320444843500A00204D41534BF3
:1018A0003A002047573A0020444E533A004C6F61AB
:1018B0006465642066726F6D20666C617368204990
:1018C000503A005374617274696E67206C616E00E7
:1018D0004142434445464748494A4B4C4D4E4F5080
:1018E0005152535455565758595A6162636465664C
:1018F0006768696A6B6C6D6E6F7071727374757600
:101900007778797A303132333435363738392B2F8E
:101910003D004261736963200061726475696E6F96
:101920003A004F544120696E697469616C697A6547
:10193000640A0044454641554C54207061737377E6
:101940006F726420666F72204F5441204150492EBF
:1019500020557365206F746170776420636F6D6DBF
:10196000616E6420746F20736574007061737377A7
:101970006F726400757074696D652C667265656858
:101980006561700024737461747300363465656139
:1019900030375F323032322D30352D3130004C69E6
:1019A0006768744875622000246E616D6500726519
:1019B00061647900546F6F206D616E79204D5154D0
:1019C0005420636F6E6E656374696F6E206572720A
:1019D0006F72732E2052657374617274204C414E85
:1019E000002074727920616761696E20696E20350C
:1019F000207365636F6E6473006661696C65642C47
:101A00002072633D004177616974696E6720666F7B
:101A1000722072657461696E656420746F706963A9
:101A20007300636F6E6E656374656420617320007C
:101A3000202E2E2E0020757365723A003A000A415E
:101A40007474656D7074696E67204D5154542063D1
:101A50006F6E6E656374696F6E20746F20002473FF
:101A60007461746500646973636F6E6E6563746539
:101A700064005573696E67204D5154542070617332
:101A800073776F72642066726F6D20636F6E666924
:101A90006700446576696365204E616D653A004173
:101AA00074206C6561737420646576696365206E6B
:101AB000616D6520616E642062726F6B6572204992
:101AC00050206D75737420626520636F6E66696760
:101AD0007572656400526562696E64207375636334
:101AE0006573732E20495020616464726573733A84
:101AF000004572726F723A20726562696E64206688
:101B000061696C0052656E65776564207375636307
:101B10006573732E20495020616464726573733A53
:101B2000004572726F723A2072656E657765642047
:101B30006661696C000A4E6F206C696E6B005265BD
:101B400073746F72696E6720636F6E666967206673
:101B5000726F6D20454550524F4D00416363657073
:101B600074696E6720636F6D6D616E64732E2E2EC7
:101B70000A004E6F204D51545420636F6E666967A2
:101B800075726564004C6F6164696E6720636F6E87
:101B90006669672066726F6D20706F7274616C2069
:101BA00064697361626C65642E2075736520676576
:101BB00074204F4E20746F20656E61626C65004327
:101BC0006F6E6669672069732076616C6964004393
:101BD0006F6E74696E7565207769746820707265C0
:101BE00076696F75736C79206C6F616465642063CE
:101BF0006F6E6669670000002100240027002A003C
:101C00002D003000330001010000040107010A012A
:101C100000002200250028002B002E003100340097
:101C200002010000050108010B0105050505070576
:101C300008080808020202020A0A08080404040448
:101C40000101010101010101030303030303030374
:101C5000040707070C0C0C0C0C0C0C0C0202020203
:101C600006060606060606060B0B0B0B0B0B0B0BEC
:101C7000050505080807070404040A0A0A0A0A0AEF
:101C8000010210202008081020401020408002018E
:101C90000201080402010102040810204080804073
:101CA0002010080402018004020180402010080472
:101CB0000201080402010102040810204080010210
:101CC0000408102040800440800480081010204048
:101CD00004081020408000000B0C030A0D0E0F09B1
:101CE00008040502000000000000000000000000E1
:101CF00000000000000000000000000000000000E4
:101D0000000013121100000000000000000000009D
:101D100000000000000000000000000000000000C3
:101D20000000000000000000000000002F6461744B
:101D300061002F736B65746368004163636573733F
:101D40002D436F6E74726F6C2D526571756573746F
:101D50002D507269766174652D4E6574776F726B64
:101D60003A2074727565004163636573732D436F28
:101D70006E74726F6C2D416C6C6F772D4865616469
:101D80006572733A202A004163636573732D436F54
:101D90006E74726F6C2D416C6C6F772D4D6574682D
:101DA0006F64733A20504F53542C4745542C4F5076
:101DB00054494F4E53004163636573732D436F6EF7
:101DC00074726F6C2D416C6C6F772D437265646516
:101DD0006E7469616C733A2074727565004F50546B
:101DE000494F4E530044454C45544500505554000E
:101DF00047455400504F535400617574686F7269C1
:101E00007A6174696F6E3A2000417574686F726907
:101E10007A6174696F6E3A2000436F6E74656E74F8
:101E20002D4C656E6774683A20006F637465742F7B
:101E300073747265616D00696D6167652F6A7065A5
:101E40006700696D6167652F6769660074657874FE
:101E50002F68746D6C006170706C69636174696F78
:101E60006E2F6A736F6E00746578742F706C616981
:101E70006E00436F6E74656E742D547970653A20F0
:101E800000436F6E6E656374696F6E3A20636C6FAA
:101E90007365004163636573732D436F6E74726F76
:101EA0006C2D416C6C6F772D4F726967696E3A20AB
:101EB000687474703A2F2F6C617A79686F6D652E33
:101EC000727500556E6B6E6F776E004E6F74204D9D
:101ED0006F646966696564004F4B004D6F76656499
:101EE000207065726D616E656E746C7900496E74F8
:101EF00065726E616C2053657276657220457272F0
:101F00006F72005061796C6F616420546F6F204C68
:101F100061726765004E6F7420666F756E6400575E
:101F200057572D41757468656E7469636174653ABD
:101F3000204261736963207265616C6D3D2241636B
:101F40006365737320726573747269637465642268
:101F500000556E617574686F72697A6564005061CE
:101F6000796C6F61642073697A652077726F6E6730
:101F70000042616420726571756573740048545441
:101F8000502F312E31200020000000000000000002
:101F900000004F4E000000000000004F46460000C9
:101FA00000000000524553540000000000544F4709
:101FB000474C4500000048414C54000000000058C8
:101FC0004F4E000000000000584F46460000000041
:101FD00000494E4352454153450044454352454113
:101FE000534500484541540000000000434F4F4C0A
:101FF00000000000004155544F0000000000464121
:102000004E5F4F4E4C5900445259000000000000F2
:1020100053544F500000000000484947480000005A
:1020200000004D454449554D0000004C4F570000FD
:102030000000000054525545000000000046414C8D
:10204000534500000000454E41424C4544000044C9
:10205000495341424C4544005247420000000000B1
:102060000048535600000000000057726F6E672052
:102070007061796C616400202D3E2041543A004328
:1020800068616E20747970653A004E6F2073746FCA
:102090007265642076616C756573202D20646566B9
:1020A00061756C743A200053617665642045544133
:1020B000473A0053657420455441473A2000C8C44C
:1020C000A6C411241FBECFEFD1E2DEBFCDBF00E01A
:1020D0000CBF16E0A0E0B2E0E6EEF6EB01E00BBFCD
:1020E00002C007900D92A83DB107D9F720E1A8EDF5
:1020F000B6E001C01D92A236B207E1F710E1C0E6DA
:10210000D0E100E006C021970109802FFE010E9466
:1021100029D6CF35D10780E00807A9F70E9462B41D
:102120000C9461DB0C940000CF93DF931F92CDB72A
:10213000DEB76983DC01ED91FC910280F381E02D33
:1021400041E050E0BE016F5F7F4F19950F90DF9126
:10215000CF910895FC01818D928D0895CF93DF93E7
:102160001F92CDB7DEB76983DC01ED91FC9102804F
:10217000F381E02D41E050E0BE016F5F7F4F199584
:102180000F90DF91CF910895FC019485FB01848528
:10219000981303C081E0983008F080E00895CF9351
:1021A000DF931F92CDB7DEB76983DC01ED91FC911F
:1021B0000280F381E02D41E050E0BE016F5F7F4F70
:1021C00019950F90DF91CF91089585ED8093BC0014
:1021D0008091BC0084FDFCCF10926008089520918E
:1021E0003C08260F3327331F21323105ECF42091B0
:1021F0006008FC0190E080E0243069F082E00895FE
:10220000A0913C082191AC01445E574FA40FB52F1B
:10221000B11D2C930196861798F380913C08680FA6
:1022200060933C0880E0089581E008958FEF9FEF70
:1022300008958FEF9FEF089580911B0890E091958E
:10224000819591090895CF93DF93CB01EA01642F23
:102250000E94EF10CE01DF91CF910895CF93DF93CD
:102260001F92CDB7DEB7698361E0CE0101960E946F
:10227000EF1081E090E00F90DF91CF91089590E012
:10228000FC01E65DF34EE491F0E0EE0FFF1FE05F2E
:10229000F34EA591B4912C918058934EFC018491FA
:1022A000822391E009F490E0892F08958F929F9204
:1022B000AF92BF92CF92DF92EF92FF920F931F9354
:1022C000CF93DF9300D000D000D01F921F92CDB7E4
:1022D000DEB77C018E010F5F1F4F68018AE0882EF8
:1022E000912CA12CB12CC601801B910B41155105DD
:1022F0006105710581F0CB01BA01A50194010E942D
:102300009ED5942F852F605DF60161936F01A90121
:10231000692F782FE8CFF801E80FF91FD701015096
:10232000110922912D93E017F107D9F7E80EF91E54
:10233000F70110822B960FB6F894DEBF0FBECDBF0B
:10234000DF91CF911F910F91FF90EF90DF90CF9091
:10235000BF90AF909F908F900895FC01DC018D910C
:102360008111FDCF30E020E050E040E08AE0919123
:10237000992301F1443051055CF59E3271F42F3FF1
:10238000310509F02CF5DB01A40FB51F12962C9333
:102390004F5F5F4F30E020E0EACF829FD001839F04
:1023A000B00D1124292F990F330B205331092A0F17
:1023B0003B1FDDCF2F3F310509F054F44430510568
:1023C0003CF4640F751FFB01228381E090E00895C7
:1023D00090E080E00895CF93DF931F921F92CDB7D6
:1023E000DEB78091561090915710009711F482E655
:1023F00090E1BE016F5F7F4F681B790B072E000CC9
:10240000880B990B0F900F90DF91CF910895DC010D
:1024100015968D919C91009739F0DC01ED91FC911E
:102420000680F781E02D19940895089583E090E0E7
:1024300008958091C3079091C40708950895DC0121
:102440001296ED91FC9113973097B9F016968D91F5
:102450009C918430910541F08530910541F00397BE
:1024600049F482E090E0089581E090E0089581E1F0
:1024700090E00895808590E0089590E080E00895D0
:102480008091C1079091C2070895089590E080E07F
:1024900008958091BF079091C007089584E090E06F
:1024A0000895DC011496ED91FC91309729F080811C
:1024B000082E000C990B089590E080E0089508958F
:1024C00085E090E008958091080790910907817058
:1024D000992708958091F7069091F8060895FC01D8
:1024E000848195810895FC01768765870895DC01D4
:1024F000ED91FC91068CF78DE02D199591E08927DF
:102500000895862F089581E08627089521E0FC0133
:102510008485883008F020E0822F0895FC018485AE
:1025200095850895FC0184899589089522E334E016
:10253000FC0131832083FB014089518962897389C1
:10254000FC0142835383648375830895DC01ED911C
:10255000FC91048CF58DE02D1994CF93DF9300D07E
:1025600000D01F921F92CDB7DEB7FC016F3F7105FF
:1025700019F014F06FEF70E077FD60E09181892F22
:1025800082958F7081508230C8F4648388E0DE01C8
:10259000119601900D928A95E1F729813A814B813C
:1025A0005C816D817E818F81988528960FB6F89425
:1025B000DEBF0FBECDBFDF91CF9108959F709061B8
:1025C0009183E3CF0F931F93CF93DF93DC01C62F4B
:1025D0001196EC911197E295EF70EC3008F0BCC0C9
:1025E000F0E08827E950FD4E8F4F0C9429D6031355
:1025F00028132813AC13AC13AC138A133413AC1385
:10260000AC130B130B1370E060E0CB01DF91CF91A3
:102610001F910F91089514968D919D910D90BC91ED
:10262000A02D8F3F9105A105B10529F024F08FEF72
:1026300090E0A0E0B0E0B7FF03C080E090E0DC01F4
:102640006FEF70E0681B790BC111DFCFBC01DDCFEC
:1026500014966C9170E0CC23C1F28FEF90E09C0156
:10266000261B370BB901D1CF862F14960C911497E6
:1026700015961C9115971696DC9116971796CC9186
:1026800020E030E0A901B801882331F18D2F9C2F83
:102690000E9454D487FD1BC020E030E04FE753E494
:1026A000B8018D2F9C2F0E945CD7181624F400E0EF
:1026B00010E0DFE7C3E498014D2F5C2F60E070E08D
:1026C0008FE793E40E9447D60E9426D79ECF00E072
:1026D00010E0D0E0C0E0EFCF8D2F9C2F0E9454D4AB
:1026E00087FD13C020E030E04FE753E4B8018D2FA1
:1026F0009C2F0E945CD7181624F400E010E0DFE75E
:10270000C3E4B8018D2F9C2FDFCF00E010E0D0E0B4
:10271000C0E0F7CF14966D917D918D919C911797A4
:1027200024E630E040E050E00E94C0D52F3F310564
:102730004105510529F024F02FEF30E040E050E052
:1027400057FF03C020E030E0A9016FEF70E0621B8B
:10275000730BC1115ACF86CF6FEF7FEF56CFDC01DD
:102760001196EC911197E295EF70E150EB3008F083
:1027700039C0F0E08827E054FC4E8F4F0C9429D6E6
:10278000E313E313F213CB13CB13D413EB13EB13B9
:10279000EB13CB13CB1314966D917D918D919C917E
:1027A00017970E945BD4089514966D917D918D9139
:1027B0009C91179724E630E040E050E00E94C0D59D
:1027C000CA01B901EECF14966C9170E090E080E000
:1027D0000E9459D4089514966D917D918D919C918C
:1027E0001797089560E070E0CB010895FC01A78180
:1027F0002A2F2E7FD1F0818182958F708150833076
:10280000A0F4A695A150BB0B2BE531E00E9440D669
:1028100024E630E040E050E00E94C0D5DA01C90172
:1028200087569F4FAF4FBF4F08958FEF9FEF08958B
:10283000DC01ED91FC91309729F090859F7081E04B
:10284000953009F080E00895FC01A481B5811097CE
:1028500021F118969C9118979F708EEF890F823006
:1028600010F091111AC019964D935D936D937C935E
:102870001C97A481B58118969C911897907F9260BF
:1028800018969C930480F581E02D8085982F907F89
:10289000903619F48F70806A80870895DC0119964C
:1028A0008D919C91009739F0DC01ED91FC910280B3
:1028B000F381E02D199408958AE090E0089581E075
:1028C00090E0089588E090E00895DC01ED91FC919E
:1028D000008CF18DE02D1994CF93DF93EC01E8810A
:1028E000F9810484F585E02D199529893A892F5FAE
:1028F0003F4F3A8B298BDF91CF910895CF93DF9390
:10290000EC018E8581110DC081E090E049895A89E2
:102910002C853D854217530708F080E0DF91CF9169
:102920000895E881F9810484F585E02DCE0119959B
:102930008F3F910549F780E090E0F0CFFC0184855E
:1029400095856817790708F4CB01928B818B0895E0
:10295000DC011E962C911E97222339F0ED91FC91FB
:102960000190F081E02D6FEF19940895FC018785A7
:102970009089089581E0089590E080E00895FC0139
:1029800022813381232B49F0868197818130910503
:1029900039F01CF00397039730F090E080E0089541
:1029A00081E090E0089582E090E00895CF93DF9376
:1029B000CDB7DEB760970FB6F894DEBF0FBECDBFC0
:1029C00019821A821B821C821D821E821F82188617
:1029D0008A818F708A836FEF70E0CE0101960E942A
:1029E000AD1260960FB6F894DEBF0FBECDBFDF917B
:1029F000CF910895CF92DF92EF92FF920F931F93A2
:102A0000CF93DF93CDB7DEB760970FB6F894DEBFF4
:102A10000FBECDBF7C016B01BA01A901CE010196A9
:102A20000E945611D701ED91FC910288F389E02DA7
:102A30009801AE014F5F5F4FB601C70119956096CF
:102A40000FB6F894DEBF0FBECDBFDF91CF911F91BF
:102A50000F91FF90EF90DF90CF90089590E080E08D
:102A60000895CF92DF92EF92FF920F931F93CF932F
:102A7000DF9300D000D0CDB7DEB78C016B017A01B7
:102A8000FC01808D883010F40E948A9482E394E0E7
:102A90009A838983F60182819381A481B5818B8396
:102AA0009C83AD83BE83B701CE0101960E9411A421
:102AB000F801808F8830A0F4F586E486128E118E9E
:102AC00081E026960FB6F894DEBF0FBECDBFDF9132
:102AD000CF911F910F91FF90EF90DF90CF900895CD
:102AE00080E0EFCFCF93DF93EC01888D883020F426
:102AF0000E948A9488E0888FDF91CF910895FC012D
:102B0000808D883040F4218D328D232B21F00E945E
:102B10005C9390E008958FEF9FEF0895CF93DF933C
:102B2000FC012485283028F08FEF9FEFDF91CF91B3
:102B30000895EC010190F081E02D0084F185E02DF5
:102B40001995892B89F38C850E945C9390E0EECFD8
:102B5000CF93DF93FC01218D328D2115310529F4AE
:102B60008FEF9FEFDF91CF910895EC01808D421799
:102B7000530708F0A9010E94AB931816190684F7B1
:102B8000298D3A8D281B390B3A8F298FEBCF0F9364
:102B90001F93CF93DF931F92CDB7DEB7FC01218D3A
:102BA000328D232B41F48FEF9FEF0F90DF91CF9168
:102BB0001F910F9108958C0141E050E0BE016F5FBD
:102BC0007F4FFC01808D0E94AB93181619065CF7AD
:102BD000F801818D928D0197928F818F898190E08C
:102BE000E4CFCF93DF931F92CDB7DEB741E050E043
:102BF000BE016F5F7F4FFC0184850E94AB93181666
:102C0000190634F4898190E00F90DF91CF910895F7
:102C10008FEF9FEFF9CFFC018485883010F40C947E
:102C2000AB9390E080E00895FC018485883010F437
:102C30000C94849390E080E008950F931F93CF93BA
:102C4000DF9300D000D01F921F92CDB7DEB78C016A
:102C5000D80159964D915C915A974115510551F003
:102C6000ED91FC91048CF58DE02D70E060E0C801E1
:102C70001995EECFF801808D0E948493892BB1F1D4
:102C800048E050E0BE016F5F7F4FD80158968C91AD
:102C90000E94AB9318161906F4F4D801509684E0FC
:102CA000FE01319601900D928A95E1F78D8190E0B9
:102CB000982F88272E81820F911DF801958B848B88
:102CC0008F81282F30E0322F22278885820F932F83
:102CD000911D928F818F28960FB6F894DEBF0FBE9C
:102CE000CDBFDF91CF911F910F91089590E080E0CB
:102CF000F2CFCF92DF92EF92FF920F931F93CF9379
:102D0000DF93CDB7DEB7AF970FB6F894DEBF0FBE37
:102D1000CDBF7C016A0102E314E01A8309831C869B
:102D20001B8688EE93E0A0E0B0E08D879E87AF879A
:102D3000B88B88E094E09A878987188F0F8B198E5B
:102D40001A8E1B8E1C8E88E089A31BA70AA71CA6BF
:102D50001DA61EA61FA68091600D9091610DA091E9
:102D6000620DB091630D8EA39FA3A8A7B9A78B8313
:102D70009C83AD83BE8318861F82AE01465D5F4F84
:102D8000CE0101960E9407AA81309105B1F4D701C6
:102D9000ED91FC910488F589E02D1DA30CA38CA571
:102DA0009DA5AEA5BFA58EA39FA3A8A7B9A7A60161
:102DB000BE016C5D7F4FC7011995AF960FB6F894B1
:102DC000DEBF0FBECDBFDF91CF911F910F91FF905E
:102DD000EF90DF90CF9008950F931F93CF93DF93E1
:102DE000EC018B01888D883010F40E948A94B80120
:102DF00082E00E94D394888F883050F41D870C871E
:102E00001A8E198E81E0DF91CF911F910F91089555
:102E100080E0F9CF0F931F93CF93DF938C01EA01EA
:102E2000FC018485883048F40E94FA92892B39F499
:102E300081E090E0F80193838283D0E0C0E0CE018E
:102E4000DF91CF911F910F910895EF92FF920F9311
:102E50001F93CF93DF937C018091CF09D4E083331C
:102E600009F0D8E00FEB19E0C0E0F80121913191B1
:102E70008F01F701848195812817390729F0CF5FE9
:102E8000DC13F3CF80E006C08C2F0E94989484312D
:102E9000B1F781E0DF91CF911F910F91FF90EF90FB
:102EA0000895CF93DF93EC018C858830D0F40E9495
:102EB0009894843189F0882379F0883169F021E091
:102EC0008C3159F4E881F9810084F185E02DCE013F
:102ED000199521E0892B09F420E0822FDF91CF9111
:102EE000089580E0FBCFCF92DF92EF92FF920F9395
:102EF0001F93CF93DF93CDB7DEB7AF970FB6F8949C
:102F0000DEBF0FBECDBF8C016B017A0182E394E07E
:102F10009A8389831B821C821D821E821C861B86CB
:102F200048EE53E060E070E04D875E876F87788BF6
:102F300028E034E03A872987988F8F8B198E1A8E74
:102F40001B8E1C8E28E029A39BA78AA71CA61DA662
:102F50001EA61FA6D8011C968C91883060F40E9492
:102F60009894882321F0F80184850E947C9488E05D
:102F7000D8011C968C938091600D9091610DA09169
:102F8000620DB091630D8EA39FA3A8A7B9A78B83F1
:102F90009C83AD83BE8318861F82AE01465D5F4F62
:102FA000B601CE0101960E9407AA0097C1F0D80190
:102FB000ED91FC910684F785E02D82E394E09DA3DA
:102FC0008CA38CA59DA5AEA5BFA58EA39FA3A8A7E6
:102FD000B9A7A701BE016C5D7F4FC8011995AF96D7
:102FE0000FB6F894DEBF0FBECDBFDF91CF911F911A
:102FF0000F91FF90EF90DF90CF9008950F931F9364
:10300000182F0E9414A704C0969587957795679509
:103010001A95D2F78B019C01015011092109310940
:103020000E3F1F4F2F4F3F4F20F061E070E080E0D8
:1030300090E01F910F910895CF93DF93EC018C8561
:10304000883060F40E949894873111F08C3131F40B
:103050008C850E94DD928115984088F3DF91CF9195
:103060000895FC018485883010F40C94DD9290E082
:1030700080E0089562E576E18BE19FE00E94C286E0
:103080008BE19FE00E942C851092C0071092BF0731
:1030900081E090E0089564E574E18BE19FE00E9497
:1030A000C2868BE19FE00E942C851092F806109258
:1030B000F70681E090E0089564E370E1811102C0B9
:1030C00066E370E18AEE9DE00C94C28660E77EE0E4
:1030D0008AEE9DE00E94C286F0E0E0E0199584EF60
:1030E00091E0089567E479E0811102C062E479E03B
:1030F0008BE19FE00C94C2864F925F926F927F9219
:10310000AF92BF92DF92EF92FF920F931F93CF93F4
:10311000DF9300D000D0CDB7DEB77C01D62E8091F2
:103120001708882309F4BEC0D70114969C9180919A
:103130002A02891708F4B6C08091150890911608E4
:10314000BAE06B13F0C08B53984FFC011082D7018B
:1031500018960D911C910115110509F49FC0F801F5
:10316000618572856115710591F44580568067808F
:10317000708480915A0D90915B0DA0915C0DB0917F
:103180005D0D481659066A067B0609F487C0D8010A
:103190001B964D915C911C974115510509F47EC019
:1031A000F701248153968C91539790E0322F37701A
:1031B00002C0959587953A95E2F780FF6FC0A22EE1
:1031C000B12CC501887F9370892B39F451968D916C
:1031D0009C91887F9370A82AB92AD8018D919C91DF
:1031E000DC01ED91FC916115710509F486C006883A
:1031F000F789E02D1995019709F050C06CE3F801AB
:10320000808191810E94CB85A50170E060E02AE079
:10321000D8018D919C910E94E084F80122818081E7
:1032200091816AE677E1222311F068E677E10E9456
:10323000C286D8011D966D917C911E978D919C91AF
:103240000E945C8660E2F801808191810E94CB85BA
:10325000D8011F966D917C9150978D919C910E9401
:103260005C86F8012281808191816DE577E12223DE
:1032700011F067E577E10E94C28665EC77E0D8013E
:103280008D919C910E945C86F80180819181DC0186
:10329000ED91FC91008CF18DE02D1995109216089E
:1032A00010921508D70115968D919C91169700974D
:1032B00009F44DC014963C9120912B02231708F479
:1032C00046C0DC01ED91FC910190F081E02D6D2D67
:1032D000199526960FB6F894DEBF0FBECDBFDF91CD
:1032E000CF911F910F91FF90EF90DF90BF90AF9023
:1032F0007F906F905F904F9008950488F589E02D3E
:1033000022E334E03A832983D80115964D905D90ED
:103310006D907C9018974B825C826D827E82BE019C
:103320006F5F7F4F67CF8F3491050CF0BBCFBDE04F
:103330006B1709F4B7CF9C012F5F3F4F30931608EE
:10334000209315088B53984FFC016083ABCF81E02D
:1033500090E0BFCF0C94DEC80C94DEC80C94DEC89D
:103360000C94DEC80C94DEC8CF93C1E068EE73E025
:1033700080E090E00E94E2A64AE050E06C2F8AEEE6
:103380009DE00E943085CF5FC43181F784EF91E0EA
:10339000CF910895CF93DF93009709F484C0FC0187
:1033A0002081222309F47FC0EC0168EE79E00E94BD
:1033B0007ECB892B09F456C06FEB79E0CE010E94D9
:1033C0007ECB892B09F451C06EE777E0CE010E94D5
:1033D0007ECB892B09F44CC06AE777E0CE010E94CE
:1033E0007ECB892B09F447C066E777E0CE010E94C7
:1033F0007ECB892B09F442C062E777E0CE010E94C0
:103400007ECB892BF1F16EE677E0CE010E947ECB78
:10341000892BD1F16AE677E0CE010E947ECB892B21
:10342000B1F165E677E0CE010E947ECB892B91F168
:1034300061E677E0CE010E947ECB892B71F16CEEC4
:1034400079E0CE010E947ECB892B51F16DE577E0CA
:10345000CE010E947ECB892B31F58EE090E0DF918A
:10346000CF91089582E090E0FACF81E090E0F7CF2D
:1034700088E090E0F4CF85E090E0F1CF86E090E046
:10348000EECF87E090E0EBCF89E090E0E8CF8AE0F4
:1034900090E0E5CF8BE090E0E2CF8CE090E0DFCFF2
:1034A0008DE090E0DCCF90E080E0D9CFCF93DF9348
:1034B000EC016DED76E18BE19FE00E94C2866C81AC
:1034C0007D818BE19FE00E94879967ED76E18BE13A
:1034D0009FE00E94C2868BE19FE00E942C8560E005
:1034E0008C810E948AA51092C4071092C30781E0C4
:1034F00090E0DF91CF910895EF92FF921F93CF93C9
:10350000DF93192F7B01C82FD92FD7FF03C0D19587
:10351000C195D10961E08C2F0E948AA582E0E8164E
:10352000F10499F460E08C2F0E945CA56CE373E1D8
:103530008BE19FE00E94C2868BE19FE0DF91CF91FB
:103540001F91FF90EF900C942C85612FEF2851F480
:103550006095661F6627661F8C2F0E945CA568E336
:1035600073E1E6CF661F6627661F8C2F0E945CA55D
:1035700063E373E1DDCFCF93DF93EC01FB012481A3
:10358000358140815181628173810E94D285CE0153
:10359000DF91CF910895EF92FF920F931F93CF93F6
:1035A000DF93EC018B011D821C821A821B82E88052
:1035B000F980E114F10409F45DC08091F206909164
:1035C000F306892B09F456C0672B09F48701F8012B
:1035D00080858F708630A9F460E474E0C8010E9491
:1035E0000599009719F0FC0181858A8369EC76E0E2
:1035F000C8010E940599009709F443C0FC01818528
:103600008B8362E474E0C7010E940599009779F505
:1036100065E177E08BE19FE00E94C2864AE050E0DE
:103620006B818BE19FE00E94308563E177E08BE165
:103630009FE00E94C2864AE050E06A818BE19FE0F1
:103640000E9430858BE19FE00E942C8520E030E0D5
:10365000A90162E474E0888199810E94BA9D62E4C4
:1036600074E0888199810E940599009719F0099664
:103670009D838C83DF91CF911F910F91FF90EF90ED
:103680000895F801808191810E9412CBB9CFCF9328
:10369000DF9300D000D01F921F92CDB7DEB7E5EDCB
:1036A000FDE0128A118A80E090E19587848784E8A2
:1036B00090E0948B838B81E0868780E090E2908B12
:1036C00087871C821B8282E293E09A838983FE8330
:1036D000ED838FEF9FEF98878F836FEB73E18AEE17
:1036E0009DE00E94C2866091F2067091F306CE01C1
:1036F00001960E94C68C85ED9DE00E9465146FEADC
:1037000073E18AEE9DE00E94C2868AEE9DE00E94EF
:103710002C850E94B6AC28960FB6F894DEBF0FBE7B
:10372000CDBFDF91CF910895FC01868197810097ED
:1037300099F0FC0120852F70223029F46185728573
:10374000838594850895253039F460E00E947A9944
:10375000009711F0FC01F2CF60E070E0CB0108951A
:103760000F931F93CF93DF93FC01C281D3812097E6
:10377000F9F088858F70823049F4672BC9F4898508
:103780009A85DF91CF911F910F910895853081F433
:103790008B01CE010E948F998017110649F044F0E9
:1037A000602FCE010E947A99FC0181859285E9CF34
:1037B00090E080E0E6CFFC016115710519F4848189
:1037C0009581089586819781681779072CF0848107
:1037D0009581860F971F0895828193810C94B01B69
:1037E000CF93DF93EC0164EB76E18BE19FE00E94E5
:1037F000C2866C817D818BE19FE00E9487996EEA91
:1038000076E18BE19FE00E94C2868BE19FE00E94FF
:103810002C85E881F981028CF38DE02DCE0119957C
:103820008130910529F0029759F060E08C811AC02F
:1038300063E070E0CE010E94DB1B60E00E948AA57D
:1038400060E08C810E948AA561E070E0CE010E9458
:10385000DB1B60E00E948AA562E070E0CE010E945E
:10386000DB1B60E00E948AA51092C2071092C1077C
:1038700081E090E0DF91CF910895CF93DF93EB014A
:1038800063E0FC01808191810E947A99FC01892B7F
:10389000A9F080858D7091F4C095D095CF6FAE0161
:1038A00070E060E081859285A385B4858C239523A3
:1038B000A623B72381879287A387B487DF91CF910F
:1038C0000895CF93DF93EB0163E0FC018081918148
:1038D0000E947A99FC01892BB9F09085892F8D700F
:1038E00099F4907F92609087CC27CE01B0E0A0E061
:1038F0004185528563857485842B952BA62BB72B28
:1039000081879287A387B487DF91CF910895CF9362
:10391000DF93EB0163E0FC01808191810E947A9941
:10392000009761F0FC0120852F70223039F48185E9
:1039300092858C239D23DF91CF91089590E080E0C4
:10394000FACFCF93C62F63E0FC01808191810E9462
:103950007A99FC01892B29F19085892F8D7009F5C1
:10396000907F9260908781859285A385B485882712
:10397000AA27BB278C2B81879287A387B48763E80C
:1039800077E08BE19FE00E94C2864AE050E06C2F16
:103990008BE19FE00E9430858BE19FE0CF910C94FA
:1039A0002C85CF91089563E0FC01808191810E9474
:1039B0007A99009719F0FC01818508958FEF089599
:1039C000FF920F931F93CF93DF93CDB7DEB764972A
:1039D0000FB6F894DEBF0FBECDBF8C01F62E8FE27E
:1039E00090E09A838983FE01339688E0DF011D927F
:1039F0008A95E9F7F8016681FF2011F081E06827D8
:103A0000D80114968C910E945CA5F801878190855D
:103A1000A185B285883E9340A105B10508F48BC00D
:103A200063E277E18BE19FE00E94C286D8011496A1
:103A30006D917C918BE19FE00E9487996EE177E127
:103A40008BE19FE00E94C2866F2D70E08BE19FE0CA
:103A50000E9487998BE19FE00E942C8565E477E1C5
:103A6000CE0101960E9473CBF801828193810E945E
:103A7000D31CFF2009F46BC06BE077E18D3051F06F
:103A80006FE077E18E3031F066E177E18B3011F055
:103A900063E077E1CE010B960E9487CB6EEE76E174
:103AA0008BE19FE00E94C286D8011296ED91FC91B5
:103AB00013970190F081E02D60817181ED91FC916F
:103AC0000288F389E02D9E012F5F3F4FAE01455FD5
:103AD0005F4FC8011995BC018BE19FE00E94879957
:103AE0006CEE76E18BE19FE00E94C286D8011296CF
:103AF000ED91FC910190F081E02D608171818BE16D
:103B00009FE00E945C86BE016F5F7F4F8BE19FE06C
:103B10000E945C8669EE76E18BE19FE00E94C2869E
:103B2000BE01655F7F4F8BE19FE00E945C868BE169
:103B30009FE00E942C8564960FB6F894DEBF0FBEFE
:103B4000CDBFDF91CF911F910F91FF9008956FEF3F
:103B500076E1823009F49ECF6AEF76E19BCF81E077
:103B600090E00895CF93DF93EC0164EA76E18BE176
:103B70009FE00E94C2866C817D818BE19FE00E9464
:103B800087996EE976E18BE19FE00E94C2868BE126
:103B90009FE00E942C858A819B81892B09F44DC06E
:103BA0008C819D81892B09F048C0E881F981028CC4
:103BB000F38DE02DCE0119958130910529F0029702
:103BC00059F061E08C811AC063E070E0CE010E9480
:103BD000DB1B61E00E948AA561E08C810E948AA5BE
:103BE00061E070E0CE010E94DB1B61E00E948AA5CB
:103BF00062E070E0CE010E94DB1B61E00E948AA5BA
:103C00008091A100887F8093A10080919100887F9E
:103C1000809391008091A10082608093A1008091A7
:103C2000910082608093910081E090E09093C207C0
:103C30008093C107DF91CF91089590E080E0FACFA3
:103C4000CF93DF93DC011496ED91FC91309709F44A
:103C50004FC0C681D7812097C1F1E881F9813097A3
:103C600081F18081882369F16BED74E0CE010E94BF
:103C70000599892B41F42FEF3FEFA9016BED74E01B
:103C8000CE010E94BA9D6CEE74E0CE010E940599AF
:103C9000892B41F42FEF3FEFA9016CEE74E0CE01C8
:103CA0000E94BA9D65E474E0CE010E940599892BBB
:103CB00041F42FEF3FEFA90165E474E0CE010E94CB
:103CC000BA9D0A80DB81C02DC6CF63E476E18BE12B
:103CD0009FE00E94C2868BE19FE00E942C8581E0DC
:103CE00090E09093C0078093BF07DF91CF91089534
:103CF0006BE276E18BE19FE00E94C2868BE19FE060
:103D00000E942C8590E080E0F0CF6CE474E18BE1C0
:103D10009FE00E94C2868BE19FE00E942C8526E0F6
:103D200040E855E260E070E082EE99E00E94798B15
:103D300081E090E09093F8068093F7060895892B30
:103D400071F0FB01828193810E94AC9A6DEA7FE061
:103D50008AEE9DE00E94C28688EC90E0089590E093
:103D600080E0F2CF892B71F0FB01828193810E9468
:103D7000499A66E97FE08AEE9DE00E94C28688EC5F
:103D800090E0089590E080E0F2CF8091C70D90918F
:103D9000C80D892B51F00E94E0AD882331F066E810
:103DA0007FE08AEE9DE00E94C2861092E70D10929D
:103DB000E60D80E090E19093E20D8093E10D84E8C0
:103DC00090E09093E90D8093E80D81E08093E30DFE
:103DD00080E090E29093E50D8093E40D85ED9DE009
:103DE0000E94A81485ED9DE00E94651488EC90E087
:103DF0000895EF92FF920F931F93CF93DF93CDB768
:103E0000DEB72C970FB6F894DEBF0FBECDBF8C0186
:103E10007B0182E394E09A8389831B821C821D824A
:103E20001E8298878F8319861A861B861C8605300A
:103E30001105ECF0BE01695F7F4FF7018085918528
:103E40000E94AD11892B99F0CE0107960E947A9BB2
:103E5000BE01695F7F4FF701868197810E94AD1196
:103E6000892B61F0CE0107960E94509C0EC0CE01B6
:103E700001960E947A9B0430110554F7CE010196F9
:103E80000E94509C033011058CF1BE01695F7F4F89
:103E9000F701848195810E94AD11892B39F1CE0102
:103EA00007960E94E59BBE01695F7F4FF701828103
:103EB00093810E94AD11892B01F1CE0107960E94DA
:103EC0000F9B6FE67FE08AEE9DE00E94C28688EC41
:103ED00090E02C960FB6F894DEBF0FBECDBFDF91F9
:103EE000CF911F910F91FF90EF900895CE01019611
:103EF0000E94E59B02301105B4F6CE0101960E94A6
:103F00000F9B01301105E9F6CE0101960E940F9B2F
:103F100066E77FE08AEE9DE00E94C286D2CF0F93D3
:103F20001F93CF93DF938C01EB010297C4F08A813A
:103F30009B810E9412CB80932B0299270E94889D1F
:103F40000230110549F08C819D810E9412CB809333
:103F50002A0299270E94929DC8ECD0E002C0C0E9D5
:103F6000D1E06BE57FE08AEE9DE00E94C2864AE0E8
:103F700050E060912B028AEE9DE00E94308566E45D
:103F80007FE08AEE9DE00E94C2864AE050E06091A8
:103F90002A028AEE9DE00E9430858AEE9DE00E9412
:103FA0002C85CE01DF91CF911F910F910895CF9372
:103FB000DF93EB010297A4F161E370E18A819B81B9
:103FC0000E9460CB892B29F40E94BB9C6F770E94D2
:103FD000189D6DE270E18A819B810E9460CB892BE4
:103FE00029F40E94BB9C60680E94189D65E37FE0F5
:103FF0008AEE9DE00E94C2860E94BB9C6095661F6F
:104000006627661F70E08AEE9DE00E9487998AEE1F
:104010009DE00E942C8588EC90E0DF91CF9108957F
:104020000E94471BF8CF2F923F924F925F926F9260
:104030007F928F929F92AF92BF92CF92DF92EF9238
:10404000FF920F93CF93DF9300D01F92CDB7DEB7CF
:104050007C017A8369835C834B83DB011C92FC01C6
:104060006081662309F44DC030FF4BC0F9E06F9FBB
:10407000B00111246757704ECD010E94B5CBD70116
:1040800011968C91807F41F04B815C8169E474E0F2
:1040900089819A810E949ADAE981FA81019000204F
:1040A000E9F7319789819A81E81BF90B1C012E0EE3
:1040B0003F1EAB81BC81AE1BBF0B1197BC83AB8392
:1040C000D7011196EC9111978E2F807F09F4BCC017
:1040D000E295EF70E150EC3008F0B6C0F0E08827D0
:1040E000EB58FF4D8F4F0C9429D68420F320592193
:1040F000BE21D921C0206F216F216F21B420A820BB
:10410000F52129803A80DCCFF7018481282F30E027
:1041100050E040E0002359F030E0A4E6B0E00E9417
:10412000F2D52FEF30E040E050E00E94C0D55F9321
:104130004F933F932F938BE494E09F938F93FC8155
:10414000FF938B818F933F922F920E94D2DA77C098
:10415000F70187818F9386818F9385818F938481E7
:104160008F938EE494E0E9CFF70187818F93868166
:104170008F9385818F9384818F9382E594E0DDCF47
:10418000F701C480D580E680F780C701B60124E638
:1041900030E040E050E00E94C0D597FF07C0909506
:1041A0008095709561957F4F8F4F9F4F9F938F9311
:1041B0007F936F93C701B60124E630E040E050E002
:1041C0000E94C0D55F934F933F932F9386E594E071
:1041D0009F938F93FC81FF938B818F933F922F92BC
:1041E0000E94D2DA2CC0C7010E94F613BC01F7016D
:1041F000C680D780D0FADD24D0F89481F580EB809A
:10420000BC80292F30E050E040E077FD35C001113F
:1042100035C07F936F931F921F921F929F931F929F
:10422000FF92DF92CF928FE594E09F938F939C81D2
:104230009F93AB81AF933F922F920E94D2DA0FB639
:10424000F894DEBF0FBECDBF89819A810F900F9089
:104250000F900F90DF91CF910F91FF90EF90DF9033
:10426000CF90BF90AF909F908F907F906F905F9016
:104270004F903F902F900895002361F0292F30E058
:10428000A4E6B0E00E94F2D52FEF30E040E050E02D
:104290000E94C0D55F934F933F932F931F92FF923D
:1042A000DF92CF9282E694E09F938F93BF92EF923A
:1042B00095CF15968C9115971F928F9316969C917A
:1042C000169717968C9181708F939F9385E694E053
:1042D0009F938F93BC81BF93EB81EF9334CF149660
:1042E0008D909D90AD90BC90179720E030E0A90193
:1042F000C501B4010E9454D42401350187FF04C0D4
:1043000077FA709477F87094C301B2010E9426D7AF
:104310006B01072E000C880B990B0E945BD49B014C
:10432000AC01C301B2010E9447D620E030E04AE769
:1043300054E40E94BAD40E94B1D70E9426D7062F17
:10434000772E20E030E0A901C501B4010E9454D4C9
:1043500087FF07C07F920F93DF92CF928BE694E0A6
:10436000B7CF7F920F93DF92CF928CE694E09F932A
:104370008F939C819F93AB81AF93E5CE14968C91E4
:1043800014971F928F9315968C9115971F928F9368
:1043900016968C911F928F9382E694E09F938F9351
:1043A000BC81BF93EB81EF933F922F920E94D2DAB0
:1043B00046CF17968C9117971F928F9314968C91D6
:1043C00014971F928F9315968C9115971F928F9328
:1043D00016968C911F928F938FE594E09F938F9305
:1043E000BC81BF93EB81EF93F9CE14966D917C91D4
:1043F0004B815C81C1010E94B8DA26CFCF92DF9257
:10440000EF92FF920F931F93CF93DF93EC0188817C
:1044100099810E948F99082F10E0043011059CF4B7
:104420000E94CB8E009739F0DC0118962C911897DA
:10443000207F18962C93BC01888199810E949E9DB3
:104440000F5F1F4FEACFC880D98060E0C6010E948D
:104450007A99FC01F184F88661E0C6010E947A999C
:104460008C019B838A8362E0C6010E947A999D83B6
:104470008C8364E0C6010E947A996C019F838E83CD
:10448000F0E1FF1609F48AC0FF1580F083E0F8160A
:1044900089F1AAE0FA1609F473C0DF91CF911F9158
:1044A0000F91FF90EF90DF90CF900895B2E1FB164F
:1044B00009F4F3C0E3E1FE12F0CF86E090E00E9441
:1044C00042C8FC01D383C2838CE392E09183808352
:1044D000C114D10409F4FCC0D60118968C91189728
:1044E0008F70823009F0F4C016968D919C9195835F
:1044F0008483EBC08AE090E00E9442C87C01DC012A
:104500001396DC93CE9312978EE592E08D939C9355
:1045100070E060E0CE010E94B01B97FD22C0F70161
:10452000958384830115110541F1F80180858F7011
:10453000823001F1853009F5C8010E948F9990E021
:10454000D70117969C938E93169782E892E0119666
:104550009C938E9319961C921E921897FA86E98660
:104560009CCF919581959109D70115969C938E9337
:104570001497D8CF81E090E0E3CF90E080E0E0CFE7
:1045800084E090E00E9442C8FC01D383C2832AEEFB
:1045900032E0318320839A8789877FCF8BE090E058
:1045A0000E9442C87C01DC011396DC93CE931297E3
:1045B00088EC92E011969C938E9316961C9270E074
:1045C00060E0CE010E94B01B97FD46C0F7019583C5
:1045D0008483F70184819581009719F086359105D0
:1045E0003CF080E290E0D70115969C938E9314974F
:1045F0000115110509F443C0F80180858F708530DD
:10460000F1F5C8010E948F998230C8F161E0C801BC
:104610000E947A99FC01892B91F180858F708230FC
:1046200039F561857285838594850E945BD420E08D
:1046300030E04AE754E40E94BAD40E942DD76115B5
:10464000710581059105F9F0D70117966D937D935A
:104650008D939C931A9782CF919581959109D7015B
:1046600015969C938E93149781E016968C93B1CFF8
:10467000833029F46185728583859485D8CF60E085
:1046800070E0CB01D4CF88E893E1A0E0B0E0F7017F
:1046900087839087A187B28761CF86E090E00E94F0
:1046A00042C8FC01D383C28386EA92E0918380836F
:1046B000158214820115110541F0D80118968C91CC
:1046C0008F70863011F415830483FA87E987E5CE6D
:1046D00090E080E00CCFCF93DF93EC017983688387
:1046E0001A8619861B861C8E1B8E0E94181488231E
:1046F00029F0CE01DF91CF910C94FE21DF91CF9173
:104700000895EF92FF920F931F93CF93DF93EC01E5
:104710007B018E819F81892BD9F4888199810E94A8
:104720008F99082F10E00530110594F40E94CB8E6C
:10473000009721F0FC012085207F20879F838E83B6
:10474000BC01888199810E949E9D0F5F1F4FEBCF16
:10475000EE81FF813097D9F08085982F9F70A9F462
:10476000807F82608087EE81FF81118612861386AA
:104770001486EE81FF81F782E682C701DF91CF9137
:104780001F910F91FF90EF900895923061F3F12CFB
:10479000E12CF3CFCF93DF93EC016CE775E18BE174
:1047A0009FE00E94E6868C819D810E94DEC870E0B9
:1047B00060E08A819B810E9481231D821C8281E0AE
:1047C00090E0DF91CF910895CF92DF92EF92FF9228
:1047D0000F931F93CF93DF93EC018C819D81892BE5
:1047E00061F40A811B8185E090E00E9442C8BC010F
:1047F000C8010E9481239D838C83EC80FD80E1149D
:10480000F104A9F464E675E184EF9DE00E94C2869C
:1048100084EF9DE00E942C8590E080E0DF91CF91B5
:104820001F910F91FF90EF90DF90CF90089510921D
:10483000BA071092B9071092B4071092B3071092FA
:10484000BB071092BC071092BD071092BE071092D2
:10485000B5071092B6071092B7071092B8071092DA
:10486000310710927307EA81FB81309759F08281FA
:104870009381009739F0DC0118962C912F70263027
:1048800009F468C06DE175E184EF9DE00E94C28685
:1048900061E070E08C819D81892B11F470E060E013
:1048A00084EF9DE00E9487996BE175E184EF9DE0C4
:1048B0000E94C28661E070E08A819B81892B11F49D
:1048C00070E060E084EF9DE00E94879969E175E106
:1048D00084EF9DE00E94C286EA81FB8161E070E086
:1048E00082819381892B11F470E060E084EF9DE078
:1048F0000E94879967E175E184EF9DE00E94C2867E
:10490000EA81FB810280F381E02D80858F7061E078
:1049100070E0863011F470E060E084EF9DE00E946A
:10492000879965E175E184EF9DE00E94C28684EF7E
:104930009DE00E942C8566E375E184EF9DE00E9476
:10494000C28684EF9DE00E942C85EC81FD8182E08F
:10495000808362CF64E774E00E940599009709F4B0
:10496000A8C0FC0120852F70243009F0A2C0C184AA
:10497000D284B6018BE19FE00E945C8661E175E123
:104980008BE19FE00E94C28610E000E0C114D104D8
:1049900009F486C0B80167537B4EC6010E947ECBE6
:1049A000892B09F077C0F801E353FB4E2591349130
:1049B000922F832FD70113969C93139714968C9361
:1049C000EA81FB816BE774E0828193810E94059903
:1049D000EC81FD81009709F472C0DC0118962C91DE
:1049E00018972F70223009F06AC019964D915D9189
:1049F0006D917C911C97411551056105710509F474
:104A00005EC05283418341815281052E000C660BAA
:104A1000770B23818CE19CE00E94798BEC81FD81F6
:104A200041815281052E000C660B770B23818FEF9D
:104A30009AE00E94798BEA81FB8161E075E08281D6
:104A400093810E940599009739F0FC018185928538
:104A500090937207809371076CE475E18AEE9DE094
:104A60000E94C286EA81FB810190F081E02D608185
:104A700071818AEE9DE00E945C868AEE9DE00E9434
:104A80002C85EC81FD8181E080838093290281E087
:104A900090E0C4CE0A5F1F4F0834110509F076CFAD
:104AA0006CEA74E18BE19FE00E94C28696E080E0B0
:104AB00081CF86E090E0F7019483838381CF80E00B
:104AC0009BE4928381839FCFCF92DF92EF92FF92FC
:104AD0000F931F93CF93DF93EC016A017B018E81CB
:104AE0009F81892BD9F4888199810E948F99082F01
:104AF00010E00530110594F40E94CB8E009721F050
:104B0000FC012085207F20879F838E83BC018881C4
:104B100099810E949E9D0F5F1F4FEBCFEE81FF8119
:104B2000309749F18085982F9F7019F5807F8260BA
:104B30008087EE81FF81C186D286E386F4866BE8AA
:104B400077E08BE19FE00E94C2862AE030E0B70167
:104B5000A6018BE19FE00E94D2858BE19FE0DF916F
:104B6000CF911F910F91FF90EF90DF90CF900C9419
:104B70002C859230F1F2DF91CF911F910F91FF9030
:104B8000EF90DF90CF900895EF92FF920F931F93D5
:104B9000CF93DF93EC017B018A0101501109A80139
:104BA00082EE99E00E94017CF701329660E0CF012D
:104BB0008E199F098017910718F48191680FF7CF1C
:104BC00082EE99E00E94CE7C0A80DB81C02D80E0DD
:104BD0000E94FE17AB01BC01CE010E94642560E873
:104BE00074E08BE19FE00E945C86E701CE018E19A4
:104BF0009F0980179107A0F4688140E150E06A3076
:104C000048F469E874E08BE19FE00E945C8640E133
:104C100050E068818BE19FE00E9430852196E6CFCD
:104C20008BE19FE0DF91CF911F910F91FF90EF906B
:104C30000C942C851F93CF93DF93FC01162FC3890F
:104C4000D489818992899C012F5F3F4F328B218BC0
:104C5000C80FD91FCE010E9478D5181721F0612FF7
:104C6000CE010E9480D581E090E0DF91CF911F912D
:104C70000895FC01818992892485358582179307DF
:104C800040F423893489820F931F0E9478D590E0E5
:104C900008958FEF9FEF08952F923F924F925F926A
:104CA0006F927F928F929F92AF92BF92CF92DF923C
:104CB000EF92FF920F931F93CF93DF93CDB7DEB7A1
:104CC00062970FB6F894DEBF0FBECDBF5C014B01FB
:104CD00029013A01CA01B9010E9426D71B013F925E
:104CE0006F9388E694E09F938F93CE0101967C01A9
:104CF0009F938F930E940FDB0F900F900F900F9058
:104D00000F900F9020E030E0A901C301B2010E9492
:104D10005CD7181624F077FA709477F87094F7013E
:104D200001900020E9F731976F01CE18DF088EE27D
:104D30008083A2E0B0E0AC0FBD1FAC0DBD1DBA8BEF
:104D4000A98BB10137FE03C0719561957109072EDA
:104D5000000C880B990B0E945BD49B01AC01C30132
:104D6000B2010E9447D620E030E040E251E40E94C8
:104D7000BAD40E9426D7605DE989FA896083FE0172
:104D8000EC0DFD1D1382D501ED91FC910288F38994
:104D9000E02D9801A701B401C501199562960FB6DF
:104DA000F894DEBF0FBECDBFDF91CF911F910F9161
:104DB000FF90EF90DF90CF90BF90AF909F908F903B
:104DC0007F906F905F904F903F902F900895DA0101
:104DD000E0918608F0E0FE2FEE27E60FF71F90E047
:104DE000982F8827A901BD018E0F9F1F0C944F900B
:104DF000CF93DF931F92CDB7DEB72091860830E0C6
:104E0000322F2227260F371F90E0982F88274983BB
:104E100041E050E0BE016F5F7F4F820F931F0E9401
:104E20004F900F90DF91CF910895CF93DF931F9212
:104E3000CDB7DEB741E050E0BE016F5F7F4F0E940B
:104E4000C48F89810F90DF91CF91089520918608BA
:104E500030E0322F2227620F731F90E0982F8827AF
:104E6000860F971F0C94152763E070E00C9426279B
:104E70009F92AF92BF92CF92DF92EF92FF920F93E9
:104E80001F93CF93DF93EC017B018091CF098111B8
:104E900021C01B821A8288EE93E0A0E0B0E08C83F0
:104EA0009D83AE83BF838CEB93E09983888388E0F6
:104EB0008C8788EE93E09E878D87CE01DF91CF911E
:104EC0001F910F91FF90EF90DF90CF90BF90AF9028
:104ED0009F90089534E0932E833311F028E0922EB2
:104EE0008FEBC82E89E0D82E10E098E0B92EA12CC7
:104EF000D6012D913D916D01F7018481958128178F
:104F0000390791F4812F0E949894082F873111F06E
:104F10008C3139F5812F0E948493892B59F50C31FE
:104F200019F4812F0E947C941F5F9112E1CFA11090
:104F300008C0D701ED91FC910084F185E02DC701F7
:104F400019951B821A8288EE93E0A0E0B0E08C8372
:104F50009D83AE83BF838CEB93E099838883BC866B
:104F6000A8CF843149F08111DFCFF6013297118249
:104F70001082DACFB12ED8CFAA24A394D5CF8F92A6
:104F80009F92AF92BF92CF92DF92EF92FF920F93D8
:104F90001F93CF93DF93CDB7DEB72F970FB6F8945B
:104FA000DEBF0FBECDBF5C014B017A018091CF09FE
:104FB0008823C9F104E0833309F008E0B501CE018C
:104FC00001960E9438278FEBC82E89E0D82E10E07A
:104FD000F601219131916F01F501848195812817A6
:104FE000390751F4812F0E949894873129F4A70141
:104FF000B401812F0E94FA921F5F0113E9CFC7010C
:105000002F960FB6F894DEBF0FBECDBFDF91CF91C4
:105010001F910F91FF90EF90DF90CF90BF90AF90D6
:105020009F908F900895F12CE12CE9CFDA01E09167
:105030008608F0E0FE2FEE27E60FF71F90E0982F8E
:105040008827A901BD018E0F9F1F0C94C48F44E0D7
:1050500050E0BC018FE090E00C944F9044E050E0B1
:10506000BC0185E090E00C944F9044E050E0BC011E
:1050700081E090E00C944F9008959F92AF92BF9280
:10508000CF92DF92EF92FF920F931F93CF93DF9314
:105090008C015B01942EE52EFC01C688D788F08C2C
:1050A00080E591E00E944EA28F2D0E94A092C92D12
:1050B000DE2D8C179D0708F4EC019E01A501B601B9
:1050C0008F2D0E941D92F801868997898C0F9D1F54
:1050D000978B868BCE01DF91CF911F910F91FF901F
:1050E000EF90DF90CF90BF90AF909F900895CF93B7
:1050F000FC01C08D80E591E00E944EA260E270E06C
:105100008C2F0E94B48F62E070E08C2F0E942627C3
:1051100084FD16C062E070E08C2F0E94262783FF7A
:105120000AC048E162E070E08C2F0E94F82680E01F
:1051300090E0CF91089580E591E00E944EA2E3CFE8
:1051400040E162E070E08C2F0E94F82681E0F0CF11
:10515000FF920F931F93CF93DF93EB01FC01178A0C
:10516000168A2A81211109C02B81211106C02C81A8
:10517000211103C02D81222301F141155105E9F0D0
:105180008A01FC01F08C80E591E00E944EA2AE0104
:105190004E5F5F4F24E030E06CE070E08F2D0E94A6
:1051A000E726B8018F2D0E94A79481E090E0DF915F
:1051B000CF911F910F91FF90089580E0F7CF0F934B
:1051C0001F93CF938C01FC016481758181E20E9461
:1051D000D394C82F8830F8F480E591E00E944EA265
:1051E0008C2F0E943427833131F08C2FCF911F9167
:1051F0000F910C947C9462E070E08C2F0E94B48F2D
:10520000F80184819581EC2FF0E0EE0FFF1FE1544F
:10521000F64F91838083CF911F910F9108950F9343
:105220001F93CF93DF931F921F92CDB7DEB7FC0180
:1052300024852830E0F48C0180E591E00E944EA2A4
:1052400022E030E0AE014F5F5F4F60E170E0F801B7
:1052500084850E94162889819A8198278927982712
:105260000F900F90DF91CF911F910F91089590E0D3
:1052700080E0F6CF0F931F93CF93DF931F921F927F
:10528000CDB7DEB7FC0124852830E0F48C0180E541
:1052900091E00E944EA222E030E0AE014F5F5F4FEE
:1052A00064E070E0F80184850E94162889819A8163
:1052B0009827892798270F900F90DF91CF911F9102
:1052C0000F91089590E080E0F6CFCF93DF93EC014B
:1052D00082E394E0998388831A821B821C821D8258
:1052E00080E591E00E944EA2BE016E5F7F4F44E0D8
:1052F00050E08FE090E00E94C48FCE01DF91CF910B
:1053000008950E941091882331F08091CF09843351
:1053100029F0873381F090E080E0089580E591E006
:105320000E944EA285E390E00E94152785FD0DC0E6
:1053300082E090E0089580E591E00E944EA28EE226
:1053400090E00E94152780FFF3CF81E090E0089560
:105350001F920F920FB60F9211240BB60F922F933C
:105360003F934F935F936F937F938F939F93AF93ED
:10537000BF93EF93FF938091B900887F803609F443
:105380004DC008F040C0883209F4A7C028F580312C
:1053900009F49BC0C8F4882309F4F7C0883009F4E5
:1053A00094C0FF91EF91BF91AF919F918F917F91A9
:1053B0006F915F914F913F912F910F900BBE0F9086
:1053C0000FBE0F901F901895883109F486C0803267
:1053D00041F780935F0814C0803409F49BC040F407
:1053E0008033B9F38833E9F680935F0885ECAEC06B
:1053F000803509F483C0883509F494C0883489F66F
:105400000E94E510CECF883909F48AC038F5883774
:1054100029F050F4883611F0803719F683E0809334
:10542000600810925E0855C0883809F479C0803948
:1054300019F0803809F0B5CF80915E08803208F00D
:105440006FC0E0915E0881E08E0F80935E088091CE
:10545000BB00F0E0E25CF74F80833BC0803B39F05B
:10546000D0F4803A09F477C0883A09F09ACF84E002
:105470008093600810923D0810923C08F0E0E0E054
:10548000199580913C0881110FC081E080933C0800
:1054900010921C0809C0803C09F4A8CF883C09F48C
:1054A000A5CF883B09F07DCFE0913D0881E08E0FCC
:1054B00080933D08F0E0E45EF74F80818093BB006D
:1054C00090913D0880913C0829C080918508809387
:1054D000BB0085EC8093BC0064CF909184088091E0
:1054E0008308981758F5E091840881E08E0F809327
:1054F0008408F0E0ED59F74F8081E9CFE09184080E
:1055000081E08E0F809384088091BB00F0E0ED591C
:10551000F74F808390918408809183089817C8F290
:1055200085E8D8CFE091840881E08E0F80938408CD
:105530008091BB00F0E0ED59F74F808380916208C5
:1055400081115ECF81E08093610884EA8093BC0082
:105550001092600826CF85EC8093BC001092600802
:1055600080915E08803230F4E0915E08F0E0E25C09
:10557000F74F108260915E0870E08EE398E0F0E0F3
:10558000E0E0199510925E080CCF10925F0838CFBA
:105590004F925F926F927F92AF92BF92CF92DF92C3
:1055A000EF92FF920F931F93CF93DF9300D01F9240
:1055B000CDB7DEB72B013C0129833A834B835C8353
:1055C000A6019501C801B701640D751D861D971DC3
:1055D000211531054105510511F00E949ED5298103
:1055E0003A814B815C816217730784079507D0F479
:1055F000241535054605570530F521E0822F0F901B
:105600000F900F900F90DF91CF911F910F91FF900E
:10561000EF90DF90CF90BF90AF907F906F905F90B2
:105620004F900895461657066806790650F421E013
:1056300089819A81AB81BC8184159505A605B70542
:10564000E8F220E0DBCF21E046165706680679062F
:10565000A8F2F7CF8F929F92AF92BF92CF92DF9234
:10566000EF92FF920F931F93CF93DF9300D000D060
:1056700000D01F92CDB7DEB76130710509F07BC253
:105680004C010E9414A79B01AC016091040770912A
:1056900005078091060790910707A12CB12C6501A1
:1056A00018E8E12E13E1F12E00E010E00E94C82A74
:1056B0008823C1F080E00E94FE1760930407709376
:1056C000050780930607909307076AE774E18BE16B
:1056D0009FE00E94E6864DE050E062E072E0C40187
:1056E0000E94C42582EE99E00E94797C8597ACF4F3
:1056F00081E090E02A960FB6F894DEBF0FBECDBFD2
:10570000DF91CF911F910F91FF90EF90DF90CF909D
:10571000BF90AF909F908F90089545E250E06AE06F
:1057200077E082EE99E00E94AE8482EE99E00E94DA
:10573000797C892B59F062E070E080E090E00E9473
:10574000E2A682EE99E00E94577CEFCF80912E076F
:1057500090910307891761F28093030780912D07C9
:1057600090E09C01205F3F4F3093300720932F073C
:10577000499708F0BDCF8091170790E090930207FA
:10578000809301078091210790E090930007809318
:10579000FF068091230790E09093FE068093FD061C
:1057A0008091250790E09093FC068093FB06809102
:1057B000270790E0909309078093080780912607B8
:1057C00090E09093FA068093F906D401ED91FC9154
:1057D00011970288F389E02D12968D919C91DC013E
:1057E0008D919C91DC016D917C91809129072BE832
:1057F00034E042E954E080FD02C045E954E0C401D0
:1058000019958091F9069091FA0680389105A9F4CE
:10581000D4011296ED91FC9113970190F081E02D47
:1058200060817181ED91FC910288F389E02D29E975
:1058300034E042E954E0C40119958091F906909151
:10584000FA06892BA9F4D4011296ED91FC911397D5
:105850000190F081E02D60817181ED91FC910288D1
:10586000F389E02D29E934E045E954E0C4011995B4
:105870006FE974E08BE19FE00E945C86609108070D
:10588000709109078BE19FE00E9487998BE19FE06F
:105890000E942C8580910807F40120813181A2812A
:1058A000B3810D90BC91A02D6D917C91D901529640
:1058B000ED91FC9126EA34E042E954E083FD02C018
:1058C00045E954E0C4011995D401ED91FC9111977B
:1058D0000288F389E02D12968D919C91DC018D91C7
:1058E0009C91DC016D917C91809108072DEA34E058
:1058F00042E954E081FD02C045E954E0C401199534
:105900002091FB063091FC06032E000C440B550B36
:10591000D4011296ED91FC9113970190F081E02D46
:1059200060817181ED91FC910684F785E02D09EB92
:1059300014E0C40119958091FD069091FE06892B13
:10594000A9F4D4011296ED91FC9113970190F08186
:10595000E02D60817181ED91FC910288F389E02D49
:1059600020EC34E045EC54E0C40119958091FD062B
:105970009091FE060197A9F4D4011296ED91FC9145
:1059800013970190F081E02D60817181ED91FC9180
:105990000288F389E02D20EC34E04AEC54E0C401A5
:1059A00019958091FD069091FE060297A9F4D40105
:1059B0001296ED91FC9113970190F081E02D60819A
:1059C0007181ED91FC910288F389E02D20EC34E0A7
:1059D00041ED54E0C40119958091FD069091FE06B9
:1059E0000397A9F4D4011296ED91FC9113970190BD
:1059F000F081E02D60817181ED91FC910288F38945
:105A0000E02D20EC34E045ED54E0C4011995D401BB
:105A1000ED91FC9111970288F389E02D12968D91FA
:105A20009C91DC018D919C91DC016D917C91809128
:105A3000FB069091FC0629EB34E045E954E0892B04
:105A400011F042E954E0C401199520912F073091DB
:105A50003007032E000C440B550BD4011296ED9128
:105A6000FC9113970190F081E02D60817181ED919F
:105A7000FC910684F785E02D0AED14E0C401199528
:105A800020910107309102072F3F3105B9F0032E15
:105A9000000C440B550BD4011296ED91FC91139719
:105AA0000190F081E02D60817181ED91FC9106847F
:105AB000F785E02D0FED14E0C4011995198280914E
:105AC000FF069091000762E974E10097C9F065E76D
:105AD00074E181309105A1F060E774E182309105B5
:105AE00079F067E674E18330910551F063E674E183
:105AF0008430910529F08D36910531F46FE574E11C
:105B0000CE0101960E9487CB2091FF0630910007BD
:105B1000032E000C440B550BD4011296ED91FC9111
:105B200013970190F081E02D60817181ED91FC91DE
:105B30000684F785E02D05EE14E0C40119958091E7
:105B40000807F40120813181A281B3810D90BC91BD
:105B5000A02D6D917C91D9015296ED91FC912BEE87
:105B600034E0AE014F5F5F4F80FD02C045E954E075
:105B7000C4011995BDCD90E080E0BCCD8F929F927D
:105B8000AF92BF92CF92DF92EF92FF920F931F934B
:105B9000CF93DF937C014A015901C0911808D0913D
:105BA0001908062F660F110B209709F45CC0888531
:105BB0008F70863009F055C060EF74E0CE010E940E
:105BC00005996C0182E08816910449F065E474E05F
:105BD000E3E08E16910429F0D0E0C0E006C065EF46
:105BE00074E0CE010E940599EC01C114D104D9F1F1
:105BF000F60180858F708430B1F561857285A801CA
:105C0000C7010E94B8DAA8016AEF74E0C7010E94D8
:105C10009ADA209779F188858F70843059F56985F3
:105C20007A85A801C7010E949ADAA8016AEF74E098
:105C3000C7010E949ADAA114B10429F0A801B501A4
:105C4000C7010E949ADAC701DF91CF911F910F918E
:105C5000FF90EF90DF90CF90BF90AF909F908F908C
:105C60000895D0E0C0E0A8016DE777E1C7010E9488
:105C7000B5CBC9CFF2E08F16910481F083E088168E
:105C8000910429F06091870870918808CACFA80113
:105C900067E777E1C7010E9497CBC7CFA80164E708
:105CA00077E1F8CFCF92DF92EF92FF920F931F939D
:105CB000CF93DF93CDB7DEB7C154D1090FB6F894B7
:105CC000DEBF0FBECDBF6C01AB0130E020E060E471
:105CD000CE0101967C010E94BE2DF70101900020AB
:105CE000E9F731978F010E191F09A801B701C60105
:105CF0000E94AADA892B11F010E000E0C801CF5B06
:105D0000DF4F0FB6F894DEBF0FBECDBFDF91CF914E
:105D10001F910F91FF90EF90DF90CF900895CF9259
:105D2000DF92EF92FF920F931F93CF93DF93CDB744
:105D3000DEB7C054D1090FB6F894DEBF0FBECDBF99
:105D400080918E0890918F08059709F449C06115DC
:105D5000710509F445C069017A018B0140E450E006
:105D6000CE0101960E94B8DA6FE270E0CE01019692
:105D70000E947FDA892B41F4980143E050E060E40F
:105D8000CE0101960E94BE2D4FE350E0B601CE0138
:105D900001960E949ADA0E942099882309F1809145
:105DA0008E0890918F080697D9F480911A08811176
:105DB00017C0B701CE0101960E94E2A781E090E0F2
:105DC000C05CDF4F0FB6F894DEBF0FBECDBFDF91D2
:105DD000CF911F910F91FF90EF90DF90CF9008959A
:105DE00090E080E0EDCFAF92BF92CF92DF92EF9242
:105DF000FF921F93CF93DF9300D000D0CDB7DEB7D3
:105E00006C017C0110E08AE0A82EB12C133061F106
:105E1000F701828190E0B0E0A0E089839A83AB83B0
:105E2000BC83BE82AD82BE016F5F7F4F8AEE9DE074
:105E30000E94BB1A62E777E10E94C2861F5FFFEFF4
:105E4000EF1AFF0A143011F726960FB6F894DEBF4A
:105E50000FBECDBFDF91CF911F91FF90EF90DF90EC
:105E6000CF90BF90AF900895F601858190E0B0E0AB
:105E7000A0E089839A83AB83BC83BE82AD82BE01DE
:105E80006F5F7F4F8AEE9DE00E94BB1A60E777E16B
:105E9000D3CF4F925F926F927F928F929F92AF92E9
:105EA000BF92CF92DF92EF92FF920F931F93CF9307
:105EB000DF93CDB7DEB760970FB6F894DEBF0FBEA5
:105EC000CDBFFC0119861A861B861C869A859F7099
:105ED00090669A87A081B181109709F4EFC08C91E8
:105EE000882309F4EBC000811181D8019C9199238A
:105EF00009F4ADC09D3209F4E5C090539A3028F002
:105F00000F5F1F4F11830083EECFC801DC016D01CD
:105F1000C81AD90A2D91022E000C330B20533109D7
:105F20002A303105A0F37F016EE270E0C8010E94C3
:105F30007FDAFC01009709F448C0DC015D01AE1A6C
:105F4000BF0A11968C911197082E000C990BC097DF
:105F500011960A9798F32181022E000C330B2053DF
:105F600031092A30310508F075C02A30310514F0A6
:105F700029E030E037FF02C030E020E0032E000CC3
:105F8000440B550BAAE0B0E00E94DFD52B013C0189
:105F90008281082E000C990BC0978A30910588F4F5
:105FA0008A30910514F089E090E097FF02C090E0FC
:105FB00080E0092E000CAA0BBB0B480E591E6A1E6E
:105FC0007B1EA114B10409F049C0C8010E9430CB66
:105FD0002A852F70206A2A872B013C016CE270E031
:105FE000D7018D919C910E947FDA009709F061C0E2
:105FF000F701118210824D865E866F86788A88E06E
:10600000FE013996DE01119601900D928A95E1F715
:1060100029813A814B815C816D817E818F81988558
:1060200060960FB6F894DEBF0FBECDBFDF91CF9163
:106030001F910F91FF90EF90DF90CF90BF90AF90A6
:106040009F908F907F906F905F904F900895D12C8C
:10605000C12C69CF20E030E0A90194CFC801B3E0A2
:10606000AB16B104ECF4E8E0CE16D104CCF40E94F7
:1060700030CB4B015C01A4E6B0E0AC019B010E9477
:10608000DFD5B7FE08C07094609450944094411CD2
:10609000511C611C711C460E571E681E791E9ECF36
:1060A0000E940ECB2B013C018A858F7080678A8706
:1060B00095CF0196D7018D939C939DCF412C512C68
:1060C000320199CFC801019621CFEF92FF920F9331
:1060D0001F93CF93DF93EC01A881B981109761F1F1
:1060E0008C91882349F108811981F80180818823E6
:1060F00051F08D3241F080538A3028F00F5F1F4FEE
:1061000019830883F0CFC8010E9412CB7C016CE296
:1061100070E0C8010E947FDA009751F4198218825A
:10612000C701DF91CF911F910F91FF90EF900895DC
:10613000019699838883F4CFF12CE12CF1CF61E1B2
:1061400073E18AEE9DE00E94C2866EEF72E18AEEF4
:106150009DE00E94C28660EF72E18AEE9DE00E949F
:10616000C28668EE72E18AEE9DE00E94C2868AEEE7
:106170009DE00E942C8568ED72E18AEE9DE00E9410
:10618000C2866CEC72E18AEE9DE00E94C28664EAEF
:1061900072E18AEE9DE00E94C28667E972E18AEEB2
:1061A0009DE00E94C28662E872E18AEE9DE00E9454
:1061B000C28663E772E18AEE9DE00E94C2866BE6CA
:1061C00072E18AEE9DE00E94C28660E672E18AEE8C
:1061D0009DE00E94C28666E572E18AEE9DE00E9423
:1061E000C2866EE472E18AEE9DE00E94C28662E49D
:1061F00072E18AEE9DE00E94C28668E272E18AEE58
:106200009DE00E94C28669E072E18AEE9DE00E94F4
:10621000C28664EF71E18AEE9DE00E94C2866CED59
:1062200071E18AEE9DE00E94C2866EEC71E18AEE19
:106230009DE00E94C28662EC71E18AEE9DE00E94C0
:10624000C2866AEB71E18AEE9DE00E94C2866FEA27
:1062500071E18AEE9DE00E94C28662EA71E18AEEF7
:106260009DE00E94C2866AE971E18AEE9DE00E948B
:10627000C2866FE871E18AEE9DE00E94C28660E806
:1062800071E18AEE9DE00E94C28667E771E18AEEC5
:106290009DE00E94C28669E671E18AEE9DE00E945F
:1062A000C2866BE571E18AEE9DE00E94C2866EE4D3
:1062B00071E18AEE9DE00E94C2868AEE9DE00C9418
:1062C0002C850F931F93CF93DF9300D000D0CDB7D1
:1062D000DEB70E949F3069EF7BE08AEE9DE00E946E
:1062E000C286CE0101960E946529CE0101960E94C8
:1062F000F32E02E314E01A8309838091600D9091DC
:10630000610DA091620DB091630D8B839C83AD8371
:10631000BE83CE0101960E94F32E1A8309831B824D
:106320001C821D821E8280E591E00E944EA244E004
:1063300050E0BE016D5F7F4F81E090E00E94C48F0E
:10634000CE0101960E94F32E1A8309831B821C82C0
:106350001D821E8280E591E00E944EA244E050E042
:10636000BE016D5F7F4F85E090E00E94C48FCE013B
:1063700001960E94F32E6FE17CE08AEE9DE00E9480
:10638000C28688EC90E026960FB6F894DEBF0FBE6A
:10639000CDBFDF91CF911F910F910895009789F0A4
:1063A000FC0120852F70253061F40E947A990097B6
:1063B00041F0FC0120852F70243019F481859285ED
:1063C000089590E080E00895CF92DF92EF92FF92DF
:1063D0000F931F93CF93DF9300D000D0CDB7DEB7DC
:1063E0008091170881119AC080918E0890918F0832
:1063F00002970CF493C08091F2069091F3060097F7
:1064000009F48CC06EEF74E00E9405998C0100972E
:1064100009F484C00E948F99E82EF12CE114F10454
:1064200009F47CC070E060E0C8010E94CE316C01CC
:10643000EA94EF2809F481C061E0C8010E947A99CA
:10644000FC0101851285CE0101960E946529CE01CD
:1064500001960E9451A26AEE7BE08AEE9DE00E94C6
:10646000C286B6018AEE9DE00E945C8669E675E010
:106470008AEE9DE00E945C86B8018AEE9DE00E9453
:10648000879969E675E08AEE9DE00E945C8660ED82
:1064900079E08AEE9DE00E945C868AEE9DE00E9493
:1064A0002C8562E072E089E39FE00E94EC16D092B6
:1064B0002F0FC0922E0F1093310F0093300F80EDED
:1064C00099E0892BE9F58CEF94E09093330F80935A
:1064D000320F8091890890918A08009741F070E00E
:1064E00060E00E94CE319093880880938708809165
:1064F000870890918808009731F19093350F809329
:10650000340F1092370F1092360F81E080931708E6
:1065100061ED7BE08AEE9DE00E94C28626960FB672
:10652000F894DEBF0FBECDBFDF91CF911F910F91C9
:10653000FF90EF90DF90CF90089502E012E083CFBC
:1065400080ED99E0C2CF8BE393E0892B19F48CEFB7
:1065500094E0D3CF8BE393E0D0CFCF92DF92EF9252
:10656000FF921F93CF93DF9300D000D0CDB7DEB75B
:106570006CEC7BE08AEE9DE00E94C2868FECE82EF8
:106580008DE0F82E10E090E1C92ED12CF701819119
:106590007F01803130F469E874E08AEE9DE00E946A
:1065A0005C86153041F1F7013197808190E0B0E0D1
:1065B000A0E089839A83AB83BC83DE82CD82BE0157
:1065C0006F5F7F4F8AEE9DE00E94BB1A6AEC7BE012
:1065D0000E94C2861F5F1630C9F626960FB6F89441
:1065E000DEBF0FBECDBFDF91CF911F91FF90EF9027
:1065F000DF90CF9008958091D40D90E0B0E0A0E0BE
:1066000089839A83AB83BC83DE82CD82BE016F5FB8
:106610007F4F8AEE9DE00E94BB1A0E942C85DACF44
:10662000EF92FF920F931F93CF93DF9300D000D090
:106630001F92CDB7DEB77B01CE0107969F938F9354
:1066400001979F938F9301979F938F9301979F93A8
:106650008F9301979F938F9301979F938F938E01B1
:106660000F5F1F4F1F930F9385E095E09F938F93CC
:10667000DB0113968C9113978F9312968C918F93C5
:106680000E943FDB0FB6F894DEBF0FBECDBF06976A
:10669000ECF463EC7FE084EF9DE00E94C286D701BA
:1066A00012966D917C9184EF9DE00E945C8680E95A
:1066B00091E027960FB6F894DEBF0FBECDBFDF91F5
:1066C000CF911F910F91FF90EF9008958091C70D8A
:1066D0009091C80D892B09F44BC00E94C89988235A
:1066E00009F446C0A091C70DB091C80D52961C92F6
:1066F0001E92519754961C921E92539784E890E0F4
:106700001D969C938E931C971E961C921E9780E05C
:1067100090E350969C938E931F97ED91FC91119767
:106720000088F189E02D64E070E0CD011995809139
:10673000C70D9091C80DDC01ED91FC910280F381B1
:10674000E02D46E050E0B801199586E0F801AFEC85
:10675000BDE001900D928A95E1F78091C70D90916F
:10676000C80DDC01ED91FC910488F589E02D1995A7
:106770000E94AD3265ED7FE08AEE9DE00E94C28608
:1067800088EC90E096CFEF92FF920F93CF93DF9338
:10679000CDB7DEB7A0970FB6F894DEBF0FBECDBF62
:1067A0007C0100E020E033E040E250E0BE016F5F9A
:1067B0007F4F0E941320BE016F5F7F4F8BE19FE0F0
:1067C0000E945C866CEB7AE08BE19FE00E94C286BF
:1067D000F701618162956F704AE050E08BE19FE0C4
:1067E0000E94308565EB7AE08BE19FE00E94C286D3
:1067F000F70161816F704AE050E08BE19FE00E94F9
:1068000030858BE19FE00E942C85A0960FB6F8940E
:10681000DEBF0FBECDBFDF91CF910F91FF90EF9004
:106820000895AF92BF92CF92EF92FF920F931F9372
:10683000CF93DF9300D000D01F921F92CDB7DEB769
:106840005C0109831A832B833C834D835E836F83B2
:1068500078876CE477E18BE19FE00E94C286CE01ED
:1068600001960E94C33365E477E1C7010E947ECBA5
:10687000009709F45EC08981811132C00A810F70CE
:10688000013099F130F010E0023009F041C0CC2025
:10689000C9F060E0CE0101960E94E212F50102818A
:1068A0001381892B91F0C8010E94941B672B682BE0
:1068B000692B41F480E00E94FE17AB01BC01C801C6
:1068C0000E94642581E090E034C040E050E0BA01CD
:1068D000C8010E94642560E0C5010E94E01CF2CF5F
:1068E0008230F1F1B0F58130B9F168E377E18BE105
:1068F0009FE00E94C2864AE050E069818BE19FE000
:106900000E9430858BE19FE00E942C8501E010E021
:1069100068E277E18BE19FE00E94C286B8018BE1DB
:106920009FE00E9487998BE19FE00E942C8590E078
:1069300080E028960FB6F894DEBF0FBECDBFDF9182
:10694000CF911F910F91FF90EF90CF90BF90AF909C
:1069500008958A50853048F6F50102811381A3CF4E
:1069600040E050E0BA01F50182819381B2CFCF922D
:10697000DF92FF920F931F93CF93DF93F12C61155A
:10698000710509F463C06A01EB018C01CB010E941F
:106990001814F82E882309F459C0D0FE05C0D80178
:1069A0006C91CE010E94A11CD1FE47C0F801448128
:1069B000558166817781818182958F70873030F033
:1069C0008930E0F08A50823008F449C0CE010E943C
:1069D0002414EC81FD81309781F180858F709EEFCA
:1069E000980F923010F0811128C0D80111969C9117
:1069F000907F80858F70892B80871FC0EC81FD81FF
:106A00003097D9F080858F709EEF980F923010F0FC
:106A1000811113C04187528763877487EC81FD81A0
:106A20008085807F83608087EC81FD818085982FC1
:106A3000907F8F7080679036F9F26EEA7AE08BE192
:106A40009FE00E94C286C8010E94C3338F2DDF9150
:106A5000CF911F910F91FF90DF90CF900895CE01BD
:106A60000E942414EACFCF92DF92EF92FF920F930D
:106A70001F93CF93DF936115710509F460C06A011C
:106A80007B018C01CB010E941814D82F882389F137
:106A9000D70114968D919C91009709F43FC0FC0199
:106AA000C0852C2F2F703EEF320F323010F02111A5
:106AB0002AC0C595C595C595C595D0FE5EC0C701D0
:106AC0000E94D31CF8018083CC2351F1C295C07F72
:106AD00081818F70C82BC183D7011496ED91FC91F1
:106AE00081859285A385B485F80184839583A683E7
:106AF000B7838D2FDF91CF911F910F91FF90EF9072
:106B0000DF90CF900895253049F460E00E947A9993
:106B1000009721F0DC011896CC91CBCFC0E0CDCF0F
:106B2000D7011496ED91FC9180858295807F8595A3
:106B3000859585958595823021F0833081F0D0E070
:106B4000D8CF4185528563857485F80181818F7026
:106B5000806A81834483558366837783CACF418566
:106B6000528563857485F80181818F708067818388
:106B70004483558366837783BCCFCC2389F2C29547
:106B8000C07FF801A5CF0F931F93CF93DF9300D061
:106B900000D01F921F92CDB7DEB719821A821B82D6
:106BA0001C821D821E821F8218862A812F702A83D2
:106BB000FC0102811381C8010E94D31C8230D9F0EC
:106BC0008530C9F08823B9F040E052E0B801CE0129
:106BD00001960E94333560E0CE0101960E94E212D8
:106BE00028960FB6F894DEBF0FBECDBFDF91CF91D0
:106BF0001F910F91089590E080E0F2CFCF93DF9343
:106C000000D000D01F921F92CDB7DEB7FC01862FB7
:106C10008F706181607F682B618388E0DE0111964F
:106C200001900D928A95E1F729813A814B815C812F
:106C30006D817E818F81988528960FB6F894DEBF8E
:106C40000FBECDBFDF91CF910895CF93DF9300D0DA
:106C500000D01F921F92CDB7DEB7FC01608398E091
:106C6000DE01119601900D929A95E1F729813A8102
:106C70004B815C816D817E818F81988528960FB6CE
:106C8000F894DEBF0FBECDBFDF91CF910895AF92D4
:106C9000BF92CF92DF92EF92FF920F931F93CF9309
:106CA000DF93CDB7DEB7CD55D1090FB6F894DEBF6F
:106CB0000FBECDBF5C0167960FAF679768961FAF99
:106CC000689769962FAF69976A963FAF6A976B96F8
:106CD0004FAF6B976C965FAF6C976D966FAF6D977C
:106CE0006E967FAF6E971AAA19AAFE01F39682E1FB
:106CF000DF011D928A95E9F772961192119287E051
:106D0000DF011D928A95E9F7CE018A5A9F4F0E94B2
:106D1000C333F0FE2CC06796EFAD6797E83108F0FB
:106D200040C1F0E08827E856F94C8F4F0C9429D6E3
:106D3000D737B036CE37D137D137CE37B036D13757
:106D4000D137D137B036B036B036B036B036D137AD
:106D5000D137D137D137D137D137D137D137D737ED
:106D600064E17AE0CE018B5B9F4F0E9487CB0E944B
:106D70002099882309F4FAC080911A088111F6C07D
:106D8000CD2809F0F3C030E020E043E050E060E3BC
:106D9000CE0101960E94BE2DD501ED91FC9160813E
:106DA00071814FE250E0CE0101960E949ADA6701AC
:106DB000CC24B2E0DB22F1FEFDC067968FAD679771
:106DC000823009F4F7C0853009F4F4C068968FADBD
:106DD000689782958F709FE0980F9F70923018F09F
:106DE000883009F0E7C001E020E032E044E150E003
:106DF000BE016F5C7F4FCE018A5A9F4F0E941320C5
:106E0000BE016F5C7F4FCE0101960E94E2A76CEF3E
:106E100079E08BE19FE00E94C286BE016F5F7F4FE9
:106E20008BE19FE00E945C8669EF79E08BE19FE057
:106E30000E94C286BE016F5C7F4F8BE19FE00E9483
:106E40005C868BE19FE00E942C8568968FAD6897E9
:106E5000807F870100271071882311F0CD2821F44D
:106E60000115110509F4DAC030E020E043E050E0FC
:106E700060E3CE0101960E94BE2DD501ED91FC91FB
:106E8000608171814FE250E0CE0101960E949ADA52
:106E90006AEF74E0CE0101960E9474DA4FE250E08E
:106EA0006CEE79E00115110511F468EE79E0CE0180
:106EB00001960E9497CB68968FAD689782958F70E8
:106EC0008450823008F096C067E1CE018A5A9F4F05
:106ED0000E9425362F962FAF2F9760963FAF609771
:106EE00061964FAF619762965FAF629763966FAF9F
:106EF000639764967FAF649765968FAF6597669644
:106F00009FAF669700E020E033E044E150E0BE012F
:106F10006F5C7F4FCE018A5A9F4F0E94132062EE12
:106F200079E08BE19FE00E94C286BE016F5F7F4FD8
:106F30008BE19FE00E945C866FED79E08BE19FE042
:106F40000E94C286BE016F5C7F4F8BE19FE00E9472
:106F50005C868BE19FE00E942C850E94209988230B
:106F600029F080911A08882309F44CC0B701C501A3
:106F70000E94611C90E080E0C35ADF4F0FB6F89486
:106F8000DEBF0FBECDBFDF91CF911F910F91FF905C
:106F9000EF90DF90CF90BF90AF90089560E17AE0DE
:106FA000E1CE62E07AE08BE19FE00E94C286E89445
:106FB000F0F8DDCEF0FE49CFBE016B5B7F4FCE0116
:106FC00001960E94E2A763EF79E08BE19FE00E94C7
:106FD000C286BE016F5F7F4F8BE19FE00E945C869F
:106FE00060EF79E08BE19FE00E94C286BE016B5B9F
:106FF0007F4F23CF20E032E0012B11F020E033E07F
:1070000000E083CFBE016F5C7F4FCE0101960E94EE
:10701000E2A760E072E0C5010E943D1CF0FE77C06F
:107020006796EFAD6797E150EE30E0F4F0E0882727
:10703000E35EF74C8F4F0C9429D6933832383238B0
:107040003238323893383238323832382B388A383E
:10705000983890388D3865ED79E0CE018B5B9F4F85
:107060000E9487CB30E020E043E050E060E3CE01B7
:1070700001960E94BE2DD501ED91FC916081718138
:107080004FE250E0CE0101960E949ADA6AEF74E076
:10709000CE0101960E9474DA4FE250E06FEB79E086
:1070A000CE0101960E9497CB69EB79E08BE19FE0DE
:1070B0000E94C286BE016F5F7F4F8BE19FE00E94FE
:1070C0005C8666EB79E08BE19FE00E94C286BE01A0
:1070D0006B5B7F4F8BE19FE00E945C868BE19FE0C2
:1070E0000E942C850E942099882309F43FCF80912B
:1070F0001A0881113BCFBE016B5B7F4FCE01019619
:107100000E94E2A760E071E0C5010E943D1C81E0A1
:1071100090E032CF60ED79E0A0CF6CEC79E09DCFCC
:1071200063EC79E09ACFF5018085853009F09ACF3C
:107130006AED79E092CFDC011196EC911197E2951E
:10714000EF70E150EB3008F037C0F0E08827E455ED
:10715000F74C8F4F0C9429D6BE38BE38DC38B73880
:10716000B738CD38C438C438C438B738B7381496AF
:107170006D917D918D919C911797089514966C91C6
:1071800070E090E080E0089514966D917D918D916E
:107190009C9117970E9426D7089514966D917D9122
:1071A0008D919C91179724E630E040E050E00E94DA
:1071B000C0D5CA01B901089560E070E0CB0108951F
:1071C0004F925F926F927F928F929F92AF92BF92F7
:1071D000CF92DF92EF92FF920F931F93CF93DF93A3
:1071E000CDB7DEB762970FB6F894DEBF0FBECDBF46
:1071F0004C010B871C872D873E874F87588B698BE7
:107200007A8B67EA74E1C7010E947ECBEFE0F0E081
:10721000892BF1F061EA74E1C7010E947ECBE1E1C4
:10722000F0E0892BA9F06BE974E1C7010E947ECBE5
:10723000E0E1F0E0892B61F01F7067E974E1C701BC
:107240000E947ECBE12FF0E0892B11F4EEE0F0E01C
:107250009B85992309F482C1309731F4EF2809F412
:107260007AC08FEF9FEF9EC03197E131F10508F0B2
:1072700040C08827E15CF64C8F4F0C9429D6AB397F
:1072800050397939793979397939143A563A79391D
:10729000793979397939793979395D3AA13A693A5F
:1072A000CE010B960E949B387093300760932F0796
:1072B0009B01205131092931310598F620EF260F25
:1072C00020932D079B01770F440B550BD401129689
:1072D000ED91FC9113970190F081E02D6081718117
:1072E000ED91FC910684F785E02D0AED14E0C401D0
:1072F000199510921B0781E0809313078DE480930A
:1073000014078FE58093150782EE99E00E94157DA2
:10731000F401828193810E94941B2B013C01411452
:1073200051046104710491F00E9414A79B01AC0107
:10733000A12CB12C650114E6E12EF12C00E010E047
:10734000C301B2010E94C82A882349F345E250E0F4
:107350006AE077E022C091509E3058F6E92FF0E0C5
:107360008827EA54F64C8F4F0C9429D6C439E93952
:1073700079397939E939C439793979397939FF393C
:10738000FB39F339033A013A809108078160809311
:1073900027074DE050E06CE172E0C4010E94C42573
:1073A00081E090E062960FB6F894DEBF0FBECDBFCD
:1073B000DF91CF911F910F91FF90EF90DF90CF90D1
:1073C000BF90AF909F908F907F906F905F904F9005
:1073D0000895809108078E7F809327074DE050E045
:1073E0006FE072E0DACF1092210780910807816088
:1073F000809327077ECF81E080932107F6CF82E03C
:10740000FBCF84E0F9CF83E08093210780910807C8
:1074100081608093270780912307833009F069CF2B
:1074200082E08093230765CF19829031A1F148F45F
:107430009C3089F0CE010B960E949B386093230705
:1074400013C0913169F19231A9F782E0809323074B
:1074500062E874E105C083E08093230762E974E188
:10746000CE0101960E9487CBD4011296ED91FC913A
:1074700013970190F081E02D60817181ED91FC9175
:107480000288F389E02D20EC34E0AE014F5F5F4FBE
:10749000C40119952ECF109223076DE874E1E0CF57
:1074A00081E08093230766E874E1DACFCE010B9682
:1074B0000E949B38609321071CCF913031F09230AD
:1074C00009F017CF1092260714CF80E58093260786
:1074D00010CF913049F09230F1F0CE010B960E941E
:1074E0009B386093250705CF83E080932607D4015E
:1074F0001296ED91FC9113970190F081E02D60813F
:107500007181ED91FC910288F389E02D29EB34E043
:1075100042E954E0BDCF10922607D4011296ED91B6
:10752000FC9113970190F081E02D60817181ED91C4
:10753000FC910288F389E02D29EB34E045E954E021
:10754000A7CF913039F0923009F0D3CE8091270740
:10755000877F4ECF8091270788604ACFE231F105BF
:1075600008F0C7CE8827E854F54C8F4F0C9429D6E5
:107570003139793950397939793979397939143A50
:10758000563A79397939793979397939793979398D
:1075900079396D3ACF93DF93EC016115710539F4B8
:1075A0008F8181708F8381E0DF91CF9108958981F0
:1075B000982F92959F7029F180E09430A8F79B0155
:1075C000770F440B550B2959310941095109A4E69C
:1075D000B0E00E94DFD52BE531E040E050E00E94B2
:1075E000C0D537FF02C030E020E02536310514F069
:1075F00024E630E02F5F220F8F818170282B2F83AC
:10760000D2CF8F7080628983DACF2F923F924F92D0
:107610005F926F927F928F929F92AF92BF92CF9222
:10762000DF92EF92FF920F931F93CF93DF93CDB72B
:10763000DEB768970FB6F894DEBF0FBECDBF1C0152
:1076400009871A872B873C874D875E876F87788BE2
:1076500022E1E216F10408F035C0F701E55BFC4FCA
:107660003081398BCE0109960E94F61397FD04C034
:10767000BC01C1010E94CA3A9A85892F8F70D1013D
:107680001196EC911197E07FE82B1196EC931197EE
:1076900089858C93E295EF70EC3008F063C0F0E0E0
:1076A0008827EA5AF44C8F4F0C9429D6633D7F3BD0
:1076B0007F3B013D643B8F3DCA3C0B3D0B3D0B3D89
:1076C000CA3CCA3C198ACECFB12C92959F709D308E
:1076D00008F0C9C4E92FF0E08827EE58F44C8F4F2A
:1076E0000C9429D6B23BC93DE93DC93D923D923D3E
:1076F000C93DC93D33403340C93DC93D963C929593
:107700009F709D3008F022C1E92FF0E08827E457F0
:10771000F44C8F4F0C9429D6B23B6A3C5E3C203C23
:107720009C3B993B413C6E3CA63CA63C2B3C2B3CF5
:10773000963C8889F10187838F85D10116968C93B9
:1077400016978E8515968C9315978D8514968C9328
:1077500014979295907F11968C9111978F70982B1A
:1077600011969C93B989BB2309F467C0F10181810B
:1077700082958F702B2F30E08217130609F45DC0BD
:107780006CE17AE08BE19FE00E94C286D101119604
:107790006C9162956F704AE050E08BE19FE00E942F
:1077A000308569E17AE08BE19FE00E94C2864AE081
:1077B00050E069898BE19FE00E94308567E17AE0C3
:1077C0008BE19FE00E94C286F101008119821A823A
:1077D0001B821C821D821E821F82188689898295C7
:1077E000807F9A819F70892B8A830983EE24EA9493
:1077F000FE2C1181228133814481558166817781FC
:10780000CE0101960E94053BD1012C9311963C9329
:10781000119712964C93129713965C9313971496A4
:107820006C93149715967C93159716968C931697D0
:1078300017969C93C1010E94C33388E0F10182C175
:107840008F859889F1018683878190FB80F98783F2
:107850008E85858387CF8D859E85AF85B8898F3F3F
:107860009105A105B10529F024F08FEF90E0A0E08B
:10787000B0E0B7FF03C080E090E0DC01F101848359
:1078800071CF6D857E858F85988924E630E040E054
:1078900050E00E94C0D52F3F31054105510529F028
:1078A00024F02FEF30E040E050E057FF03C020E02D
:1078B00030E0A901D10114962C9354CF8F8598897B
:1078C000F1018683878190FB80F987838E8585838C
:1078D0008D85D5CF8D8514968C9344CFCD84DE8451
:1078E000EF84F88820E030E0A901C701B6010E94CA
:1078F00054D487FD17C020E030E04FE753E4C701C0
:10790000B6010E945CD7181634F4C12CD12CAFE715
:10791000EA2EA3E4FA2EC701B6010E942DD7F10189
:10792000648320CFC12CD12C7601F5CFD1011196E3
:107930008C9111978F70806C11968C9311978D8517
:107940009E8515969C938E9314970CCF6CE97AE0E4
:107950008BE19FE00E94C2866A8562956F704AE063
:1079600050E08BE19FE00E94308569E97AE08BE18D
:107970009FE00E94C286F101618162956F704AE0CA
:1079800050E08BE19FE00E9430858BE19FE00E94F8
:107990002C85E8CE92959F70933091F09C3031F217
:1079A0004D855E856F857889F101448355836683B3
:1079B00077839295907F81818F70982B9183D2CE1F
:1079C00060E0C1010E94E212D10114968C931497D9
:1079D0008F85988916968C93169717968C91179782
:1079E00090FB80F917968C9317978E8515968C933C
:1079F000159711968C9111978F70806211968C93C8
:107A0000B1CE60E0CE0109960E94E212D101149637
:107A10008C931497EECF92959F709D3008F066C0BE
:107A2000E92FF0E08827E85EF24C8F4F0C9429D6BE
:107A3000B23B333D623DE03C623D623D253D523DFF
:107A4000523D523D413D4D3D963C8D859E85AF85D5
:107A5000B889F10184839583A683B78381818F7070
:107A6000806681837FCE6D8570E090E080E00E942B
:107A700059D4D10114966D937D938D939C93179750
:107A800071CE6D857E858F8598890E945BD4F101CA
:107A9000648375838683978365CE6D857E858F85A8
:107AA0009889E5CF9295907FF10181818F70982B15
:107AB00091838D859E85AF85B88984839583A683C0
:107AC000B78350CE9295907FD10111968C911197EA
:107AD0008F70982B11969C938D859E85AF85B88964
:107AE000F10184839583A683B7833CCE67E87AE06F
:107AF0008BE19FE00E94C2866A8562956F704AE0C2
:107B000050E08BE19FE00E94308564E87AE08BE1F1
:107B10009FE00E94C286D10111966C912ECFBB24AA
:107B2000B394D3CD4D855E856F857889F10144830B
:107B30005583668377839295907F81818F70982B90
:107B4000918388E0DE01119601900D928A95E1F70C
:107B500029813A814B815C816D817E818F819885FD
:107B600068960FB6F894DEBF0FBECDBFDF91CF9100
:107B70001F910F91FF90EF90DF90CF90BF90AF904B
:107B80009F908F907F906F905F904F903F902F903D
:107B90000895963009F43AC148F46D85913071F03A
:107BA0006FEF70E0933051F060E008C0973009F457
:107BB00039C19A506D857E859230B0F784E68F8703
:107BC00088898E7F888B1E868A858F7080628A87DF
:107BD0006D872E8530E0AFEFB0E00E94F2D524E64D
:107BE00030E040E050E00E94C0D569017A01FFEF2B
:107BF000CF16D104E104F10429F024F0C12CD12CDA
:107C00007601CA9486012D852A8B622E712CBB20A9
:107C100009F471C088898695A82FA150BB0B2D014E
:107C2000BFEF4B165B0609F01EC1003811050CF0C2
:107C300000C18FE790E08C199D09869DD001879D3A
:107C4000B00D969DB00D11242FEF30E00E9440D66C
:107C500021E83EE740E050E00E94C0D5F1012783D3
:107C6000ABE9B0E0A70196010E94DFD5EFE78E2EC9
:107C7000912CA12CB12CA50194010E94C0D58901A1
:107C80009A010C591F4F2F4F3F4FAEEFB1E0A701A4
:107C900096010E94DFD5A50194010E94C0D5D301B1
:107CA0000E94DFD52FEF30E040E050E00E94C0D5C9
:107CB00039012FEF6216710421F01CF066246A94DA
:107CC000712C67E77AE08BE19FE00E94C286B801E1
:107CD0008BE19FE00E94879969E67AE08BE19FE063
:107CE0000E94C286B3018BE19FE00E9487998BE1DD
:107CF0009FE00E942C85EAE2FCE1E491F0E0EE0FC7
:107D0000FF1FE05FF34E85919491E0E8FCE1E49180
:107D10002F8538893170AFEFBFEF0E94F2D52DE685
:107D200031E040E050E00E94C0D544275527AAEF3B
:107D3000B5E00E94DFD5DC01CB019058AF4FBF4FBB
:107D4000CD01BB2797FDB095AB2F8E3FE1E09E079D
:107D500008F062C1382F8F3F910508F47FC14EEFC4
:107D6000481B50E03FEFF301319678012FEFE21A04
:107D7000F20A009510E03E9DC0013F9D900D112438
:107D8000292F3327200F311FDF010E9440D64B01DE
:107D90005C018824AA24BB245E9D90015F9D300D68
:107DA0001124232F3327200F311F0E9440D6BB27D9
:107DB000A92F982F872F882A992AAA2A4E9D9001A9
:107DC0004F9D300D1124232F3327200F311FDF014A
:107DD0000E9440D6B82FA72F962F8827882799274B
:107DE000BB2788299929AA29F101A6839583848331
:107DF0006DE37AE08BE19FE00E94C286C1010E94A0
:107E0000C33360E080E00E948AA5ACCC6D857E859E
:107E10008F85988924E630E040E050E00E94C0D58C
:107E2000B901CCCE6D857E858F8598890E9426D735
:107E3000C5CEA70196012058310941095109ABE986
:107E4000B0E00E94DFD52FE730E040E050E00E9434
:107E5000C0D589019A010C591F4F2F4F3F4FD101B7
:107E600017961C922ECF9201AAEBBFEF0E9438D634
:107E700044E6842E912CA12CB12CA50194010E94E2
:107E8000C0D5DA01C9018C599F4FAF4FBF4F8B8BC3
:107E90009C8BAD8BBE8B26E430E0D2010E9440D695
:107EA000A50194010E94C0D549015A019EE1890EA5
:107EB000911CA11CB11C003811050CF093C08FE778
:107EC00090E08C199D09869DD001879DB00D969DEF
:107ED000B00D1124A50194010E94EAD59B01AC01CB
:107EE000AFEFB0E00E94DFD524E63AE640E050E094
:107EF0000E94C0D5D10117962C932B893C894D89BE
:107F00005E892C0D3D1D4E1D5F1DAEEFB1E00E9440
:107F1000DFD523EE30E040E050E00E94C0D52901DB
:107F20003A01388F2F8BAFEFB0E0A70196010E9486
:107F3000DFD52FE730E040E050E00E94C0D5890156
:107F4000EA89AE2FB0E0A30192010E94DFD52FEFA6
:107F500030E040E050E00E94C0D539012F3F3105AC
:107F600021F01CF066246A94712C63E67AE08BE1C0
:107F70009FE00E94C2862AE030E04B895C896D89CF
:107F80007E898BE19FE00E94D2856DE57AE08BE1EE
:107F90009FE00E94C2862AE030E0B501A4018BE197
:107FA0009FE00E94D28565E57AE08BE19FE00E9428
:107FB000C286B8018BE19FE00E9487996DE47AE068
:107FC0008BE19FE00E94C286B3018BE19FE00E949B
:107FD000879964E47AE08BE19FE00E94C2866F8912
:107FE000788D81CEA70196012058310941095109A8
:107FF000ABE9B0E00E94DFD52FE730E040E050E091
:108000000E94C0D589019A010C591F4F2F4F3F4F35
:10801000D10117961C92A9CF8C3FF3E09F0768F41B
:108020008D3F22E0920728F452E0580F3FEF40E0E6
:108030009ACE3CEF381B5FEFFACF8A3F35E09307CB
:1080400081F08B3FE4E09E0728F444E0480F5FEFA7
:1080500030E089CE5AEF581B30E001C050E04FEFBE
:1080600082CE50E0F9CF6BE27AE08BE19FE00E9494
:10807000C2866A8562956F704AE050E08BE19FE0AE
:108080000E94308568E27AE042CDAF92BF92CF92F3
:10809000DF92EF92FF920F931F93CF93DF93CDB7B1
:1080A000DEB768970FB6F894DEBF0FBECDBFFC01F8
:1080B000098B1A8B2B8B3C8B4D8B5E8B6F8B788F48
:1080C00082819381009709F49FC024813581232BFD
:1080D00009F49AC0CC2009F497C06F0170E060E009
:1080E0000E94B01B192FD601ED91FC91028CF38DEB
:1080F000E02DC60119955C018230910509F478C024
:10810000039709F447C095E0F1E0AF16B10409F018
:1081100091E019861A861B861C861D861E861F8680
:10812000188A9295907F8A858F70892B8A87EE2492
:10813000EA94FE2C09891A892B893C894D895E892C
:108140006F89788DCE0109960E94053BF1E0AF164C
:10815000B10409F44FC082E0A816B10409F045C08B
:108160006F8570E0D60114968C910E94C6A561E0DF
:1081700070E0C6010E94DB1B6E8570E00E94C6A500
:1081800062E070E0C6010E94DB1B6D8570E00E941A
:10819000C6A52BC0612F661F6627661FCE014196BC
:1081A0000E94E2125C01BC01D60114968C910E94DF
:1081B000C6A560EC76E18BE19FE00E94C286F601E5
:1081C000648175818BE19FE00E9487996EEB76E177
:1081D0008BE19FE00E94C286B5018BE19FE00E9487
:1081E00087998BE19FE00E942C8581E090E00EC092
:1081F00094E08FCF63E070E0C6010E94DB1B6889CA
:1082000070E00E94C6A5ACCF90E080E068960FB603
:10821000F894DEBF0FBECDBFDF91CF911F910F91BC
:10822000FF90EF90DF90CF90BF90AF900895FC014A
:108230009181892F82958F7021F0823029F080E022
:1082400008959F70906291839B0177FF02C030E098
:1082500020E02E3681E0380714F02DE631E0268349
:10826000878130FB80F9878381E00895AF92BF92C8
:10827000CF92DF92EF92FF920F931F93CF93DF93F2
:1082800000D000D01F921F92CDB7DEB75C017B01FA
:1082900060FF03C0E894E0F8F3F8F3FC0DC00E941F
:1082A000EB11663971058105910530F080918E08DA
:1082B00090918F080597F9F4B70166277370C5018F
:1082C0000E94611C65EA79E08BE19FE00E94C28612
:1082D0008FEF9FEF28960FB6F894DEBF0FBECDBF8D
:1082E000DF91CF911F910F91FF90EF90DF90CF9092
:1082F000BF90AF90089519821A821B821C821D8242
:108300001E821F8218868A818F708A8340E053E024
:10831000B501CE0101960E94333560E073E0C501DE
:108320000E94871CE82AF92AD12CC12C09811A81C4
:108330002B813C814D815E816F817885C5010E94D2
:108340004736C8CF4F925F926F927F92AF92BF92A3
:10835000CF92EF92FF920F931F93CF93DF9300D0B2
:1083600000D01F921F92CDB7DEB75C0109831A833C
:108370002B833C834D835E836F8378876AE077E04D
:108380008BE19FE00E94C286CE0101960E94C3331A
:108390008981811134C00A810F700130A9F160F127
:1083A000023021F010E0053009F041C0D501ED9117
:1083B000FC91068CF78DE02D09811A812B813C817F
:1083C0004D815E816F817885C501199581E090E0CE
:1083D00028960FB6F894DEBF0FBECDBFDF91CF91C8
:1083E0001F910F91FF90EF90CF90BF90AF907F9033
:1083F0006F905F904F900895CC24C394D7CF813075
:1084000061F1823009F4E0C06DEF76E08BE19FE02E
:108410000E94C2864AE050E069818BE19FE00E94A1
:1084200030858BE19FE00E942C8501E010E06DEE2D
:1084300076E08BE19FE00E94C286B8018BE19FE06D
:108440000E9487998BE19FE00E942C85CE010196C6
:108450000E94C33390E080E0BBCF1A8112951F7059
:10846000163009F478C088F48FEF810F823048F518
:108470002D8130E0A4E6B0E00E94F2D52FEF30E08D
:1084800040E050E00E94C0D519C01730E9F186EFF6
:10849000810F8230B0F48D819E81AF81B8858536A1
:1084A0009105A105B10524F084E690E0A0E0B0E0DC
:1084B000B7FF03C080E090E0DC019C01243131056E
:1084C000D4F4163009F47BC008F05EC011501230AD
:1084D00008F469C0F5016281738140E052E0CE0189
:1084E00001960E94B73460E07AE0D50112968D9132
:1084F0009C910E943641D501ED91FC91068CF78D3F
:10850000E02DCC24C39458CF4D805E806F8078845A
:1085100020E030E0A901C301B2010E9454D487FDDC
:1085200011C020E030E048EC52E4C301B2010E94E7
:108530005CD7181654F4412C512C88EC682E82E438
:10854000782E03C0412C512C3201C301B2010E948C
:1085500026D79B01B3CF6D817E818F81988524E6DC
:1085600030E040E050E00E94C0D52536310541059D
:10857000510524F024E630E040E050E057FF9ECF64
:1085800020E030E0A9019ACF173081F01A508CE436
:1085900090E0A0E0B0E0123008F09CCF8D839E8385
:1085A000AF83B88797CF8CE48D8394CF80E090E041
:1085B000A8E9B2E48D839E83AF83B8878BCF82EE28
:1085C0009DE1A0E0B0E0EACF1D821E821F821886E6
:1085D000D501ED91FC91068CF78DE02DCC24C39450
:1085E00002E01A812B813C8140E0EBCE0F931F9378
:1085F000CF93DF938C01FC01C081D1816FE270E0E9
:10860000CE010E94C7DA0097D9F0FC011192CF0188
:108610000E94CA19EC0167E977E08BE19FE00E94B4
:10862000C286BE018BE19FE00E9487998BE19FE0AB
:108630000E942C85CE01DF91CF911F910F9108955B
:10864000CE010E94CA19EC01892BA1F3F801118215
:108650001082F0CF2F923F924F925F926F927F9253
:108660008F929F92AF92BF92CF92DF92EF92FF9242
:108670000F931F93CF93DF93CDB7DEB7C15CD109C2
:108680000FB6F894DEBF0FBECDBF1C01C755DF4F3C
:108690000883C95AD040C655DF4F1883CA5AD04004
:1086A000C555DF4F2883CB5AD040C455DF4F3883A0
:1086B000CC5AD040C355DF4F4883CD5AD040C25525
:1086C000DF4F5883CE5AD040C155DF4F6883CF5A11
:1086D000D040C055DF4F7883C05BD040CF54DF4FD0
:1086E000F982E882C15BD040CF53DF4FC882C15CC2
:1086F000D0400E9414A7C354DF4F688379838A83D4
:108700009B83CD5BD040C655DF4F8881CA5AD0408D
:108710008F70C82ED12CCD54DF4FD982C882C35B55
:10872000D040E0908E08F0908F08C554DF4FF9825A
:10873000E882CB5BD040CF54DF4FE881F981C15B49
:10874000D040309721F0808181110C94074FD101E6
:108750001B968C91882341F0C1010B96CF54DF4FBB
:1087600099838883C15BD040CD54DF4FC880D980C6
:10877000C35BD040CD2811F00C94634FCF54DF4F32
:10878000E881F981C15BD040309711F00C94104F13
:10879000D1015B960D90BC91A02DCD54DF4FB983D4
:1087A000A883C35BD040AB2B11F40C94634FC65528
:1087B000DF4F8881CA5AD0408F7011F00C94634FFC
:1087C000CD54DF4F6881C35BD040CE0187559F4FAA
:1087D0000E94FE35C756DF4F2883C959D040C65680
:1087E000DF4F3883CA59D040C556DF4F4883CB5935
:1087F000D040C456DF4F5883CC59D040C356DF4FCA
:108800006883CD59D040C256DF4F7883CE59D040CF
:10881000C156DF4F8883CF59D040C056DF4F988371
:10882000C05AD0400C94634FD1018D919C91009718
:1088300009F407C2CD54DF4FE881F981C35BD04012
:108840003D9709F0ACC00E948F99082F10E00630C8
:108850001105A4F40E94CB8E009739F0DC01189624
:108860002C911897207F18962C93BC01F1018081E0
:1088700091810E949E9D0F5F1F4FE9CF65E0D1015E
:108880008D919C910E947A998C01892BE9F410E0DA
:1088900000E0C801CF53DF4F0FB6F894DEBF0FBE24
:1088A000CDBFDF91CF911F910F91FF90EF90DF909F
:1088B000CF90BF90AF909F908F907F906F905F9080
:1088C0004F903F902F900895C755DF4F8881C95A28
:1088D000D0408031E0F6CE0187559F4F0E949B38F3
:1088E000161617061806190624F4F80180858D70EF
:1088F000A1F0D80118968C9118978F7018968C93C8
:1089000062E079E08BE19FE00E94C2868BE19FE00C
:108910000E942C8501E010E0BCCF0E9414A76B01DF
:108920007C01CE0187559F4F0E949B38C60ED71EF3
:10893000E81EF91EF801C186D286E386F486C75583
:10894000DF4F8881C95AD0408295807F82608087BE
:1089500067EF78E08BE19FE00E94C286CE018755E9
:108960009F4F0E949B38AB01BC012AE030E08BE1B5
:108970009FE00E94D28561EF78E08BE19FE00E944A
:10898000C286D80119964D915D916D917C911C978D
:108990002AE030E08BE19FE00E94D285B7CFC75537
:1089A000DF4F1881C95AD040143009F4A9C228F405
:1089B000112391F1B12CA12C60C288EF810F82307C
:1089C000C8F788E0FE01E755FF4FDE0111960190E0
:1089D0000D928A95E1F7C655DF4FE881CA5AD0401B
:1089E0008E2F807F09F400C3E295EF70E150EB30E9
:1089F00008F0FAC2F0E08827EF5FFA4B8F4F0C9433
:108A000029D6E247E247F447D347D3477F486E4829
:108A10006E486E48D347D34719821A821B821C8244
:108A20001D821E821F8218868A818F708A83C65596
:108A3000DF4F8881CA5AD040807F09F4BBCFCD5424
:108A4000DF4FE881F981C35BD040E930F10509F4DB
:108A500016C20CF0F9C0309709F41EC1329709F024
:108A6000A9CFB12CA12CC12CDD24DA94B101CE0107
:108A700001960E94F99D8A81982F92959F70945F2C
:108A80009F70923060F4C655DF4F9881CA5AD0402B
:108A900092959F70923019F48F7080628A83D10111
:108AA00018969C91973071F4C655DF4F8881CA5A49
:108AB000D040807E803211F0803421F48A818F7022
:108AC00080628A83F101A185B285892F90E0109799
:108AD00041F0ED91FC911197028CF38DE02DCD01C9
:108AE00019957C01C755DF4F0881C95AD040C6553A
:108AF000DF4F1881CA5AD040C555DF4F2881CB5A65
:108B0000D040C455DF4F3881CC5AD040C355DF4FD9
:108B10004881CD5AD040C255DF4F5881CE5AD040FF
:108B2000C155DF4F6881CF5AD040C055DF4F7881A3
:108B3000C05BD040CE0101960E94053BCF57DF4F6E
:108B40002883C158D040CE57DF4F3883C258D04019
:108B5000CD57DF4F4883C358D040CC57DF4F5883A1
:108B6000C458D040CB57DF4F6883C558D040CA5750
:108B7000DF4F7883C658D040C957DF4F8883C75826
:108B8000D040C857DF4F9883C858D040CE010196D7
:108B90000E94C333CC2069F1C655DF4F8881CA5A81
:108BA000D04082958F709FE0980F9F70923020F098
:108BB0008A5F8F708230E8F48A8182958F7081504D
:108BC0008230B8F42D8130E0AFEFB0E00E94F2D5F2
:108BD00024E630E040E050E00E94C0D52F3F310550
:108BE0004105510529F024F02FEF30E040E050E03E
:108BF0002D8388E0FE013196DE01A755BF4F01901D
:108C00000D928A95E1F7FAE0BF2A512CD10118960E
:108C10008C911897873009F071C5C954DF4FE881EE
:108C2000F981C75BD040EE35F1400CF04AC46BECE3
:108C300078E084EF9DE00E94C28684EF9DE00E9470
:108C40002C850FEF1FEF25CECD54DF4F28813981C2
:108C5000C35BD0402A30310509F4BFC02B30310549
:108C600009F0A8CEB101CE0101960E94F99DCE0176
:108C700087559F4F0E94F613BC01CE0101960E94BA
:108C8000CA3A88E0FE013196DE01A755BF4F019038
:108C90000D928A95E1F7EEC0C1010E9412538C013A
:108CA00061E070E01816190614F070E060E08BE1E6
:108CB0009FE00E94879969E474E08BE19FE00E9445
:108CC0005C86CE0187559F4F0E949B38AB01BC014B
:108CD0002AE030E08BE19FE00E94D2858BE19FE0AB
:108CE0000E942C85CE0187559F4F1016110614F057
:108CF0000C94FB4E0E949B38B12CA12C672B682B47
:108D0000692B89F562E0CE0187559F4F0E94253679
:108D1000CF56DF4F2883C159D040CE56DF4F38831E
:108D2000C259D040CD56DF4F4883C359D040CC56AE
:108D3000DF4F5883C459D040CB56DF4F6883C559A5
:108D4000D040CA56DF4F7883C659D040C956DF4F4E
:108D50008883C759D040C856DF4F9883C859D04040
:108D6000AA24A394BA2CCC24C394DD24D3947ECE1D
:108D700061E0CE0187559F4F0E942536C757DF4FD0
:108D80002883C958D040C657DF4F3883CA58D040CF
:108D9000C557DF4F4883CB58D040C457DF4F588367
:108DA000CC58D040C357DF4F6883CD58D040C2570E
:108DB000DF4F7883CE58D040C157DF4F8883CF58DC
:108DC000D040C057DF4F9883C059D040AA24A39405
:108DD000BA2CCC24C394D12C49CEB101CE0101963A
:108DE0000E94F99DC255DF4F8881CE5AD0409A81AA
:108DF00092959F7041F0923051F0B12CA12C5524E6
:108E00005394C12C0EC29A819F7090629A8390E015
:108E10008536910514F084E690E08E8388E0FE01AB
:108E20003196DE01A755BF4F01900D928A95E1F76B
:108E300062E0CE0187559F4F0E94FE35EA962FAF24
:108E4000EA97EB963FAFEB97EC964FAFEC97ED962A
:108E50005FAFED97EE966FAFEE97EF967FAFEF9720
:108E6000C158DF4F8883CF57D040C058DF4F988319
:108E7000C058D040A12CBAE0BB2E512CC2CFB101BA
:108E8000CE0101960E94F99DC155DF4F6881CF5AEE
:108E9000D040C055DF4F7881C05BD0407170CE01AB
:108EA00001960E941741C82E882309F49FC288E0CA
:108EB000FE013196DE01A755BF4F01900D928A95B4
:108EC000E1F762E0CE0187559F4F0E94FE35E296A2
:108ED0002FAFE297E3963FAFE397E4964FAFE49767
:108EE000E5965FAFE597E6966FAFE697E7967FAFBB
:108EF000E797E8968FAFE897E9969FAFE997BACFE3
:108F0000C1010E941253181619063CF562E0CE0109
:108F100087559F4F0E942536AA962FAFAA97AB96EA
:108F20003FAFAB97AC964FAFAC97AD965FAFAD97F9
:108F3000AE966FAFAE97AF967FAFAF97E0968FAF1D
:108F4000E097E1969FAFE197AA24A394BA2C512C05
:108F5000CC24C394DD24D39459CE61E0CE0187554F
:108F60009F4F0E942536A2962FAFA297A3963FAFA0
:108F7000A397A4964FAFA497A5965FAFA597A69683
:108F80006FAFA697A7967FAFA797A8968FAFA89722
:108F9000A9969FAFA997AA24A394BA2C512CCC24AC
:108FA000C394D12C33CEC355DF4F288139814A81F8
:108FB0005B81CD5AD040A4E6B0E00E94DFD54B01E2
:108FC0005C010DC0C355DF4F8880CD5AD04024E6E8
:108FD000829E40011124092C000CAA08BB088114B0
:108FE0009104A104B10429F4E5E08E2E912CA12C6A
:108FF000B12C193041F4B094A09490948094811CC9
:10900000911CA11CB11CB101CE0187559F4F0E943C
:10901000F99D60E0CE0187559F4F0E9425366A96E4
:109020002FAF6A976B963FAF6B976C964FAF6C976D
:109030006D965FAF6D976E966FAF6E976F967FAFC1
:109040006F97A0968FAFA097A1969FAFA197CD5491
:10905000DF4F88819981C35BD0408230910509F44C
:10906000ABC00CF055C0CC24C394892B09F0A2CC22
:10907000F10181859285009709F0A0C0808590E07C
:1090800060E5462E512C612C712C8530910549F0FC
:10909000412C512C3201449721F0412C512C3201AA
:1090A0004A94C655DF4FE881CA5AD040E295EF7026
:1090B000E150EB3008F090C1F0E08827ED59F74B14
:1090C0008F4F0C9429D6E648E648EC49EC49EC4928
:1090D000B9498349834983491449144920E030E060
:1090E00048EC52E4C355DF4F688179818A819B81C6
:1090F000CD5AD0400E94BAD40E9426D760CFC35523
:10910000DF4F88809980AA80BB80CD5AD04067CF3E
:10911000CD54DF4FA881B981C35BD040A930B105E0
:1091200009F469C11A9709F045CCC655DF4F88810B
:10913000CA5AD04082958F70823009F0B7C1C501FC
:10914000B40124E630E040E050E00E94C0D5C255B2
:10915000DF4F8881CE5AD04090E0280F391F37FF6B
:1091600002C030E020E02536310514F024E630E07E
:10917000C255DF4F2883CE5AD04062E0CE018755DA
:109180009F4F0E94FE352A962FAF2A972B963FAF0E
:109190002B972C964FAF2C972D965FAF2D972E9631
:1091A0006FAF2E972F967FAF2F9760968FAF6097F8
:1091B00061969FAF61975ECEC12C5ACFDC01ED91D5
:1091C000FC91028CF38DE02D19955ACFC355DF4FDA
:1091D0001881CD5AD040C501B40124E630E040E00A
:1091E00050E00E94C0D5DA01C901810F911DA11D77
:1091F000B11DB7FF03C080E090E0DC018F3F910517
:10920000A105B10529F024F08FEF90E0A0E0B0E0D7
:10921000C355DF4F8883CD5AD040A12C5AE0B52EDC
:10922000512CDD24DA94F2CCC355DF4FE880F9806D
:109230000A811B81CD5AD040B4E68B169104A1045B
:10924000B104DCF5A4E6B0E0A80197010E94DFD5E7
:10925000860E971EA81EB91E4114510461047104A4
:10926000B9F0A30192010E94DFD5362F272FB50157
:10927000A40177FF03C040E050E0BA01832E922E94
:109280005C01481559056A057B0514F44A015B0128
:10929000C355DF4F88829982AA82BB82CD5AD040C3
:1092A000C655DF4F8881CA5AD0408F708066C65538
:1092B000DF4F8883CA5AD040B0CFC501B40124E63D
:1092C00030E040E050E00E94C0D5E20EF31E041FE3
:1092D000151F411451046104710461F017FF03C0AC
:1092E000E12CF12C87014E145F046006710614F422
:1092F00083017201C355DF4FE882F9820A831B8321
:10930000CD5AD0408ACFC355DF4F688179818A8199
:109310009B81CD5AD0400E9426D77B018C01C5018C
:10932000B40124E630E040E050E00E94C0D5CA011C
:10933000B9016E0D7F1D801F911F411451046104FE
:10934000710461F097FF03C060E070E0CB01461646
:1093500057066806790614F4C301B2010E945BD473
:10936000C355DF4F688379838A839B83CD5AD0406E
:1093700054CFC355DF4F88819981AA81BB81CD5AD3
:10938000D040880E991EAA1EBB1E411451046104D0
:109390007104C9F0A4E6B0E0A30192010E94DFD5F8
:1093A000362F272FB501A40177FF03C040E050E01E
:1093B000BA01832E922E5C01481559056A057B057A
:1093C00014F44A015B01C355DF4F88829982AA8257
:1093D000BB82CD5AD04021CF88E0FE013196DE011C
:1093E000A755BF4F01900D928A95E1F7B12CA12CA2
:1093F0005524539416CFC655DF4F8881CA5AD040A2
:1094000082958F70823009F051C0C501B40124E605
:1094100030E040E050E00E94C0D5C155DF4F888168
:10942000CF5AD040C055DF4F6881C05BD040962FE7
:109430009170280F391F2E36E1E03E072CF437FFDC
:1094400005C02DE631E002C030E020E0C155DF4F1D
:109450002883CF5AD040C055DF4F8881C05BD040B1
:1094600030FB80F9C055DF4F8883C05BD04062E09D
:10947000CE0187559F4F0E94FE3562962FAF6297AF
:1094800063963FAF639764964FAF649765965FAFFF
:10949000659766966FAF669767967FAF6797689692
:1094A0008FAF689769969FAF6997E4CC88E0FE011B
:1094B0003196DE01A755BF4F01900D928A95E1F7D5
:1094C0009CCCCF53DF4FD880C15CD040DD20E1F091
:1094D0001296ED91FC9190859F709530A9F4C5543A
:1094E000DF4F28813981CB5BD0402530310561F0D9
:1094F000CF54DF4F48815981C15BD040BE016755D1
:109500007F4FCF010E945252C755DF4F8881C95A01
:10951000D040853009F4CAC020F4833079F1C50108
:109520006CC0863009F47CC08730C9F7C1010E9445
:10953000D31C182F863009F062C06BEA78E08BE10B
:109540009FE00E94C28666E070E08BE19FE00E948F
:1095500087998BE19FE00E942C8562E0CE018755C0
:109560009F4F0E94253629AF3AAF4BAF5CAF6DAF2E
:109570007EAF8FAF21969FAF21973CC0C1010E9463
:10958000D31C853019F003E010E083C96CEB78E060
:109590008BE19FE00E94C28665E070E08BE19FE076
:1095A0000E9487998BE19FE00E942C85B101CE013A
:1095B00087559F4F0E94F99D61E0CE0187559F4FCF
:1095C0000E94253622962FAF229723963FAF2397EE
:1095D00024964FAF249725965FAF259726966FAFB9
:1095E000269727967FAF279728968FAF289729969B
:1095F0009FAF2997C50181609160D12C30C063E98C
:1096000078E08BE19FE00E94C286612F70E08BE1E1
:109610009FE00E9487998BE19FE00E942C85B3CF49
:10962000C1010E94125318161906CCF1B101CE01E6
:1096300087559F4F0E94F99D61E0CE0187559F4F4E
:109640000E94253629AB3AAB4BAB5CAB6DAB7EAB26
:109650008FAB98AFC5018160916046E0D42E5C016C
:109660006894A0F8C655DF4F2881CA5AD040322FDF
:109670003F70323058F4C755DF4F3881C95AD04057
:10968000332321F05C016894A0F8B0F8207F59F1F1
:109690006894B1F801E010E0511079C432C26FE76C
:1096A00078E08BE19FE00E94C2866DCFC1010E94ED
:1096B000125318161906A4F462E0CE0187559F4F85
:1096C0000E94253629A73AA74BA75CA76DA77EA7BE
:1096D0008FA798ABC5018160916035E0D32EBFCFD5
:1096E00068E678E0DECF40E052E0B101CE01875578
:1096F0009F4F0E9433358111CBCFCCCF3FEFD31298
:10970000AAC0C1010E941253DD24D3941816190671
:109710000CF4A4C0D12C60E678E08BE19FE00E94BD
:10972000C2868D2C0D2C000C9908B4018BE19FE0B2
:109730000E94879969E578E08BE19FE00E94C286EC
:109740006C2D70E08BE19FE00E9487998BE19FE098
:109750000E942C85CF54DF4FE880F980C15BD04058
:10976000E114F10409F483C064E17AE0C7010E94C6
:109770007ECB01E010E0892B09F44BC060E17AE078
:10978000C7010E947ECB02E010E0892B09F441C0A2
:1097900067EA77E0C7010E947ECB05E010E0892BE5
:1097A000C1F163EA77E0C7010E947ECB06E010E0DA
:1097B000892B79F165ED79E0C7010E947ECB0AE043
:1097C00010E0892B31F160ED79E0C7010E947ECB7A
:1097D0000BE010E0892BE9F06AED79E0C7010E9407
:1097E0007ECB0CE010E0892BA1F063EC79E0C7019F
:1097F0000E947ECB0DE010E0892B59F06CEC79E0F3
:10980000C7010E947ECB10E000E0892B11F40EE02E
:1098100010E0C1010E94D31C682E712C61147104E8
:1098200009F434010115110509F440C060167106F0
:10983000C1F063E478E08BE19FE00E94C286B3014F
:109840008BE19FE00E9487998BE19FE00E942C852D
:109850000DEF1FEF1EC8DD2009F45DCFCC24C394AB
:109860005ACFCF54DF4F19821882C15BD040C75501
:10987000DF4F9881C95AD0409F3008F02BC1E92FA3
:10988000F0E08827E95BF34B8F4F0C9429D6794D94
:10989000454D364D904C794D1D4DFA4CD24C794D7D
:1098A000794D524D524D524D524D524DD101199656
:1098B0008D919C91009711F40C944744DC01ED913B
:1098C000FC910488F589E02DC755DF4F0881C95AFE
:1098D000D040C655DF4F1881CA5AD040C555DF4F1A
:1098E0002881CB5AD040C455DF4F3881CC5AD04064
:1098F000C355DF4F4881CD5AD040C255DF4F588104
:10990000CE5AD040C155DF4F6881CF5AD040C055A4
:10991000DF4F7881C05BD04019958C010C9449448D
:10992000C1010E94D31C853009F02DCE64E378E09C
:109930008BE19FE00E94C28665E070E08BE19FE0D2
:109940000E9487998BE19FE00E942C85B101CE0196
:1099500087559F4F0E94F99DF1018085853099F4CC
:109960006CE0CE0187559F4F0E94253629A33AA36C
:109970004BA35CA36DA37EA38FA398A76894A0F8C4
:10998000B0F8D12C52C061E0CE0187559F4F0E94A4
:109990002536298F3A8F4B8F5C8F6D8F7E8F8F8FFF
:1099A00098A3ECCFC1010E94D31C182F8630F9F484
:1099B00063E278E08BE19FE00E94C28666E070E09F
:1099C0008BE19FE00E9487998BE19FE00E942C85AC
:1099D00062E0CE0187559F4F0E942536298B3A8B36
:1099E0004B8B5C8B6D8B7E8B8F8B988FC7CF6BE097
:1099F00078E007CED1101EC0B101CE0187559F4F30
:109A00000E94F99D61E0CE0187559F4F0E94253647
:109A100029873A874B875C876D877E878F87988BEE
:109A20006894A0F8B0F826E0D22E0FEF1FEFCC24F8
:109A3000C39432CE67EF77E034CEDD20A1F062E050
:109A4000CE0187559F4F0E94253629833A834B8349
:109A50005C836D837E838F8398876894A0F8B0F8C9
:109A600095E0D92EE2CF60EE77E01BCEC655DF4FF2
:109A70008881CA5AD0408F708230C8F5C1010E94D7
:109A8000D31C853009F07ACF7ECDC655DF4F888153
:109A9000CA5AD0408F70823050F5DD2019F06DEC3D
:109AA00077E0FFCDC655DF4F8881CA5AD040282FB6
:109AB0002F702230E0F49923D1F0807F31F4B1018E
:109AC000CE0187559F4F0E94F99D6894A0F8F3E05E
:109AD000BF2A57CFC655DF4F8881CA5AD040807FF2
:109AE00019F46894B0F84DCF23E0B22A4ACFCC24C1
:109AF000C39451104CC2D12C0FEF1FEFA114B1042D
:109B000039F0A501B101CE0187559F4F0E94B734AE
:109B1000D10119968D919C91009709F482C0CF5480
:109B2000DF4FE880F980C15BD040DC01ED91FC9112
:109B30000488F589E02DC755DF4F0881C95AD04008
:109B4000C655DF4F1881CA5AD040C555DF4F28810E
:109B5000CB5AD040C455DF4F3881CC5AD040C35582
:109B6000DF4F4881CD5AD040C255DF4F5881CE5A81
:109B7000D040C155DF4F6881CF5AD040C055DF4F2C
:109B80007881C05BD04019958C01F1018185928567
:109B9000DC01ED91FC91028CF38DE02D1995059778
:109BA00011F46894A0F8DD2021F06D2DC1010E9410
:109BB000A11CC554DF4FE881F981CB5BD0403597BC
:109BC00021F0B501C1010E94364163EB77E08BE1E2
:109BD0009FE00E94C286B8018BE19FE00E948799B6
:109BE0006CEA77E08BE19FE00E94C2860E9414A796
:109BF000AB01BC01C354DF4FC880D980EA80FB8031
:109C0000CD5BD0404C195D096E097F092AE08BE1DC
:109C10009FE00E94E0848BE19FE00E942C850C94E1
:109C20004944F1018085853009F464C0863009F02B
:109C3000BACF70E060E0C1010E94B01B7C010097C8
:109C400009F4B1CF912C812C97FF06C0F194E194D7
:109C5000F10888248394912CC701019786359105DA
:109C600008F0A1CFC755DF4F0881C95AD04010E096
:109C7000CE2C61E08E2D0E948AA5892859F10130F1
:109C8000110521F061E00C30110509F460E0062FA8
:109C900010E08C2D0E945CA568EC77E08BE19FE0E2
:109CA0000E94C286B7018BE19FE00E94879966EC13
:109CB00077E08BE19FE00E94C286B8018BE19FE0D4
:109CC0000E9487998BE19FE00E942C856894A0F800
:109CD000B0F88AC00130110551F091E080E00C30FD
:109CE000110509F090E0092F182F602FD2CF01E065
:109CF00010E0FBCFCD54DF4F28813981C35BD040CA
:109D00002230310509F473C02C30310529F021309F
:109D1000310509F048CFDACFC1010E94941B892B8D
:109D200049F4D101ED91FC916081718189E195E067
:109D30000E94FDA7CE0187559F4F0E94AF1320E0E0
:109D400030E048EC52E40E94BAD40E9426D7C954AD
:109D5000DF4F688379838A839B83C75BD040C95474
:109D6000DF4F48805980C75BD04088E00E94FE17D3
:109D7000CD54DF4F688379838A839B83C35BD04054
:109D8000CD54DF4F68807980C35BD04062EC77E0D0
:109D90008BE19FE00E94C286C954DF4F68817981C0
:109DA000C75BD0408BE19FE00E9487996DEB77E025
:109DB0008BE19FE00E94C286CD54DF4F48815981DC
:109DC0006A817B81C35BD040662777272AE08BE1DD
:109DD0009FE00E94E0848BE19FE00E942C85B3010C
:109DE000A201C1010E94642501E010E0DCCE68946C
:109DF000A0F8B1F8F9CF0E949B38672B682B692B2C
:109E000011F00C94B846B12CA12C0C94E946CD5419
:109E1000DF4FC880D980C35BD040CD2809F053C044
:109E20008081882311F40C94C843CE018F549F4F36
:109E30000E94F642CD54DF4F99838883C35BD040A4
:109E4000C655DF4F8881CA5AD0408F7091F5CD54E6
:109E5000DF4F6881C35BD040CE0187559F4F0E9482
:109E6000FE35CF55DF4F2883C15AD040CE55DF4F46
:109E70003883C25AD040CD55DF4F4883C35AD040B3
:109E8000CC55DF4F5883C45AD040CB55DF4F688341
:109E9000C55AD040CA55DF4F7883C65AD040C955FD
:109EA000DF4F8883C75AD040C855DF4F9883C85AC0
:109EB000D040CD54DF4FC880D980C35BD040CD287F
:109EC00011F40C94C8430E94EB116B01C954DF4F8D
:109ED00079836883C75BD0406DE379E08BE19FE0D5
:109EE0000E94C286B6018BE19FE00E94879966E3DB
:109EF00079E08BE19FE00E94C286D101ED91FC9157
:109F0000608171818BE19FE00E945C8660E379E073
:109F10008BE19FE00E94C286CF54DF4F6881798138
:109F2000C15BD0408BE19FE00E945C866EE279E0ED
:109F30008BE19FE00E94C286C954DF4FE881F9811E
:109F4000C75BD04060E279E0E83CF10514F40C9482
:109F50001946CE0187559F4F0E94C333CF54DF4F20
:109F6000E881F981C15BD040309711F40C9414441E
:109F70008081843211F00C9414446CE079E08BE120
:109F80009FE00E94C2868BE19FE00E942C850CEF2F
:109F90001FEF0C9449442F923F924F925F926F9221
:109FA0007F928F929F92AF92BF92CF92DF92EF9269
:109FB000FF920F931F93CF93DF93CDB7DEB7A69792
:109FC0000FB6F894DEBF0FBECDBF5C013B015090D1
:109FD000DA06552009F4B8C080918C088F5F809311
:109FE0008C08E0919008F0919108309709F4A4C092
:109FF0008680978020909008309091082114310439
:10A0000009F496C08114910409F492C0D401189601
:10A010008C918F70853091F7C4010E948F998230A6
:10A0200068F3B401CE0101960E946B23CE01019624
:10A030000E941814882309F45EC060E074E0CE0129
:10A0400001960E94871C892B09F455C01E8E1F8E15
:10A0500018A219A21AA21BA21CA21DA28F8D8F707A
:10A060008F8F40E053E0BE016F5F7F4FCE014E9671
:10A070000E94333561E879E08BE19FE00E94C2865F
:10A0800060E074E0CE0101960E943D1C8A859B85AC
:10A09000009789F1DC01ED91FC910488F589E02DB0
:10A0A000CC24C394F12CE12C0E8D1F8D28A139A155
:10A0B0004AA15BA16CA17DA119958F3F9807D9F0AA
:10A0C000E981FA8160817181892BE9F48BE19FE05C
:10A0D0000E945C866FE779E08BE19FE00E94C28678
:10A0E00067E779E08BE19FE00E94C2868BE19FE009
:10A0F0000E942C85512CF40182809380CE01019620
:10A100000E944E1477CF8BE19FE00E945C8665E74A
:10A1100079E08BE19FE00E94C28661E779E08BE104
:10A120009FE00E94C2868BE19FE00E942C85E3CFD6
:10A130008BE19FE00E942C8580918C088150809358
:10A140008C0851101092DA0665E0D5018D919C9132
:10A150000E947A994C01009709F487C0FC01808520
:10A1600085958595859585958EA321843284438434
:10A1700054840E9414A7FEA1FF2309F476C0261A76
:10A18000370A480A590A1E8E1F8E18A219A2FE8F7E
:10A190001F8D1F70106A1F8F2AA23BA24CA25DA2C6
:10A1A00024E06216710449F5D12CC12CE12C90E118
:10A1B000F92E0F2F28A139A14AA15BA16CA17DA185
:10A1C000C5010E944736C201B10128EE33E040E0EC
:10A1D00050E00E94C0D5BA01A9012AE030E08BE12D
:10A1E0009FE00E94D28566E979E08BE19FE00E94C2
:10A1F000C2868BE19FE00E942C8557FE36C082E02C
:10A2000028163104410480E858067CF1D12CC12C79
:10A21000E12C80E1F82E0E8D1F8D28A139A14AA1D5
:10A220005BA16CA17DA1C5010E94473619821A82EB
:10A230001B821C821D821E821F8218861A811F703B
:10A240001A83AEA1A983CC24C394F12CE12C0A2F4C
:10A250002B813C8140E05E816F817885C5010E9441
:10A260002A43F40180858F708087F1E06F167104B6
:10A27000B9F460E073E0C5010E94871C009781F08B
:10A2800020918E0830918F082630310549F4BC01A9
:10A29000C5010E94364160E073E0C5010E943D1C8B
:10A2A000D50119968D919C910097D9F490E080E0AA
:10A2B000A6960FB6F894DEBF0FBECDBFDF91CF914B
:10A2C0001F910F91FF90EF90DF90CF90BF90AF90D4
:10A2D0009F908F907F906F905F904F903F902F90C6
:10A2E0000895DC01ED91FC910484F585E02D19952C
:10A2F000892BE1F2F50181859285DC01ED91FC91DC
:10A300000480F581E02DB3011995D2CFAF92BF92B1
:10A31000CF92DF92EF92FF920F931F93CF93DF9331
:10A32000CDB7DEB76D970FB6F894DEBF0FBECDBFC9
:10A330000E9414A79B01AC016091EC067091ED06A0
:10A340008091EE069091EF06A12CB12C650118EEDC
:10A35000E12E13E0F12E00E010E00E94C82AF82E52
:10A36000882351F00E9414A76093EC067093ED06C9
:10A370008093EE069093EF0680918C088F5F809318
:10A380008C08E0919008F09191080681178194E083
:10A39000C92ED12CF11003C082E0C82ED12CA09080
:10A3A0009008B0909108A114B10429F1011511058C
:10A3B00011F1F80180858F708530A9F7C8010E94DE
:10A3C0008F99823080F3B801CE0101960E946B23F1
:10A3D000CE0101960E941814882329F0B601CE01FF
:10A3E00001960E94CB4FF80102811381CE010196A4
:10A3F0000E944E14D4CF80918C08815080938C0899
:10A4000080918E0890918F080597D9F1FF20C9F1AE
:10A4100010E06091F4067091F5066115710589F1FF
:10A4200011112FC0FB0180858F70853091F4CE0112
:10A4300001960E946B2361E070E0CE0101960E94BC
:10A44000CB4F11E0892B09F410E0CE0101960E9458
:10A450004E14E091F406F091F506309791F0828168
:10A4600093819093F5068093F406892B91F6E09101
:10A470009008F0919108868197819093F5068093DA
:10A48000F4066D960FB6F894DEBF0FBECDBFDF9118
:10A49000CF911F910F91FF90EF90DF90CF90BF90E1
:10A4A000AF9008954F925F926F927F928F929F929A
:10A4B000AF92BF92CF92EF92FF920F931F93CF93E1
:10A4C000DF93CDB7DEB76D970FB6F894DEBF0FBE42
:10A4D000CDBF009709F4A4C0FC0120852F70253062
:10A4E00009F09EC02A015B018680978080918C08CC
:10A4F0008F5F80938C088114910409F48CC0F4015F
:10A5000080858F70843009F082C06185728580916A
:10A510009008909191080E9405993C01009709F4D8
:10A5200076C0FC0180858F70853009F070C0B30162
:10A53000CE0101960E946B23A114B104A9F0CE01B3
:10A5400001960E941814882379F0C12C7201F5013C
:10A550000081118122813381448155816681778117
:10A56000CE0101960E942A4360E0C3010E947A99BD
:10A570000097D1F1FC0120852F702230A9F581854B
:10A580009285A385B4850797A105B10569F561E0BA
:10A59000C3010E947A99A201B5010E945252A114EE
:10A5A000B10489F5882379F180918C0881508093DA
:10A5B0008C08CE0101960E944E1481E06D960FB674
:10A5C000F894DEBF0FBECDBFDF91CF911F910F91E9
:10A5D000FF90EF90CF90BF90AF909F908F907F9023
:10A5E0006F905F904F900895A114B10461F4CE0173
:10A5F00001960E941814882331F0CE0101960E9422
:10A600001253892B89F6CE0101960E944E14F40153
:10A610008280938070CF80918C08815080938C08C9
:10A6200080E0CCCFDF92EF92FF920F931F93CF93F6
:10A63000DF9300D000D01F921F92CDB7DEB77C0110
:10A6400019821A821B821C821D821E821F8218861A
:10A650008A818F708A83D701ED91FC91608171812D
:10A660008BE19FE00E945C866FE679E08BE19FE0E2
:10A670000E94C286C7010E94181481111BC066E6A1
:10A6800079E08BE19FE00E94C2868BE19FE00E940F
:10A690002C850FEF1FEFC80128960FB6F894DEBF88
:10A6A0000FBECDBFDF91CF911F910F91FF90EF9023
:10A6B000DF900895C7010E94D31CD82EF701818531
:10A6C0009285009791F0DC01ED91FC910688F78965
:10A6D000E02D19958C0197FD08C081E00115110549
:10A6E00009F480E00E947218D6CFF7018085873088
:10A6F00059F0F5E0DF1689F1FD15F8F081E0D81684
:10A7000019F1A2E0DA1649F140E052E0B701CE01BA
:10A7100001960E943335F7018085873009F445C0E2
:10A7200010F5833009F46AC0843011F167E579E0EF
:10A730008BE19FE00E94C28613C0B6E0DB1621F0D9
:10A7400086EF8D0D833000F767E479E08BE19FE0C1
:10A750000E94C28601E010E09ECF80E00E94721845
:10A7600010E000E098CF883009F448C08930F1F655
:10A7700060E0CE0101960E94E2128C016CE479E067
:10A780008BE19FE00E94C286B8018BE19FE00E94AE
:10A7900087998BE19FE00E942C8591E080E0012B5E
:10A7A00009F490E0092F182F76CF0280F381E02D75
:10A7B00080858F7010E000E0853001F764E679E075
:10A7C0008BE19FE00E94C28650E040E070E060E0D4
:10A7D000F701828193810E945252F82E082F10E0D7
:10A7E00061E679E08BE19FE00E94C2868F2D0E9496
:10A7F00072188BE19FE00E942C854DCFCE0101960F
:10A800000E949B388B01BACF2F923F924F925F925A
:10A810006F927F928F929F92AF92BF92CF92DF9270
:10A82000EF92FF920F931F93CF93DF93CDB7DEB7D5
:10A8300060970FB6F894DEBF0FBECDBF61307105D3
:10A8400009F495C0DC0112966D917C91611571053A
:10A8500009F48DC04C0119821A821B821C821D8250
:10A860001E821F8218868A818F708A8340E052E0A0
:10A87000CE0101960E94333560E0CE0101960E9420
:10A88000E2121C01F401828193810E94941B2B012E
:10A890003C01D40117962D913D914D915C911A97F1
:10A8A000D1010E94EAD52FEF30E040E050E00E9455
:10A8B0009ED529873A874B875C870E9414A79B0106
:10A8C000AC0189859A85AB85BC850097A105B1054A
:10A8D00009F468C0A12CB12C65017C018D01C30174
:10A8E000B2010E94C82A898741145104610471048D
:10A8F000F1F1D40117968D919D910D90BC91A02DF1
:10A900008D879E87AF87B88B0E9414A79B01AC01EF
:10A910008D859E85AF85B8890097A105B10561F049
:10A92000A12CB12C65017C018D01C301B2010E94F3
:10A93000C82A882309F451C0D40112966D907C90E6
:10A9400080E00E94FE17AB01BC01C3010E94642598
:10A95000232869F0F40184810E943F11D4011696E6
:10A960009C91891304C061E0C4010E94E01C90E046
:10A9700080E060960FB6F894DEBF0FBECDBFDF91CA
:10A98000CF911F910F91FF90EF90DF90CF90BF90EC
:10A99000AF909F908F907F906F905F904F903F907F
:10A9A0002F90089591E099879FCFB985BB23F1F04F
:10A9B00060E0C4010E94E01CF401828193810E9446
:10A9C0001253892BA1F640E050E0BA01D40112964F
:10A9D0008D919C910E946425CACFF40184810E94CC
:10A9E0003F11D40116969C918913DFCF232809F4D7
:10A9F000BECFF40184810E943F11D40116969C9130
:10AA00008913B5CFB985B111B2CFADCFCF93DF9355
:10AA1000EC016BEC76E18BE19FE00E94C2866C81D9
:10AA20007D818BE19FE00E94879965EC76E18BE167
:10AA30009FE00E94C2868BE19FE00E942C8561E02E
:10AA40008C810E948AA56E818C810E945CA58A817E
:10AA50009B81009729F040E050E0BA010E946425F4
:10AA600081E090E09093C4078093C3078A819B8123
:10AA70000E941253181619065CF40A80DB81C02D5F
:10AA800080E00E94FE17AB01BC01CE010E9464254C
:10AA900081E090E0DF91CF9108952F923F924F9205
:10AAA0005F926F927F928F929F92AF92BF92CF925E
:10AAB000DF92EF92FF920F931F93CF93DF93CDB767
:10AAC000DEB7C955D1090FB6F894DEBF0FBECDBFB2
:10AAD0000E9414A79B01AC016091E8067091E90601
:10AAE0008091EA069091EB06A12CB12C650110E350
:10AAF000E12E15E7F12E00E010E00E94C82A88231D
:10AB000009F401C2E0919008F0919108309709F49E
:10AB1000FAC180918C088F5F80938C0826803780E3
:10AB200010E02114310409F434C1F10180858F70E3
:10AB30008530F9F460E0C1010E947A99FC018185B9
:10AB40009285A385B4850597A105B10591F4B1015E
:10AB5000CE0101960E946B23CE0101960E9418142B
:10AB600066968FAF6697811108C0CE0101960E944C
:10AB70004E14F10122803380D4CF25961CAE1DAE39
:10AB80001EAE1FAE259729961CAE1DAE1EAE1FAE83
:10AB9000299740E052E0BE016F5F7F4FCE018F5B8F
:10ABA0009F4F0E943335CE0101960E94941B6B018A
:10ABB0007C0169966FAF69976A96DFAE6A9770E01D
:10ABC00060E0CE0101960E94B01B4C01CE018F5B6C
:10ABD0009F4F0E94AF1365966CAF7DAF8EAF9FAF56
:10ABE0006597CE0101960E94D31C182FB601DD0C8B
:10ABF000880B990B0E945BD420E030E048EC52E4D3
:10AC00000E94B4D62B013C01CE0101960E94125342
:10AC100068969FAF8EAF689769EA73E18BE19FE01A
:10AC20000E94C28665966CAD7DAD8EAD9FAD659779
:10AC30000E9429A163EA73E18BE19FE00E94C28632
:10AC4000C301B2010E9429A16DE973E18BE19FE08C
:10AC50000E94C286612F70E08BE19FE00E9487997D
:10AC6000E114F10409F48EC088E00E94FE179B01F4
:10AC7000AC0144275527B70190E080E0AA24AA94AC
:10AC8000BA2CC12CD12C17E2E12E19E0F12E00E0F4
:10AC900010E00E94C82A882371F1F101608171815E
:10ACA00084EF9DE00E945C866DE873E184EF9DE097
:10ACB0000E94C286F1016081718188E295E00E9464
:10ACC000FDA790E080E0BC0169964FAD69976A9658
:10ACD0005FAD6A97CE0101960E94642562E070E044
:10ACE000C4010E947C1ACE0101960E944E14669601
:10ACF0001FAD66973ECF20E030E048E152E4C3014B
:10AD0000B2010E945CD718163CF4F1016081718198
:10AD100084E395E00E94FDA768968EAD9FAD68978D
:10AD2000892B19F461E070E0DBCF20E030E040E8EF
:10AD30005FE365966CAD7DAD8EAD9FAD65970E946E
:10AD400047D69B01AC01C301B2010E9454D470E00C
:10AD500060E087FDC5CFA301920165966CAD7DAD26
:10AD60008EAD9FAD65970E9454D41816DCF66EE741
:10AD700073E18BE19FE00E94C2868BE19FE00E941D
:10AD80002C85B1CF64E773E18BE19FE00E94C2861E
:10AD9000AACF80918C08815080938C080E9414A7C0
:10ADA0006093E8067093E9068093EA069093EB06B9
:10ADB0000E94EB112B013C010E9414A76B017C0146
:10ADC0000E942099882309F466C080911A08811195
:10ADD00062C030E020E041E050E060E4CE01019646
:10ADE0000E94BE2D40E450E064E879E1CE01019676
:10ADF0000E9497CB6AEF74E0CE0101960E9474DA4C
:10AE000040E450E06BE473E1CE0101960E9497CBE1
:10AE1000B301A201CE018F5B9F4F0E945611BE016C
:10AE20006F5B7F4FCE0101960E94E2A730E020E0E9
:10AE300041E050E060E4CE0101960E94BE2D40E466
:10AE400050E064E879E1CE0101960E9497CB6AEF69
:10AE500074E0CE0101960E9474DA40E450E064E4AC
:10AE600073E1CE0101960E9497CBC701B60128EE8F
:10AE700033E040E050E00E949ED5BA01A901CE0126
:10AE80008F5B9F4F0E945611BE016F5B7F4FCE01BB
:10AE900001960E94E2A7112309F44FC06EE673E108
:10AEA0008BE19FE00E94C2860E94EB11AB01BC01C6
:10AEB0002AE08BE19FE00E94E08466E673E18BE18B
:10AEC0009FE00E94C28660918C08062E000C770BD2
:10AED0008BE19FE00E94879964E573E18BE19FE03D
:10AEE0000E94C2864091E4065091E5066091E60614
:10AEF0007091E7062AE08BE19FE00E94E0848BE1FD
:10AF00009FE00E942C85C75ADF4F0FB6F894DEBF32
:10AF10000FBECDBFDF91CF911F910F91FF90EF90AA
:10AF2000DF90CF90BF90AF909F908F907F906F9069
:10AF30005F904F903F902F90089564E673E18BE10E
:10AF40009FE00E94C2860E94EB11AB01BC012AE087
:10AF50008BE19FE00E94E0846CE573E1B0CF8F92BB
:10AF60009F92AF92BF92CF92DF92EF92FF920F9398
:10AF70001F93CF93DF93CDB7DEB767970FB6F894E3
:10AF8000DEBF0FBECDBF8C017B014C018BE0880E74
:10AF9000911C9F8A8E8AF801128611861386148E60
:10AFA000138E672B09F463C0A0909008B0909108AD
:10AFB000A114B10409F45BC06FE270E0C7010E9404
:10AFC0007FDA6C01892B09F44AC0F701DE01119682
:10AFD00090E080E0BD012191222341F02F3231F039
:10AFE0008431910519F02D930196F5CF860F971FA7
:10AFF000FC011082C5010E940599F80191838083AC
:10B00000B6016F5F7F4F4FE050E0C4010E94B8DA95
:10B01000CE0146960E94F642F801948F838F8E8966
:10B020009F89892B09F41386C8010E94181488236C
:10B0300019F0C8010E94FE2167960FB6F894DEBF92
:10B040000FBECDBFDF91CF911F910F91FF90EF9079
:10B05000DF90CF90BF90AF909F908F900895B701F1
:10B06000C5010E940599F80191838083DDCFF80125
:10B0700011821082D9CF2F923F924F925F926F929E
:10B080007F928F929F92AF92BF92CF92DF92EF9278
:10B09000FF920F931F93CF93DF93CDB7DEB7C955C0
:10B0A000D1090FB6F894DEBF0FBECDBF3C01562EBE
:10B0B0006296EFAE62976396FFAE639764960FAFAA
:10B0C000649765961FAF659766962FAF66976796EC
:10B0D0003FAF679768964FAF689769965FAF69977C
:10B0E0006A96CFAE6A972D2C4A2C3B2C009709F418
:10B0F0005CC1FC0180858295807F859585958595CD
:10B100008595843009F43CC12CF4882309F441C1AD
:10B1100080E02DC0853009F444C08630C9F761E471
:10B1200075E0C3010E9405994C01009709F46FC0B6
:10B13000B12CA12CD12CC12C6296EFAC62976396F6
:10B14000FFAC639764960FAD649765961FAD6597E6
:10B1500066962FAD669767963FAD679768964FAD39
:10B16000689769965FAD6997652D0E943B58C75AED
:10B17000DF4F0FB6F894DEBF0FBECDBFDF91CF918A
:10B180001F910F91FF90EF90DF90CF90BF90AF9005
:10B190009F908F907F906F905F904F903F902F90F7
:10B1A000089580918C088F5F80938C0886809780AB
:10B1B0008114910431F1A42CB32C6A96CFAC6A9718
:10B1C000D22C6296EFAC62976396FFAC639764965D
:10B1D0000FAD649765961FAD659766962FAD669720
:10B1E00067963FAD679768964FAD689769965FAD74
:10B1F0006997652DC4010E943B58F40182809380B9
:10B20000D7CF80918C08815080938C0881CF65E4E2
:10B2100075E0C3010E9405997C016AE475E0C301F1
:10B220000E9405996C01552039F0F1E05F1609F490
:10B2300088C010E000E00CC06FE475E0C3010E941C
:10B2400005994C0164E575E0C3010E9405998C01E4
:10B250008114910409F443010115110509F48301D6
:10B26000E114F10421F46A96EFAC6A97F22CC11450
:10B27000D10411F4C42CD32C8114910409F492C08C
:10B28000F40180858F70843009F08CC081849284B1
:10B290000115110509F491C0F80180858F70843083
:10B2A00009F08BC001851285E114F10409F4C9C0CD
:10B2B0008114910409F490C064EA77E18BE19FE086
:10B2C0000E94C286F701618572858BE19FE00E9432
:10B2D0005C866FE977E18BE19FE00E94C286B40152
:10B2E0008BE19FE00E945C868BE19FE00E942C85B1
:10B2F000CE018F5A9F4F0E94C333C114D10409F06D
:10B30000F8C0F70180858F70843009F0F0C0618546
:10B310007285CE0101960E94AF57CE0101960E9420
:10B320001814882349F08114910409F469C0B40108
:10B33000CE0101960E948E9ECE0101960E944E146F
:10B34000D6C069E575E0C3010E9405994C016EE520
:10B3500075E0C3010E9405998C018114910409F0E4
:10B36000CDC06FE475E0C3010E9405994C01011541
:10B37000110509F467CF892B09F072CF430170CF13
:10B3800010E000E0912C812CD12CC12CF12CE12C6F
:10B390005FCF10E000E0912C812CD12CC12CF12C3E
:10B3A000E12C5ECF912C812C73CFCA2CDB2C6A96BA
:10B3B000EFAC6A97F22C912C812C00E020E033E076
:10B3C00040E150E0BE016F5B7F4FCE018F5A9F4F2F
:10B3D0000E9413208C0168CF65E977E18BE19FE043
:10B3E0000E94C286F701618572858BE19FE00E9411
:10B3F0005C8660E977E18BE19FE00E94C28678CFAE
:10B40000CC24C394F12CE12C62960FAD6297639625
:10B410001FAD639764962FAD649765963FAD6597B2
:10B4200066964FAD669767965FAD679768966FAD06
:10B43000689769967FAD6997CE0101960E942A436D
:10B440007BCFC114D10409F452C00115110509F4D0
:10B450004EC0F60180858F70843009F044C069E8E1
:10B4600077E18BE19FE00E94C286F60161857285DB
:10B470008BE19FE00E945C8664E877E18BE19FE0CE
:10B480000E94C286B8018BE19FE00E945C868BE13E
:10B490009FE00E942C85F6016185728540E450E0B2
:10B4A000CE0101960E94B8DA0E9420998823D9F033
:10B4B00080911A08811117C06FE270E0CE010196E9
:10B4C0000E947FDA892B51F4F6012185328543E011
:10B4D00050E060E4CE0101960E94BE2DB801CE017D
:10B4E00001960E94E2A7E114F10409F00ACF81E07D
:10B4F0003ECE0115110509F0ACCF03CF892B09F021
:10B50000AFCEA0CE2F923F924F925F926F927F92DA
:10B510008F929F92AF92BF92CF92DF92EF92FF9263
:10B520000F931F93CF93DF93CDB7DEB7E2970FB69C
:10B53000F894DEBF0FBECDBF9AA389A3098F1A8FDF
:10B540002B8F3C8F4D8F5E8F6F8F78A3FAAAE9AA5D
:10B55000DC011496ED91FC91309709F4D8C0668017
:10B56000778018AA1FA61AA619A6312C212C912C77
:10B57000812C512C412C6114710409F4D0C06BED65
:10B5800074E0C3010E9405995C016CEE74E0C30194
:10B590000E9405999EA38DA3A114B10409F4AFC024
:10B5A000892B09F4ACC0F50180858F70823009F0D9
:10B5B000A6C0ADA1BEA118968C918F70823009F003
:10B5C0009EC063E675E0C3010E940599DC011996EF
:10B5D0002D913D914D915C911C972BA73CA74DA7B8
:10B5E0005EA7E9A9FAA9309709F459C0D301CD9013
:10B5F000DC90BF01C6010E948ADA892B09F04FC096
:10B60000098D002309F1802F90E0B0E0A0E0EDA1CA
:10B61000FEA181879287A387B48780918E0890913D
:10B620008F08059789F0E12CFF24F3941A8D2B8D58
:10B630003C8D4D8D5E8D6F8D78A1A9A1BAA112961A
:10B640008D919C910E9447361A8D812F807F39F110
:10B6500060E0CE0149960E94E212092E000CAA0B6E
:10B66000BB0BF50181879287A387B48780918E08F1
:10B6700090918F08059799F0D301CD90DC90E12C43
:10B6800092E0F92E098D2B8D3C8D4D8D5E8D6F8D49
:10B6900078A1E9A1FAA1828193810E944736D50160
:10B6A00019964D915D916D917C911C97EDA1FEA134
:10B6B00081859285A385B4850297A105B10521F105
:10B6C0002BA53CA5429FC001439F900D529F900D1A
:10B6D0001124480E591EABA5BCA58A0E9B1EEFA5D2
:10B6E000F8A98F01FF0F220B330B0417150726074C
:10B6F00037072CF458AB4FA79AA789A71D01D30190
:10B7000012966D907C9037CF90E080E0E4CF1AA63F
:10B7100019A6312C212C912C812C512C412C8114D7
:10B72000910409F486C0C201B4010E9415D67B01C0
:10B7300065E976E18BE19FE00E94C286B4018BE16E
:10B740009FE00E9487996AE876E18BE19FE00E9482
:10B75000C2860FEF10E0C201B8010E9415D68BE13E
:10B760009FE00E94879963E876E18BE19FE00E9469
:10B77000C286B7018BE19FE00E94879965E776E179
:10B780008BE19FE00E94C28689A59AA5B8010E941C
:10B7900015D68BE19FE00E9487996EE676E18BE1FA
:10B7A0009FE00E94C286B1018BE19FE00E948799D1
:10B7B0006AE676E18BE19FE00E94C2868BE19FE022
:10B7C0000E942C8519821A821B821C821D821E8275
:10B7D0001F8218868A818F708A83B701CE010196F5
:10B7E0000E94AD1279018A013B014C01298BFA8A32
:10B7F0004B8B1C8B6D8B7E8A8F8B988E6DE576E0E4
:10B80000E9A1FAA1848195810E940599B12CA12C0E
:10B81000D12CC12C9301A4016FEF0E943B58A9A128
:10B82000BAA11496ED91FC913097E9F488248394A1
:10B83000912CC401E2960FB6F894DEBF0FBECDBFC7
:10B84000DF91CF911F910F91FF90EF90DF90CF90FC
:10B85000BF90AF909F908F907F906F905F904F9030
:10B860003F902F900895868097809101330C440B70
:10B87000550B29A33AA34BA35CA389A59AA5092E2E
:10B88000000CAA0BBB0B8DA39EA3AFA3B8A781147A
:10B89000910461F263E675E0C4010E9405997C01A0
:10B8A00065E474E0C4010E9405993C016BED74E00D
:10B8B000C4010E9405995C016CEE74E0C4010E9411
:10B8C00005996114710409F4B6C0A114B10409F416
:10B8D000B2C0009709F4AFC0D30118962C912F7015
:10B8E000223009F0A8C0F50120852F70223009F020
:10B8F000A2C0DC0118962C9118972F70223009F005
:10B900009AC0F701C184D284E384F484C114D104C1
:10B9100009F491C019968D919D910D90BC91A02D27
:10B920000297A105B10509F48AC029A53AA5232BE0
:10B9300009F485C0D50119968D919C918C9D50017B
:10B940008D9DB00C9C9DB00C11242FEF30E0D501E3
:10B950000E9440D69601DD0C440B550B0E94C0D5C9
:10B9600069A17AA18BA19CA10E948ED52DA13EA197
:10B970004FA158A50E94C0D519012A01F401608188
:10B9800071818BE19FE00E945C8665E675E08BE14A
:10B990009FE00E945C86C5016FEF70E00E9415D6A3
:10B9A0008BE19FE00E94879964E676E18BE19FE05E
:10B9B0000E94C2862AE030E0B201A1018BE19FE043
:10B9C0000E94D2858BE19FE00E942C85F301818546
:10B9D0009285A385B48582159305A405B50559F113
:10B9E00019861A861B861C861D861E861F86188A47
:10B9F0008A858F708A87B101CE0109960E94AD12A7
:10BA000029833A834B835C836D837E838F839887FE
:10BA1000B12CA12CD12CC12C79018A019B01AC0144
:10BA20006FEFC4010E943B58D30119962D923D92AD
:10BA30004D925C921C97F4018280938028CF212C38
:10BA4000312C2101C3CF6F927F928F929F92AF9240
:10BA5000BF92CF92DF92EF92FF920F931F93CF93FB
:10BA6000DF93CDB7DEB7A0970FB6F894DEBF0FBE59
:10BA7000CDBF8C01862E7A01DC018D919C911197AE
:10BA8000892B09F466C01496ED91FC91309709F466
:10BA900060C080818071BFEF6B135DC0B1F481E045
:10BAA000A0960FB6F894DEBF0FBECDBFDF91CF9149
:10BAB0001F910F91FF90EF90DF90CF90BF90AF90CC
:10BAC0009F908F907F906F9008954330510539F388
:10BAD000818082942FE0822263E577E08BE19FE012
:10BAE0000E94C2864AE050E0D80113966C918BE127
:10BAF0009FE00E94308561E577E08BE19FE00E9446
:10BB0000C286D8011496ED91FC9161816F704AE074
:10BB100050E08BE19FE00E9430856EE477E08BE19E
:10BB20009FE00E94C2864AE050E0682D8BE19FE0D2
:10BB30000E9430858BE19FE00E942C85D8011496ED
:10BB4000ED91FC9181818F70881207C080818F7E7A
:10BB5000808380E0A5CF8111FCCF198E1A8E1B8EB9
:10BB60001C8E1D8E1E8E1F8E18A28A8D8F708A8F3E
:10BB7000D8011496ED91FC9181818F708815A9F1FF
:10BB8000B3E0EB16F10489F16CE477E08BE19FE020
:10BB90000E94C2864AE050E0F80163818BE19FE099
:10BBA0000E9430856AE477E08BE19FE00E94C286C4
:10BBB000D8011496ED91FC9161816F704AE050E0DC
:10BBC0008BE19FE00E94308567E477E08BE19FE0A6
:10BBD0000E94C2864AE050E0682D8BE19FE00E94FF
:10BBE00030858BE19FE00E942C85F8012081318116
:10BBF000FCE0F81508F416C1E82DF0E08827EC5FAA
:10BC0000F14A8F4F0C9429D6115E4E5ECF5EE65EF0
:10BC1000F25ECF5EA85ECF5EF55E005FBC5E035F46
:10BC20000F5FD8011496CD90DC90F60181818F7062
:10BC3000853009F4F7C050F48230C1F069E775E04F
:10BC4000C9010E9405993C01912C4BC08730D1F06D
:10BC50008A30A1F762E775E0C9010E9405993C01AD
:10BC6000D6019C9092FA992490F83BC06CE675E05E
:10BC7000C9010E9405993C01D6019C9090FA992433
:10BC800090F82FC06BE675E0C9010E9405993C0150
:10BC9000F601908091FA992490F823C06EE775E040
:10BCA000C9010E9405993C01D8011496ED91FC91BF
:10BCB000808180FB992490F8982F9E7F80FF91606F
:10BCC00090836114710469F461E0CE0149960E9489
:10BCD0002536298B3A8B4B8B5C8B6D8B7E8B8F8BB8
:10BCE000988FF801A080B18065E475E0C5010E94DD
:10BCF00005996C016AE475E0C5010E9405995C0133
:10BD0000892B81F4C114D10469F460E0CE01499615
:10BD10000E94253629833A834B835C836D837E831F
:10BD20008F839887D8011496ED91FC91611471046A
:10BD300009F07CC0898D811179C0B82DBF708B2E20
:10BD40008181807F882A818280818F7E8083A7CEB7
:10BD500063E875E0C9010E9405993C01D801149679
:10BD6000ED91FC91808181FB992490F8982F9D7F23
:10BD700081FF92609083B5CF69E875E0C9010E94A8
:10BD800005993C01D8011496ED91FC91808182FBCC
:10BD9000992490F8982F9B7F82FF9460EBCF69E7FE
:10BDA00075E0C9010E9405993C01892B09F04CCF2F
:10BDB00062E0CE0149960E94253629873A874B8753
:10BDC0005C876D877E878F87988B3ECF6FE875E0A5
:10BDD000C9010E9405993C01D8011496ED91FC918E
:10BDE00090804CCF64E975E0F3CF6AE975E0C90152
:10BDF0000E9405993C01D8011496ED91FC9149CF20
:10BE000060EA75E0F4CF67EA75E0C9010E94059920
:10BE10003C01D8011496ED91FC91908023CF6DEAFE
:10BE200075E0F3CF912C712C612C5BCF83E0E81689
:10BE3000F104B9F0982D9F70892E8181807F882A26
:10BE4000818280818F7E8083E98CFA8C0B8D1C8DA2
:10BE50002D8D3E8D4F8D58A1692DC3010E943B58F9
:10BE60001ECE81818F70881509F419CE829490EFCF
:10BE70008922882A81828081806168CF8F929F92F7
:10BE8000AF92BF92CF92DF92EF92FF920F931F93E8
:10BE9000CF93DF93CDB7DEB7CD55D1090FB6F89468
:10BEA000DEBF0FBECDBF8C016B016115710519F0AE
:10BEB00041155105D1F468EC7BE08BE19FE00E94D5
:10BEC000C2866FEB7BE08BE19FE00E94C286B801E7
:10BED0008BE19FE00E945C866DEB7BE08BE19FE055
:10BEE0000E94C2868BE19FE030C0460F571FDA01E7
:10BEF0001C920E94EB114B016BEB7BE08BE19FE00E
:10BF00000E94C286B4018BE19FE00E94879968EB92
:10BF10007BE08BE19FE00E94C286B8018BE19FE04D
:10BF20000E945C8665EB7BE08BE19FE00E94C2860D
:10BF3000BAE38B16B1E09B06F4F468EA7BE084EF89
:10BF40009DE00E94C28684EF9DE00E942C85C35A2A
:10BF5000DF4F0FB6F894DEBF0FBECDBFDF91CF919C
:10BF60001F910F91FF90EF90DF90CF90BF90AF9017
:10BF70009F908F90089566EA7BE08BE19FE00E949E
:10BF8000C286B6018BE19FE00E945C8664EA7BE09A
:10BF90008BE19FE00E94C2868BE19FE00E942C858E
:10BFA0001A821982FE0133968EE3DF011D928A9573
:10BFB000E9F780918E0890918F080597D9F563E095
:10BFC00070E0C8010E94522E7C01892B09F045C007
:10BFD000E0916E0DF0916F0D808180FFB8CF62E02F
:10BFE00070E0C8010E94522E892BD9F064E270E003
:10BFF000C8010E94C7DA892B09F0A9CF6CE87BE061
:10C000008BE19FE00E94C286B8018BE19FE00E9415
:10C010005C868BE19FE00E942C85C8010E94B9A339
:10C0200096CF61E070E0C8010E94522E892B09F47E
:10C030008ECFDCCF61E070E0C8010E94522E7C01FF
:10C04000892B21F562E070E0C8010E94522E7C012C
:10C0500061E87BE0892B09F441CFE00EF11E68E72F
:10C060007BE0C7010E947ECB892BC1F4F6010190D1
:10C070000020E9F73197EC19FD09329778F0C801F3
:10C080000E94B9A3C6010E94FF8B61CF4FE350E02D
:10C09000B801CE0101960E94B8DADFCF64E270E009
:10C0A000C8010E94C7DA892B09F051CFB701CE0130
:10C0B0008F5B9F4F0E94AF57CE018F5B9F4F0E94B7
:10C0C0001814882339F1B601CE018F5B9F4F0E946F
:10C0D0008E9E18161906F4F489818823D9F0809170
:10C0E0008E0890918F080597A9F060E67BE08BE1C0
:10C0F0009FE00E94C286BE016F5F7F4F8BE19FE091
:10C100000E945C868BE19FE00E942C85CE01019607
:10C110000E94B9A3CE018F5B9F4F0E944E1417CF90
:10C120003F924F925F926F927F928F929F92AF92C7
:10C13000BF92CF92DF92EF92FF920F931F93CF9314
:10C14000DF93CDB7DEB7CE56D1090FB6F894DEBF78
:10C150000FBECDBFDC0114962D913C91232B09F429
:10C1600021C69B01225031092230310508F091C2CD
:10C170003B014C01FC018281803409F4F7C208F0D4
:10C180004AC0843008F085C28091D9068F5F8093C1
:10C19000D906A3016FEFC4010E94235DD40112965A
:10C1A0000C9112970695017013961C9113978AECC7
:10C1B000810F803108F043C064EB75E08D919C9154
:10C1C0000E9405997C010097D1F1FC0180858F7058
:10C1D0008530A9F58091640D181324C08091650DF8
:10C1E000803401F58091660D9091670D5C01990F87
:10C1F000CC08DD0860E0C7010E947A99FC018185C6
:10C200009285A385B485A816B906CA06DB060CF08C
:10C2100065C0512C3EC0823409F4A8C208F439C26A
:10C220008058AFCF1093640D80E48093650D812F0B
:10C230000E949DA69093670D8093660DD7CF212F06
:10C2400030E0F901EA52F34E8491F901E058F34EDF
:10C250001491F901E65DF34EF490FF2009F43BC020
:10C2600081110E94F5A4EF2DF0E0EE0FFF1FE35DBA
:10C27000F84FA591B491EC911E2331E020E009F430
:10C2800030E0832F922F552453940817190609F094
:10C29000C0CFF3E06F16710409F488C0D40114967E
:10C2A000ED91FC91E181EF70E150EC3008F07EC03F
:10C2B000F0E08827E15AFE498F4F0C9429D680611F
:10C2C000FC62B661EC61FC620562FC623962666226
:10C2D0007F62C162E36290E080E0D5CF61E0C70198
:10C2E0000E947A9955245394FC0181859285A385F7
:10C2F000B4858A159B05AC05BD050CF0CACF89CF66
:10C300000E9414A79B01AC0144275527D401149621
:10C31000ED91FC916281738190E080E0AA24AA945F
:10C32000BA2CC12CD12C18EEE12E13E0F12E00E036
:10C3300010E00E94C82A8823C9F1F401008111810C
:10C340006FE875E0C8010E940599892B41F464E902
:10C3500075E0C8010E940599892B09F40EC142E0DD
:10C3600050E063E0C4010E94235D20C00E9414A736
:10C370009B01AC0144275527D4011496ED91FC9103
:10C380006281738190E080E0AA24AA94BA2CC12C27
:10C39000D12C1CE2E12EFF24F39400E010E00E9477
:10C3A000C82A42E050E064E0811184C0D4011496B0
:10C3B000ED91FC91808183FB992790F9951509F403
:10C3C000D2C1982F907E09F439C1982F907E905257
:10C3D0008F71892B808358C10E9414A79B01AC01E7
:10C3E00044275527D4011496ED91FC916281738105
:10C3F00090E080E0AA24AA94BA2CC12CD12C16E992
:10C40000E12EF12C00E010E0CACF0E9414A79B019E
:10C41000AC0144275527D4011496ED91FC9162811B
:10C42000738190E080E0AA24AA94BA2CC12CD12C6C
:10C4300018EEE12E13E0F12E00E010E00E94C82A71
:10C44000882309F4B3CFF401008111816AE975E012
:10C45000C8010E940599892B41F460EA75E0C80182
:10C460000E940599892B09F488C042E050E068E0F9
:10C4700079CF0E9414A79B01AC0144275527D40112
:10C480001496ED91FC916281738190E080E0AA2482
:10C49000AA94BA2CC12CD12C1CE2E12EFF24F394D7
:10C4A00000E010E00E94C82A42E050E069E08823E2
:10C4B00009F47CCFC4010E94235D0E9414A7D4011B
:10C4C0001496ED91FC917383628370CF0E9414A740
:10C4D0009B01AC0144275527D4011496ED91FC91A2
:10C4E0006281738190E080E0AA24AA94BA2CC12CC6
:10C4F000D12C16E9E12EF12C00E010E0D3CF0E9400
:10C5000014A79B01AC0144275527D4011496ED9143
:10C51000FC916281738190E080E0AA24AA94BA2CF5
:10C52000C12CD12C18EEE12E13E0F12E00E010E02A
:10C530000E94C82A882309F439CFF40100811181AF
:10C5400067EA75E0C8010E940599892B39F46DEA04
:10C5500075E0C8010E940599892B21F042E050E066
:10C560006BE000CF69E875E0C8010E94059942E0E0
:10C5700050E066E0892B09F4F5CE42E050E06DE032
:10C58000F1CE0E9414A79B01AC0144275527D4018A
:10C590001496ED91FC916281738190E080E0AA2471
:10C5A000AA94BA2CC12CD12C1CE2E12EFF24F394C6
:10C5B00000E010E00E94C82A882309F4F7CE42E088
:10C5C00050E06CE077CF0E9414A79B01AC01442798
:10C5D0005527D4011496ED91FC916281738190E00E
:10C5E00080E0AA24AA94BA2CC12CD12C16E9E12E01
:10C5F000F12C00E010E0DECF0E9414A79B01AC01FB
:10C6000044275527D4011496ED91FC9162817381E2
:10C6100090E080E0AA24AA94BA2CC12CD12C18E571
:10C62000E12E12E0F12E00E010E00E94C82A8823DB
:10C6300009F4BCCE42E050E060E094CE0E9414A722
:10C64000D4011496ED91FC91159773836283E18177
:10C65000EF70552009F445C0E230F1F050F4EE23BC
:10C66000E9F1D4011496ED91FC91808150FA83F99F
:10C67000B1CEE53089F0A3016AE0E73091F7C4015B
:10C680000E94235D8111EDCF8091D9068150809366
:10C69000D90690E080E088C3F4010081118163E84D
:10C6A00075E0C8010E940599892BA9F46AE975E033
:10C6B000C8010E940599892B71F460EA75E0C801F0
:10C6C0000E940599892B39F46BE675E0C8010E9438
:10C6D0000599892B19F0A30166E0D1CFA30161E090
:10C6E000CECFE150ED3008F0BCCFF0E08827E45821
:10C6F000FC498F4F0C9429D6896331638C638C631A
:10C7000031638F633163B063B063B063B063B063B0
:10C710008C63A30162E0B3CFA30165E0B0CF0D91BC
:10C720001C9163E875E0C8010E940599892BA9F462
:10C730006AE975E0C8010E940599892B71F460EAE5
:10C7400075E0C8010E940599892B39F46BE675E004
:10C75000C8010E940599892B19F0A30167E08FCFCA
:10C76000A30160E08CCF8F71806434CEB3E06B1690
:10C77000710409F48ECF64EB75E0F401808191813E
:10C780000E9405998C01D40113968C919091640DAF
:10C790008913EBC09091650D903409F0E6C080914B
:10C7A000660D9091670D3C010115110509F40DC14D
:10C7B000F80120852F70253009F007C1C8010E94BB
:10C7C0008F99382EF3E0F81708F0DBC063E0C8015A
:10C7D0000E947A99DC0119968D919C913AE0E32EA2
:10C7E000E89E6001E99ED00C1124A396DFAECEAE88
:10C7F000A39762E0C8010E947A99DC0119968D9195
:10C800009C91E89E2001E99E500C11246201052CA8
:10C81000000CEE08FF08AF96CCAEDDAEEEAEFFAE7C
:10C82000AF9761E0C8010E947A995C0160E0C8019D
:10C830000E947A99DC011996CD90DD90ED90FC90E4
:10C840001C97A796CCAEDDAEEEAEFFAEA7979301D8
:10C85000072C000C440B550B2C193D094E095F09A0
:10C86000A396CEACDFACA397B601DD0C880B990B79
:10C87000AF96CCACDDACEEACFFACAF976C197D09DC
:10C880008E099F090E948ED5D50119962D913D9153
:10C890004D915C911C97A796CCACDDACEEACFFAC97
:10C8A000A7972C193D094E095F09A7962CAF3DAFFC
:10C8B0004EAF5FAFA7970E94C0D5AF96ACACBDACF2
:10C8C000CEACDFACAF97A20EB31EC41ED51E45E0A2
:10C8D000E42E3E1409F468C081E090E0A396EEAC2B
:10C8E000FFACA397A701FF0C660B770B4A155B05FE
:10C8F0006C057D050CF461C0B601A5016201052C33
:10C90000000CEE08FF084C155D056E057F050CF464
:10C9100059C06A017B0122E032126BC06301770CBF
:10C92000EE08FF0860E0C8010E947A99FC01818549
:10C930009285A385B485C816D906EA06FB060CF4D1
:10C940004CC261E0C8010E947A99FC018185928500
:10C95000A385B4858C159D05AE05BF050CF099CE59
:10C9600081E090E0A0E0B0E03BC28093640D90E4F1
:10C970009093650D0E949DA69093670D8093660D20
:10C9800012CF8AE0869D5001879DB00C11240B2C9C
:10C99000000CCC08DD08512C412C20E038E2A39695
:10C9A0003FAF2EAFA39798CF64E0C8010E947A9959
:10C9B000DC0119968D919C9191CF66246A9423E0B5
:10C9C000722E9CCF712C612CA6CF2AE0289F60018B
:10C9D000299FD00C11240D2C000CEE08FF08512CBF
:10C9E000412C20E038E2A3963FAF2EAFA39781E021
:10C9F00090E0D4011496ED91FC9162817381A301C2
:10CA0000461B570B57FF03C0519541955109841799
:10CA100095070CF4BFC08081982F929596959770DA
:10CA2000963008F0BAC09F5F9295990F907E8F71F3
:10CA3000892BB2C0F70161857285DB018C91811170
:10CA40005EC2A114B10409F472C0D50118968C918C
:10CA500018978F70843009F06AC019966D917C9197
:10CA6000CE0101960E94AF57CE0101960E94181484
:10CA7000882309F458C06114710409F45FC0E114FB
:10CA8000F10431F0F70180858F70843009F441C0E2
:10CA900025961CAE1DAE1EAE1FAE259729961CAE68
:10CAA0001DAE1EAE1FAE299723961FAD23971F7094
:10CAB00023961FAF239781E022968FAF2297CC2435
:10CAC000C394F12CE12C01E024962FAD24972596F8
:10CAD0003FAD259740E027965FAD279728966FAD2D
:10CAE000289729967FAD2997CE0101960E942A4367
:10CAF0001AC00115110529F0F80180858F70843066
:10CB000019F065E974E0FBC161857285FB018081E4
:10CB100096CF61857285FB018081882321F0CE014B
:10CB200001960E948E9ECE0101960E944E14D40161
:10CB30001496ED91FC9173826282ABCD01151105C3
:10CB400031F0D80118968C918F708430E9F02596D9
:10CB50001CAE1DAE1EAE1FAE259729961CAE1DAE97
:10CB60001EAE1FAE299723961FAD23971F702396E5
:10CB70001FAF239782E022968FAF2297CC24C394D5
:10CB8000F12CE12C02E0A0CFF80161857285DB0178
:10CB90008C91C3CF80818F7180838081803AB8F07F
:10CBA000C201550CAA0BBB0BC816D906EA06FB0638
:10CBB00071F0A396EEADFFADA397CF01FF0FAA0BC7
:10CBC000BB0BC816D906EA06FB0609F062CD66164D
:10CBD000770609F45ECD6D961CAE1DAE1EAE1FAE7F
:10CBE0006D976B968FAD6B978F7080666B968FAFDE
:10CBF0006B976D968CAD9DADAEADBFAD6D976596E7
:10CC00008CAF9DAFAEAFBFAF6597AAE0B0E0A70114
:10CC100096010E94DFD569966CAF7DAF8EAF9FAF56
:10CC200069976CE177E08BE19FE00E94C2864AE061
:10CC300050E0D40113966C918BE19FE00E94308507
:10CC40006AE177E08BE19FE00E94C286CE018F5AB5
:10CC50009F4F0E94C33361E475E0F40180819181AC
:10CC60000E940599B12CA12CD12CC12C6296EFAC5D
:10CC700062976396FFAC639764960FAD6497659671
:10CC80001FAD659766962FAD669767963FAD679720
:10CC900068964FAD689769965FAD69976FEF0E9490
:10CCA0003B58D4010D911C9165E475E0C8010E94C8
:10CCB00005997C016AE475E0C8010E9405998C0120
:10CCC0000097E1F1FC0180858F708430B9F56185B2
:10CCD000728540E450E0CE0101960E94B8DA6FE21E
:10CCE00070E0CE0101960E947FDA892B59F4D801B9
:10CCF00019962D913C9143E050E060E4CE010196FD
:10CD00000E94BE2D00E020E032E040E150E0BE0194
:10CD10006F5B7F4FCE018F5A9F4F0E9413200E945E
:10CD20002099882359F080911A08811107C0BE010B
:10CD30006F5B7F4FCE0101960E94E2A7E114F104E0
:10CD400009F4F5CEF70180858F70843009F0EFCEBD
:10CD500061857285CE0101960E94AF57CE01019682
:10CD60000E941814882309F4DECECC24C394F12C3D
:10CD7000E12C62960FAD629763961FAD6397649640
:10CD80002FAD649765963FAD659766964FAD6697F4
:10CD900067965FAD679768966FAD689769967FAD48
:10CDA0006997A2CE8FEF9FEFC259DF4F0FB6F8946D
:10CDB000DEBF0FBECDBFDF91CF911F910F91FF90CE
:10CDC000EF90DF90CF90BF90AF909F908F907F902B
:10CDD0006F905F904F903F90089580E090E0DC016D
:10CDE000F40124813581F90142815381052E000C23
:10CDF000660B770B84179507A607B70709F449CC8C
:10CE00003C01D4010D911C9165E475E0C8010E94BC
:10CE100005995C016AE475E0C8010E9405996C01FE
:10CE2000A114B10419F4892B09F481CE6EE775E0E1
:10CE3000C8010E9405997C0169E775E0C8010E945C
:10CE400005998C0162E277E08BE19FE00E94C28647
:10CE50004AE050E0F40163818BE19FE00E9430855D
:10CE600060E277E08BE19FE00E94C286B3018BE134
:10CE70009FE00E9487998BE19FE00E942C85C1145E
:10CE8000D10409F4DECDD60118968C9118978F70D5
:10CE9000843009F0D6CD19966D917C9140E450E034
:10CEA000CE0101960E94B8DA0E942099882309F4E5
:10CEB000C8CD80911A088111C4CD6FE270E0CE0117
:10CEC00001960E947FDA892B51F4F6012185328583
:10CED00043E050E060E4CE0101960E94BE2D611453
:10CEE000710409F406CEE114F10439F0D701189663
:10CEF0008C918F70843009F49DCD62E974E0CE018D
:10CF000001960E94E2A79DCD8F929F92AF92BF9211
:10CF1000CF92DF92EF92FF920F931F93CF93DF9305
:10CF200000D000D0CDB7DEB72091F0063091F106E9
:10CF3000232B09F4C5C02091E3062111C1C04C0187
:10CF40008091E3068F5F8093E30680918C088F5F6A
:10CF500080938C080E9414A79B01AC016091DF06AE
:10CF60007091E0068091E1069091E206A12CB12C2F
:10CF700065011BE0E12EF12C00E010E00E94C82AC0
:10CF8000882309F452C0E091F006F091F106068181
:10CF9000178101151105B9F1F80180858F70863070
:10CFA00071F561E475E0C8010E9405990097D1F020
:10CFB000FC0120852F702530A9F4E680F780E1146C
:10CFC000F104E9F0FA82E982B801CE0101960E94EB
:10CFD000CB1AB401CE0101960E949060F701E28065
:10CFE000F380EDCF1A83098370E060E0CE010196F3
:10CFF0000E94CB1AB401CE0101960E949060F80104
:10D0000002811381C6CFF3E08F16910451F00E9484
:10D0100014A76093DF067093E0068093E106909377
:10D02000E2061092640D1092650D83E0881691045B
:10D03000E9F10E9414A79B01AC016091DB0670919D
:10D04000DC068091DD069091DE06A12CB12C6501F5
:10D0500018E8E12E13E1F12E00E010E00E94C82A4A
:10D06000882321F1E091F006F091F1060681178105
:10D070000115110589F0F80180858F70863041F423
:10D080001A83098370E060E0CE0101960E94CB1AFA
:10D09000F80102811381ECCF0E9414A76093DB0694
:10D0A0007093DC068093DD069093DE0680918C08F9
:10D0B000815080938C088091E30681508093E30631
:10D0C00026960FB6F894DEBF0FBECDBFDF91CF918D
:10D0D0001F910F91FF90EF90DF90CF90BF90AF9096
:10D0E0009F908F9008954F925F926F927F92AF9230
:10D0F000BF92CF92DF92EF92FF920F931F93CF9345
:10D10000DF93CDB7DEB76D970FB6F894DEBF0FBED5
:10D11000CDBF67E374E18BE19FE00E94C2868BE1A3
:10D120009FE00E942C850E9414A72B013C01809156
:10D130008C08882351F10E9414A79B01AC01A12CFB
:10D14000B12C650110E1E12E17E2F12E00E010E0B4
:10D15000C301B2010E94C82A811117C00E94808CAD
:10D1600080918E0890918F08059741F080919008EA
:10D1700090919108892B11F00E9486510E944D5583
:10D1800082E090E00E948467D2CF80918C08FF24D7
:10D19000F394882359F064E174E184EF9DE00E94E8
:10D1A000C28684EF9DE00E942C85F12C6EEF73E126
:10D1B0008BE19FE00E94C2868BE19FE00E942C855C
:10D1C0008091F6068F5F8093F606E0919008F091CB
:10D1D0009108309781F1068117810115110559F1E8
:10D1E000D80118968C918F708530B9F7C8010E94CC
:10D1F0008F99882391F3F80160817181CE010196A6
:10D200000E94AF57CE0101960E941814882359F04E
:10D210008A859B85009739F0DC01ED91FC910284B1
:10D22000F385E02D1995CE0101960E944E14F80168
:10D2300002811381D2CF1092F5061092F40666EFA8
:10D2400073E18BE19FE00E94C2868BE19FE00E9428
:10D250002C8564E670E080E090E00E94E2A61092E7
:10D26000170810928D086EED73E18BE19FE00E942C
:10D27000C2860E94EB11AB01BC012AE08BE19FE06A
:10D280000E94E0848091F2069091F3060E94FEA134
:10D290001092F3061092F2061092F1061092F00628
:10D2A0001092910810929008109219081092180884
:10D2B00010928A08109289081092880810928708A4
:10D2C00069ED73E18BE19FE00E94C2860E94EB1141
:10D2D000AB01BC012AE08BE19FE00E94E0848BE17E
:10D2E0009FE00E942C8510928B088091F606815059
:10D2F0008093F6068F2D6D960FB6F894DEBF0FBEA5
:10D30000CDBFDF91CF911F910F91FF90EF90DF90F4
:10D31000CF90BF90AF907F906F905F904F900895A7
:10D3200080911A088F5F80931A08A89583E090E097
:10D330000E9484670E94808C80911A08815080939B
:10D340001A080895CF92DF92EF92FF92CF93DF9366
:10D35000EC018C85883068F40E947C940E9414A7AC
:10D360006B017C018C850E949894811109C088E032
:10D370008C87DF91CF91FF90EF90DF90CF90089551
:10D380000E94906961E070E080E090E00E94E2A677
:10D390000E9414A7AB01BC014C195D096E097F09FD
:10D3A0008D859E85B0E0A0E0481759076A077B0786
:10D3B000C8F28C850E948A94DACFCF92DF92EF92E6
:10D3C000FF921F93CF93DF93EC017B016A018C8561
:10D3D000883048F40E949894882319F08C850E9424
:10D3E0007C9488E08C87F70182819381A481B58148
:10D3F0000097A105B10551F490E080E0DF91CF9155
:10D400001F91FF90EF90DF90CF9008958F3F9F4F37
:10D41000AF4FBF4F89F370E060E081E20E94D39488
:10D42000182F8C87883040F780E591E00E944EA24B
:10D43000A7014E5F5F4F24E030E06CE070E0812F89
:10D440000E94E726B601812F0E94A79464E070E055
:10D45000812F0E94B48F0E9414A76B017C018C85E0
:10D460000E949894873121F18C3111F1882321F2A7
:10D470000E9414A7AB01BC014C195D096E097F091C
:10D480008D859E85B0E0A0E084179507A607B707B5
:10D4900048F00E94906961E070E080E090E00E94B6
:10D4A000E2A6DDCF8C850E948A9488E08C87A4CF89
:10D4B00081E090E0A3CF8F929F92BF92CF92DF92B4
:10D4C000EF92FF920F931F93CF93DF93CDB7DEB709
:10D4D000A3970FB6F894DEBF0FBECDBF8091F206C2
:10D4E0009091F306892B09F44AC280918C0881112E
:10D4F00046C280918C088F5F80938C086DEC7EE033
:10D500008AEE9DE00E94C2868AEE9DE00E942C85F4
:10D510000091F2061091F30668EB75E0C8010E94D5
:10D52000059990939108809390086EEB75E0C8017F
:10D530000E94059990931908809318086FE176E08E
:10D54000C8010E9405999093F1068093F00665EC5E
:10D5500075E0C8010E94059990938A088093890814
:10D560000E94E4311092F5061092F406E0919008C2
:10D57000F0919108309709F4F2C0E680F7800091AD
:10D580009008109191080115110509F4E1C0E1140A
:10D59000F10409F4DDC0D70118968C918F708530A5
:10D5A00091F7C7010E948F99823068F3B701CE01CD
:10D5B00001960E946B23CE0101960E9418148823C5
:10D5C00009F464C08A859B85009769F570E060E086
:10D5D000CE0101960E94B01B8C01912C812C97FFEB
:10D5E00006C011950195110988248394912CCE01D0
:10D5F00001960E94D31CC82ED12C8985853009F450
:10D600004EC0863009F042C0B02E61E0802F0E94EB
:10D610008AA561E0892809F479C0CA94CD2809F067
:10D6200079C060E077C0DC01ED91FC910484F58560
:10D63000E02D1995892B49F08A859B85DC01ED91B8
:10D64000FC910284F385E02D19958A859B85DC0188
:10D65000ED91FC910680F781E02D1995892BB1F0B1
:10D66000CE0101960E94D31C882331F060E071E066
:10D67000CE0101960E94611C8D819E81892B31F023
:10D6800060E072E0CE0101960E94611CD701129603
:10D69000ED90FC90CE0101960E944E1470CFCD28E3
:10D6A00029F462E0CE0101960E94A11C60E071E0C5
:10D6B000CE0101960E94611C8D819E81892B31F0E3
:10D6C00060E072E0CE0101960E94611C61E0802F53
:10D6D0000E948AA560E0802F0E945CA565EC7EE038
:10D6E0008BE19FE00E94C286B8018BE19FE00E941F
:10D6F000879960EC7EE08BE19FE00E94C2866EEB32
:10D700007EE08BE19FE00E94C286C0CFCA94CD2804
:10D7100009F087CFC62ED12C8B2D0E945CA569EB1A
:10D720007EE08BE19FE00E94C286B8018BE19FE022
:10D730000E94879967EB7EE08BE19FE00E94C286A2
:10D74000B6018BE19FE00E94879965EB7EE0D9CF1F
:10D75000F801868197819093F5068093F4068BE11A
:10D760009FE00E942C85E091F006F091F106309741
:10D7700009F48AC080918C088F5F80938C080681A1
:10D7800017810115110509F47AC0D80118968C91FA
:10D790008F70863009F069C01F8F0E8F70E060E0D7
:10D7A000CE014E960E94CB1A8AA19BA1892B09F427
:10D7B0005CC08091F2069091F306892B09F455C064
:10D7C000EE8CFF8CF70180858F70863099F561E4CF
:10D7D00075E0C7010E9405990097F1F0DC011896E9
:10D7E0002C9118972F702530B9F41696CD90DC90B7
:10D7F000C114D104F9F0DA82C982B701CE010196D1
:10D800000E94CB1AED81FE81108211821282138256
:10D81000F601C280D380ECCFFA82E98270E060E04A
:10D82000CE0101960E94CB1A62E070E0CE01019613
:10D830000E949060EAA1FBA11082118212821382E1
:10D8400088A1843068F462E0823008F060E089A149
:10D850000E948AA5EAA1FBA18181807F818305C006
:10D86000803441F060E0823431F0D80112960D919D
:10D870001C9187CF62E089A10E948AA5F6CF809192
:10D880008C08815080938C0868EA7EE08AEE9DE0E7
:10D890000E94C28660EA7EE08AEE9DE00E94C28617
:10D8A00081E02091900830919108232B09F480E0C9
:10D8B0000E945C1867E97EE08AEE9DE00E94C286C5
:10D8C00081E02091F0063091F106232B09F480E0ED
:10D8D0000E945C1860E97EE08AEE9DE00E94C286AC
:10D8E00081E02091890830918A08232B09F480E097
:10D8F0000E945C1867E87EE08AEE9DE00E94C28686
:10D90000809117080E945C188AEE9DE00E942C8589
:10D9100062E87EE08AEE9DE00E94C2860E94EB11E2
:10D92000AB01BC012AE08AEE9DE00E94E0848AEE11
:10D930009DE00E942C8581E080938D0888EB9DE01E
:10D940000E945117882351F088EB9DE00E94A26944
:10D9500084E090E090938F0880938E0880918E08E9
:10D9600090918F08079731F484E090E090938F08AE
:10D9700080938E0880918C08815080938C08A396A8
:10D980000FB6F894DEBF0FBECDBFDF91CF911F91D0
:10D990000F91FF90EF90DF90CF90BF909F908F906E
:10D9A0000895EF92FF920F931F93CF93DF9300D0D0
:10D9B0001F92CDB7DEB78C017B01FB0184858830D7
:10D9C000A8F082E394E0F8019183808312821382AD
:10D9D00014821582C8010F900F900F900F90DF9165
:10D9E000CF911F910F91FF90EF90089580E591E006
:10D9F0000E944EA224E030E0AE014F5F5F4F6CE02A
:10DA000070E0F70184850E941628BE016F5F7F4F8A
:10DA1000C8010E94F886DECFEF92FF920F931F930A
:10DA2000CF93DF93CDB7DEB764970FB6F894DEBF20
:10DA30000FBECDBF0D871E872F87388B498B5A8B22
:10DA40006B8B7C8B64E276E18BE19FE00E94C28667
:10DA5000CE010D960E94C3339E85892F8F70082FAB
:10DA600010E02D85222309F4A8C00115110509F441
:10DA700074C0813009F471C08130A0F18230C1F1ED
:10DA80008E3009F081C092959F7069897A899C30A7
:10DA900011F070E060E0CE0101960E9443846BE3D8
:10DAA00076E0C7010E948ADA892B09F03FC0BE01E7
:10DAB0006F5F7F4FCE0107960E943A84CE01079692
:10DAC0000E9402A4BC018CE19CE00E94B486CE01BD
:10DAD00007960E94078401E010E0CE0101960E94A3
:10DAE000078416C063E176E18BE19FE00E94C28665
:10DAF0006FEF75E18BE19FE00E94C2868BE19FE0B2
:10DB00000E942C858E85807F01E010E009F400E002
:10DB1000C80164960FB6F894DEBF0FBECDBFDF918B
:10DB2000CF911F910F91FF90EF9008956BE476E0F5
:10DB3000C7010E948ADA00E0892B71F6BE016F5F8F
:10DB40007F4FCE0107960E943A84CE0107960E942D
:10DB500002A4BC018FEF9AE0B8CF213031F122301E
:10DB600049F162EF75E18BE19FE00E94C2864AE0D5
:10DB700050E06D858BE19FE00E9430858BE19FE056
:10DB80000E942C8501E010E062EE75E18BE19FE0E0
:10DB90000E94C286B8018BE19FE00E9487998BE1C9
:10DBA0009FE00E942C8500E003C02093290201E041
:10DBB00010E0AECF10922902FACF813009F05CCF8D
:10DBC000D0CFAF92BF92CF92DF92EF92FF920F939E
:10DBD0001F93CF93DF93CDB7DEB7CA59D1090FB6E4
:10DBE000F894DEBF0FBECDBF8E010F5B1F4FD80173
:10DBF0001D921C92FE01ED5BFF4F8EE1DF011D9235
:10DC00008A95E9F78091C70D9091C80D892B09F489
:10DC10009FC10E94C899882309F49AC1A091C70D99
:10DC2000B091C80D52961C921E92519754961C9218
:10DC30001E92539784E890E01D969C938E931C97B8
:10DC40001E961C921E9780E090E350969C938E93B4
:10DC50001F97ED91FC9111970088F189E02D60E20A
:10DC600070E0CD0119954FE150E0B8018091C70DEA
:10DC70009091C80D0E941F9A7C018091C70D9091D0
:10DC8000C80DDC01ED91FC910488F589E02D199512
:10DC9000E114F10409F45CC1F801EE0DFF1D1082DE
:10DCA0008091D40D1F928F938091D30D1F928F93EB
:10DCB0008091D20D1F928F938091D10D1F928F93DF
:10DCC0008091D00D1F928F938091CF0D1F928F93D3
:10DCD0008AEC95E09F938F931F9280E48F93FE01CF
:10DCE00031966F01FF93EF930E94D2DA60E171E108
:10DCF0008AEE9DE00E94C286B8018AEE9DE00E94F5
:10DD00005C86B6018AEE9DE00E945C868AEE9DE00C
:10DD10000E942C857E01F1E6EF0EF11CD7011396CF
:10DD20001C921E92129788EE93E0A0E0B0E0F701FB
:10DD300084839583A683B78388E0848788EE93E005
:10DD4000968785878CEB93E091838083108A178672
:10DD5000128B018B148A138A80E590E0968B858B59
:10DD6000118E6FE370E18BE19FE00E94C28669EC47
:10DD70007DE0CE0185589F4F0E943A84BE016558D0
:10DD80007F4F8BE19FE00E94B4868BE19FE00E9471
:10DD90002C85CE0185589F4F0E94078469EF75E05E
:10DDA000CE0183579F4F0E94438469EF75E0CE01F7
:10DDB00085589F4F0E944384BE0165587F4FCE0116
:10DDC0008B579F4F0E943A8469EC7DE0CE018B57C0
:10DDD0009F4F0E94A383BE0163577F4F0E94A3837E
:10DDE000BC01CE018D569F4F0E943A84CE018B57C5
:10DDF0009F4F0E940784CE0185589F4F0E94078441
:10DE0000CE0183579F4F0E9407848BEF95E0CB573D
:10DE1000DF4F99838883C558D040C757DF4F198299
:10DE20001882C958D040C557DF4F19821882CB5885
:10DE3000D040CD56DF4F88819981C359D040C95712
:10DE4000DF4F99838883C758D0406AE071E18BE146
:10DE50009FE00E94C2860E94EB11AB01BC012AE048
:10DE60008BE19FE00E94E0848BE19FE00E942C8583
:10DE700064E670E080E090E00E94E2A683E298E72A
:10DE8000D70150969C938E931F9767E375E88EEFAA
:10DE90009EE80E9466CC8C010FB6F894DEBF0FBEE0
:10DEA000CDBF892BA1F183E090E00E9442C8D80148
:10DEB0001D969C938E931C97FC01F182E082128246
:10DEC000C7010E945117882319F0C7010E94A26957
:10DED000D70153966D917C9154975596AD90BC9017
:10DEE0006115710509F44BC0CE0185589F4F0E9402
:10DEF000F886A501BE0165587F4FC7010E94DD6904
:10DF0000181619060CF489C1C8010E94D78E61EA5F
:10DF100070E18BE19FE00E94C286EE24EA94FE2C21
:10DF2000CE018D569F4F0E940784C701C656DF4F12
:10DF30000FB6F894DEBF0FBECDBFDF91CF911F911A
:10DF40000F91FF90EF90DF90CF90BF90AF9008952A
:10DF500040E250E062E471E1C8010E94B5CB64E2A6
:10DF600071E18AEE9DE00E94C286B8018AEE9DE0D2
:10DF70000E945C868AEE9DE00E942C8591CEF7017E
:10DF800061897289A501C7010E947317B9CF8AE917
:10DF900090E19F938F931F930F930E94EDCCD70135
:10DFA00058961C921E925797D8011C96ED91FC91A1
:10DFB000A080B1800F900F900F900F9093E3C92E27
:10DFC000D12CD501ED91FC910084F185E02DC501A6
:10DFD000199541975CF4B1E0CB1AD10839F064E1AE
:10DFE00070E080E090E00E94E2A6EBCF6E01E9E9EC
:10DFF000CE0ED11CDF92CF928AE490E19F938F9353
:10E000001F930F930E940ACD0F900F900F900F90C7
:10E010000F900F900197D1F4D6018D919C91F7014B
:10E02000908F878B6DE576E0CE0183579F4F0E94DE
:10E03000438480E0C12CFAE0CF1272C08A3009F02C
:10E0400073C0CE0183579F4F0E940784D701579614
:10E05000ED90FC90B8ECEB16F10409F0BCC06EEF4B
:10E0600070E18AEE9DE00E94C28664EF71E080E07C
:10E0700090E00E94E2A6EF961FAE1EAEEF97C15849
:10E08000DF4F19821882CF57D0408FEF9FEFCF57C5
:10E09000DF4F99838883C158D0408CE093E0ED96A0
:10E0A0009FAF8EAFED97CD57DF4F19830883C358CD
:10E0B000D040F8948091F2069091F306892B11F0EC
:10E0C0000E947368CE0185589F4F0E9430A29093A2
:10E0D000F3068093F2067894C8010E94D78E80914F
:10E0E000F2069091F306892B09F063C06DE576E0A6
:10E0F000CE0183579F4F0E944384CE0183579F4F89
:10E100000E9442ADCE0183579F4F0E94078467EE65
:10E1100070E184EF9DE00E94C286F12CE12C00CFDB
:10E120009DE0C91201C0C82EC8010E94B1CCD82EF2
:10E13000D7011F96AD90BC90A114B10499F1BAE03B
:10E140008B1779F0EDE08E1761F0FFEF8F1749F034
:10E15000682FCE0183579F4F0E94F9828C2DCD2CC2
:10E160006ACFCF56DF4F88819981C159D040892B22
:10E1700091F0BE0163577F4FCE0185589F4F0E949B
:10E180003A84CE0185589F4FF5011995CE018558E7
:10E190009F4F0E9407846DE576E0CE0183579F4F25
:10E1A0000E94D783FFEFDF12D9CFC8010E94D78E1C
:10E1B00048CF0E945B6A80918D08882329F00E94D5
:10E1C000BB9C67FF0E94471B60EE70E18AEE9DE0FA
:10E1D0000E94C286A5CEE0E3EE16E1E0FE0651F411
:10E1E0006CEC70E18AEE9DE00E94C286C8010E943C
:10E1F000D78E96CE64EB70E184EF9DE00E94C286DC
:10E20000C8010E94D78EB70184EF9DE00E948799D4
:10E2100084EF9DE00E942C8583CED7015196BC905F
:10E2200051975296AC90DF92CF928DE990E19F93F7
:10E230008F931F930F930E94EDCCDF92CF9288E9CA
:10E2400090E19F938F931F930F930E94EDCCD80181
:10E250001C96ED91FC9181E08283DF92CF9285E95B
:10E2600090E19F938F931F930F930E94EDCCD80161
:10E270001C96ED91FC911282AF92BF928FE590E1D6
:10E280009F938F931F930F930E94EDCC0FB6F8943A
:10E29000DEBF0FBECDBFB12C86E5C82E80E1D82EE3
:10E2A0008B2D94E08902F0011124A5E8B0E0AC0FB9
:10E2B000BD1FEA0FFB1F80819181009709F467CE93
:10E2C0002281338121153105C1F33F932F939F9311
:10E2D0008F93DF92CF921F930F930E94EDCCB39454
:10E2E0000FB6F894DEBF0FBECDBFDACF0F931F93EA
:10E2F000CF93DF93EB0102970CF49DC00A811B8141
:10E3000061E370E1C8010E9460CB892B51F481E088
:10E310000E947E9D88EC90E0DF91CF911F910F913C
:10E3200008956DE270E1C8010E9460CB892B11F461
:10E3300080E0EECF6DE070E18AEE9DE00E94C28643
:10E340000E94BB9C63FB662760F981E0682770E050
:10E350008AEE9DE00E9487998AEE9DE00E942C85BE
:10E360008091C70D9091C80D892B09F454C00A8182
:10E370001B810E94C899882309F44DC0F8010190BF
:10E380000020E9F73197E01BF10BB09708F043C08C
:10E39000A091C70DB091C80D52961C921E92519734
:10E3A00054961C921E92539784E890E01D969C937D
:10E3B0008E931C971E961C921E9780E090E35096B9
:10E3C0009C938E931F97ED91FC9111970088F18992
:10E3D000E02D60E270E0CD011995B8018091C70D84
:10E3E0009091C80D0E945C868091C70D9091C80DD8
:10E3F000DC01ED91FC910190F081E02D60E0199538
:10E400008091C70D9091C80DDC01ED91FC910488BD
:10E41000F589E02D19956A817B818AEE9DE00E9445
:10E420005C8666E070E18AEE9DE00E94C2868AEE1C
:10E430009DE00E942C8580918E0890918F08029714
:10E440007CF10E94E16D883C910539F424E030E0D4
:10E4500030938F0820938E085FCF8F3F9807C9F4C1
:10E460006BEE7FE08BE19FE00E94C2868BE19FE034
:10E470000E942C8510928B0883E090E090938F0887
:10E4800080938E0888EB9DE00E94A26989EC90E061
:10E4900043CF20918D082111D9CF2FE030E0D8CF84
:10E4A0006EED7FE084EF9DE00E94C28684EF9DE0E8
:10E4B0000E942C8584EF91E02FCFCF93DF93CDB7CF
:10E4C000DEB72E970FB6F894DEBF0FBECDBF80919A
:10E4D0008C0881116BC06AE17FE08AEE9DE00E94AA
:10E4E000C2868AEE9DE00E942C851092E70D109264
:10E4F000E60D80E090E19093E20D8093E10D84E8D9
:10E5000090E09093E90D8093E80D81E08093E30D16
:10E5100080E090E29093E50D8093E40D85ED9DE021
:10E520000E9439268B37910509F0C4C01C821B82DA
:10E5300082E293E09A83898385ED9DE09E838D83BB
:10E540008FEF9FEF98878F838091F2069091F3066B
:10E55000892B11F00E947368CE0101960E9430A2AF
:10E560009093F3068093F20685ED9DE00E9465147A
:10E570008091F2069091F306892BD9F46EE07FE04A
:10E5800084EF9DE00E94C28684EF9DE00E942C856E
:10E590006DE576E0CE0109960E944384CE0109968E
:10E5A0000E9442ADCE0109960E94078490E080E06F
:10E5B00014C06BEF7EE08AEE9DE00E94C2868AEE78
:10E5C0009DE00E942C850E945B6A8091C70D90910E
:10E5D000C80D892B59F481E090E02E960FB6F8947F
:10E5E000DEBF0FBECDBFDF91CF9108950E94C899C5
:10E5F000882389F3A091C70DB091C80D52961C9243
:10E600001E92519754961C921E92539784E890E064
:10E610001D969C938E931C971E961C921E9780E0CD
:10E6200090E350969C938E931F97ED91FC911197D8
:10E630000088F189E02D60E670E0CD0119956091C8
:10E64000C70D7091C80D40E0CE0109960E948684E6
:10E65000BE01675F7F4F89EC9DE00E940D83CE0174
:10E6600009960E9407848091C70D9091C80DDC0126
:10E67000ED91FC910488F589E02D19956DED7EE012
:10E680008BE19FE00E94C28669EC7DE0CE01099695
:10E690000E943A84BE01675F7F4F8BE19FE00E943A
:10E6A000B4868BE19FE00E942C85CE0109960E94E2
:10E6B000078491CF85ED9DE00E947E14892BA1F007
:10E6C00085ED9DE00E94A8146DE576E0CE010196EF
:10E6D0000E944384CE0101960E9442ADCE01019674
:10E6E0000E9407840E94B6AC85ED9DE00E946514EF
:10E6F0006AEE7EE08AEE9DE00E94C2868AEE9DE090
:10E700000E942C8553CF0E945D72892B49F486EFBD
:10E710009FEF90938F0880938E0884EF91E0089587
:10E7200088EC90E00895BF92CF92DF92EF92FF9233
:10E730000F931F93CF93DF9300D000D0CDB7DEB7F8
:10E740008C016B01FB0184819581892BD9F1E080DB
:10E75000F1806FE370E0C7010E947FDA009791F1CA
:10E760009C012E193F09790137FD2CC06DE576E03B
:10E77000CE0101960E944384F60184819581009721
:10E78000B9F08E159F0508F47C01F6016081718156
:10E79000FB01EE0DFF1DB0801082CE0101960E949C
:10E7A000E183F60180819181E80EF91EF701B082C4
:10E7B000BE016F5F7F4FC6010E940D83CE0101969F
:10E7C0000E94078469E076E0C6010E94888288235F
:10E7D00019F1F801128A118A80E090E19587848707
:10E7E00084E890E0948B838B81E0868780E090E2E0
:10E7F000908B878781E090E026960FB6F894DEBF75
:10E800000FBECDBFDF91CF911F910F91FF90EF9081
:10E81000DF90CF90BF90089566E176E0C6010E9438
:10E820008882882369F0F801128A118A148A138A6F
:10E8300084E890E095878487168680E090E3D8CFBF
:10E8400090E080E0D9CFDF92EF92FF920F931F9379
:10E85000CF93DF9300D000D0CDB7DEB78C017B0122
:10E8600063EC75E1CE0101960E940C84BE016F5FDE
:10E870007F4FC7010E949D82D82ECE0101960E9433
:10E880000784DD2019F1D8011296ED91FC911397C0
:10E890000190F081E02D60817181ED91FC91028801
:10E8A000F389E02D22E236E04BEA55E0C8011995E4
:10E8B00026960FB6F894DEBF0FBECDBFDF91CF9185
:10E8C0001F910F91FF90EF90DF90089568EA75E136
:10E8D000CE0101960E940C84BE016F5F7F4FC7017D
:10E8E0000E949D82D82ECE0101960E940784DD20D1
:10E8F000A1F0D8011296ED91FC9113970190F0814F
:10E90000E02D60817181ED91FC910288F389E02D09
:10E9100022E236E04EE955E0C9CF6DE875E1CE015F
:10E9200001960E940C84BE016F5F7F4FC7010E9459
:10E930009D82F82ECE0101960E940784FF2009F4E3
:10E94000B7CFD8011296ED91FC9113970190F08109
:10E95000E02D60817181ED91FC910288F389E02DB9
:10E9600022E236E044E856E0A1CF6F927F928F9288
:10E970009F92AF92BF92CF92DF92EF92FF920F934E
:10E980001F93CF93DF93CDB7DEB72C970FB6F894D4
:10E99000DEBF0FBECDBF4C018CE19CE00E94797CB4
:10E9A000892B39F180E00E94FE176093BB077093BA
:10E9B000BC078093BD079093BE078CE19CE00E944A
:10E9C000577C682E8DE290E09A83898369824FE3B9
:10E9D00050E0BE016F5F7F4F81E397E00E949ADABB
:10E9E0008091B9079091BA0701969093BA078093E6
:10E9F000B9078FEF9AE00E94797C892B39F180E08A
:10EA00000E94FE176093B5077093B6078093B7070F
:10EA10009093B8078FEF9AE00E94577C782E8DE292
:10EA200090E09A83898379824FE350E0BE016F5F63
:10EA30007F4F83E797E00E949ADA8091B307909125
:10EA4000B40701969093B4078093B3078091BB07F6
:10EA50009091BC07A091BD07B091BE07892B8A2B6E
:10EA60008B2B09F0C7C08AE26812DEC01092BB0788
:10EA70001092BC071092BD071092BE071092BA0701
:10EA80001092B90761E377E0CE0107960E944384B4
:10EA900010923107CE0107960E949B818B859C8541
:10EAA000892B09F4DEC169E276E0CE0101960E946D
:10EAB0004384BE016F5F7F4FCE0107960E946D8237
:10EAC000182FCE0101960E940784112321F0809116
:10EAD00029028823A1F0BE01695F7F4FCE01019614
:10EAE0000E943A84CE0101960E9402A4BC018FEFDD
:10EAF0009AE00E94B486CE0101960E940784BE016E
:10EB0000695F7F4FCE0101960E943A84BE016F5F1C
:10EB10007F4FC4010E942374CE0101960E94078496
:10EB200062E376E0CE0101960E944384BE016F5FEE
:10EB30007F4FCE0107960E946D82182FCE0101965D
:10EB40000E940784112309F44FC1BE01695F7F4F02
:10EB500084E59FE00E949D82811183C1BE01695FAF
:10EB60007F4F84E59FE00E94F0834F815885D40158
:10EB70001296ED91FC9113970190F081E02D608148
:10EB80007181ED91FC910288F389E02D28E336E054
:10EB9000C40119958091710790917207892B09F42E
:10EBA00060C16EED75E18BE19FE00E94C28610E0CE
:10EBB00000E0F0E1EF2EF12CB801CE0107960E94A3
:10EBC0005B82FC018081882309F447C18B859C8589
:10EBD0000817190708F041C18091710790917207D9
:10EBE0008130910509F442C1029709F46AC10F5FAF
:10EBF0001F4FE2CF0E9414A79B01AC016091BB079D
:10EC00007091BC078091BD079091BE07A12CB12CDB
:10EC100065011AE0E12EF12C00E010E00E94C82A04
:10EC2000882309F420CF22CFADE06A1609F41ECF65
:10EC30008091B9079091BA078034910508F016CFFA
:10EC40008091B5079091B607A091B707B091B8072A
:10EC5000892B8A2B8B2B09F040C1BAE27B1257C15A
:10EC60001092B5071092B6071092B7071092B80726
:10EC70001092B4071092B30763E777E0CE010796CE
:10EC80000E94438410927307CE0107960E949B81D5
:10EC90008B859C85892B09F49AC169E276E0CE01C7
:10ECA00001960E944384BE016F5F7F4FCE0107969D
:10ECB0000E946D82182FCE0101960E9407841123B5
:10ECC00021F0809129028823A1F0BE01695F7F4F66
:10ECD000CE0101960E943A84CE0101960E9402A4C0
:10ECE000BC018CE19CE00E94B486CE0101960E949A
:10ECF0000784BE01695F7F4FCE0101960E943A846E
:10ED0000BE016F5F7F4FC4010E942374CE01019644
:10ED10000E94078462E376E0CE0101960E9443845C
:10ED2000BE016F5F7F4FCE0107960E946D82182F44
:10ED3000CE0101960E940784112309F40BC1BE0184
:10ED4000695F7F4F80E69FE00E949D8281113FC1F5
:10ED5000BE01695F7F4F80E69FE00E94F0834F8194
:10ED60005885D4011296ED91FC9113970190F08192
:10ED7000E02D60817181ED91FC910288F389E02D95
:10ED800028E436E0C40119958091710790917207CB
:10ED9000892B09F41CC160EE75E18BE19FE00E94B4
:10EDA000C286912C812C00E110E0B401CE010796BF
:10EDB0000E945B82FC018081882309F404C18B8559
:10EDC0009C858816990608F0FEC080917107909185
:10EDD00072078130910509F4FFC0029709F427C139
:10EDE000BFEF8B1A9B0AE1CF6DE376E0CE0101966F
:10EDF0000E944384BE016F5F7F4FCE0107960E9441
:10EE00006D82182FCE0101960E940784112309F408
:10EE1000C1CEBE01695F7F4F8AE59FE00E949D825F
:10EE200081111FC0BE01695F7F4F8AE59FE00E948C
:10EE3000F0834F815885D4011296ED91FC91139780
:10EE40000190F081E02D60817181ED91FC9102884B
:10EE5000F389E02D23E436E09BCE8BE19FE00E9416
:10EE60002C85CE0107960E940784EACEB801CE0118
:10EE700007960E945B82DC018C916DE576E0803123
:10EE800014F469E874E08BE19FE00E945C86B801AD
:10EE9000CE0107960E945B82FC018081082E000C47
:10EEA000990BAA0BBB0B89839A83AB83BC83FE822D
:10EEB000ED82BE016F5F7F4F8BE19FE00E94BB1A26
:10EEC00096CEB801CE0107960E945B82DC016C9160
:10EED0008BE19FE00E94CB858ACE0E9414A79B0104
:10EEE000AC016091B5077091B6078091B70790911A
:10EEF000B807A12CB12C65011AE0E12EF12C00E03D
:10EF000010E00E94C82A882309F4A7CEA9CEEDE01C
:10EF10007E1609F4A5CE8091B3079091B407803492
:10EF2000910508F09DCE81E090E02C960FB6F89404
:10EF3000DEBF0FBECDBFDF91CF911F910F91FF902C
:10EF4000EF90DF90CF90BF90AF909F908F907F9089
:10EF50006F9008956DE376E0CE0101960E944384A0
:10EF6000BE016F5F7F4FCE0107960E946D82182F02
:10EF7000CE0101960E940784112309F405CFBE013A
:10EF8000695F7F4F86E69FE00E949D8281111FC0CE
:10EF9000BE01695F7F4F86E69FE00E94F0834F814C
:10EFA0005885D4011296ED91FC9113970190F08150
:10EFB000E02D60817181ED91FC910288F389E02D53
:10EFC0002DE436E0DFCE8BE19FE00E942C85CE0160
:10EFD00007960E940784A7CFB401CE0107960E942E
:10EFE0005B82DC018C916DE576E0803114F469E898
:10EFF00074E08BE19FE00E945C86B401CE0107962D
:10F000000E945B82FC018081082E000C990BAA0BE8
:10F01000BB0B89839A83AB83BC831E830D83BE01A4
:10F020006F5F7F4F8BE19FE00E94BB1AD9CEB40186
:10F03000CE0107960E945B82DC016C918BE19FE020
:10F040000E94CB85CDCEFF920F931F93CF93DF937A
:10F0500000D000D0CDB7DEB78C01BC01CE01019647
:10F060000E943A84BE016F5F7F4F8BE19FE00E9458
:10F07000B4868BE19FE00E942C85CE0101960E9410
:10F08000078468E370E1CE0101960E940C84BE0102
:10F090006F5F7F4FC8010E946D82F82ECE010196EE
:10F0A0000E940784FF2069F0B801CE0101960E94FA
:10F0B0003A84CE0101960E9442ADCE0101960E9493
:10F0C000078426960FB6F894DEBF0FBECDBFDF9142
:10F0D000CF911F910F91FF9008955F926F927F9251
:10F0E0008F929F92AF92BF92CF92DF92EF92FF9258
:10F0F0000F931F93CF93DF93CDB7DEB7CF56D109D0
:10F100000FB6F894DEBF0FBECDBF4C018B01F42EBD
:10F110004AE050E06F2D8BE19FE00E9430856EE564
:10F120007BE08BE19FE00E94C286B801CE01019690
:10F130005C010E943A84B5018BE19FE00E94B48695
:10F140008BE19FE00E942C85C5010E94078492E01C
:10F15000F9126BC26CE57BE0C5010E940C84B5011D
:10F16000C8010E949D82F82EC5010E940784FF20DD
:10F1700009F4D0C220E04DE251E0B40186E99DE0FF
:10F180000E94D18BE0908708F090880865E57BE0CD
:10F19000CE0186599F4F0E940C846EE47BE0CE0125
:10F1A0008C599F4F0E940C84CE01885A9F4F0E9419
:10F1B00065296E961FAD6E976D960FAD6D976C9627
:10F1C000DFAC6C976B96CFAC6B976DE576E0CE01BC
:10F1D00081960E944384BE016F5D7F4FC5010E94EE
:10F1E0003A846C2DC5010E94588362E576E00E9446
:10F1F00089836D2D0E94588362E576E00E948983A1
:10F20000602F0E94588362E576E00E948983612F17
:10F210000E945883BC01CE01825A9F4F0E943A84BB
:10F22000C5010E940784CE0181960E94078469E48B
:10F230007BE0CE018E5A9F4F0E940C846DE576E0F4
:10F24000CE01845B9F4F0E94438407EC1DE0D801F0
:10F2500018966C9170E084E0759567958A95E1F752
:10F26000C5010E949C994D815E8169817A81CE01A0
:10F27000845B9F4F0E94CD82C5010E940784F801E4
:10F2800060856F7070E0C5010E949C994D815E8120
:10F2900069817A81CE01845B9F4F0E94CD82C50136
:10F2A0000E9407840F5F1F4FFDE00D3C1F0779F69A
:10F2B00063E47BE0CE018A5B9F4F0E940C8462E294
:10F2C0007BE0CE0181960E940C84BE016F5D7F4F72
:10F2D000CE01CE960E943A84BE016A5B7F4FCE017A
:10F2E000CE960E94A383BE01645B7F4F0E94A383DE
:10F2F000BE016E5A7F4F0E94A383BE01625A7F4FA8
:10F300000E94A383BE016C597F4F0E94A3838C018E
:10F310004AE0B50180E590E00E94FACBF50101904A
:10F320000020E9F73197AF014A195B09B501C8011F
:10F330000E94CD82811103C0C8010E944683BE0194
:10F3400066597F4FC8010E94A383B7010E94898339
:10F35000BC01C4010E94B486C4010E942C85CE0168
:10F36000CE960E940784CE0181960E940784CE012A
:10F370008A5B9F4F0E940784CE01845B9F4F0E944F
:10F380000784CE018E5A9F4F0E940784CE01825A75
:10F390009F4F0E940784CE018C599F4F0E94078483
:10F3A000CE0186599F4F0E940784C4010E942C857C
:10F3B00064E670E080E090E00E94E2A6D401ED9166
:10F3C000FC910488F589E02DC401199501E010E055
:10F3D00088C028966EAD7FAD2897CE0181960E9499
:10F3E0008E9E892B09F450C122961CAE1DAE1EAE16
:10F3F0001FAE229726961CAE1DAE1EAE1FAE2697E0
:10F400008FAD8F708FAF40E053E0BE016F5D7F4FD7
:10F41000CE01CE960E94333500E020E033E040E29A
:10F4200050E0B501CE01CE960E941320BC01C6016A
:10F430000E94E18308EC10E129C1EE2009F4F3C039
:10F4400046E050E070E060E0C8010E94F881D80119
:10F450006D917C91CE0181960E94AF57CE0181962D
:10F460000E94181400E911E08823B9F189A58730BA
:10F4700061F4CE0181960E94125361E0892B09F458
:10F4800062E0CE0181960E94A11C22961CAE1DAEA8
:10F490001EAE1FAE229726961CAE1DAE1EAE1FAE30
:10F4A00026978FAD8F708FAF40E053E0BE016F5D48
:10F4B0007F4FCE01CE960E94333500E020E033E04E
:10F4C00040E250E0B501CE01CE960E941320BC016F
:10F4D000C6010E94E18308EC10E1CE0181960E94F2
:10F4E0004E14C801C159DF4F0FB6F894DEBF0FBEEE
:10F4F000CDBFDF91CF911F910F91FF90EF90DF90E3
:10F50000CF90BF90AF909F908F907F906F905F90C3
:10F510000895F801608171810E9405997C01892B11
:10F5200009F040C104E911E0DCCFEE2009F47BC012
:10F5300049E050E070E060E0C8010E94F8814AE0D4
:10F54000B401C5010E94868441E050E069E474E0A2
:10F55000C8010E94CD824D815E8169817A81C80196
:10F560000E94CD826EEF7AE08BE19FE00E94C2861E
:10F57000B801CE0181960E943A84BE016F5D7F4F33
:10F580008BE19FE00E94B4868BE19FE00E942C8576
:10F59000CE0181960E94078466EF7AE0CE018196C3
:10F5A0000E940C84F801848195812DA13EA18217CF
:10F5B0009307E1F4892BA1F1E080F18069A07AA0A2
:10F5C000D7018D917D01882359F1082E000C990BEC
:10F5D0000E940FDA6C01F30181913F01082E000CAB
:10F5E000990B0E940FDAC816D90651F3CE01819605
:10F5F0000E940784552041F021E048EC50E0B4011E
:10F6000086E99DE00E94D18BD8018D919C910E944A
:10F61000FF8B009711F484E991E08C01C5013DC096
:10F6200055245394E3CF01E97ECFB1E0FB1270C0C3
:10F630006BE17BE0C5010E940C84B501C8010E940A
:10F640006D82582EC5010E940784552049F1EE2095
:10F6500051F346E050E070E060E0C8010E94F8819C
:10F660004AE0B401CE018A5B9F4F0E948684F80174
:10F6700060817181CE0181960E94AF57CE01819643
:10F680000E9418148111A5CE00E911E0CE018196E7
:10F690000E944E14CE018A5B9F4F0E94078421CFA7
:10F6A00064E07BE0C5010E940C84B501C8010E94A2
:10F6B0006D82F82EC5010E940784F11036CF69EEE5
:10F6C0007AE0C5010E940C84B501C8010E946D82D8
:10F6D000182FC5010E94078400E0112309F401CF0F
:10F6E00080E00E947E9D61EC7AE08AEE9DE00E94BF
:10F6F000C2868AEE9DE00E942C856DE576E0C5010C
:10F700000E944384C5010E9442ADC5010E94078446
:10F7100000E05DCE64E17BE0C5010E940C84B50190
:10F72000C8010E946D82F82EC5010E940784F11065
:10F7300084CE6EE07BE0C5010E940C84B501C80157
:10F740000E946D82F82EC5010E940784FF2001F3FC
:10F75000EE2009F468CF45E050E070E060E0C801B9
:10F760000E94F88162E576E0C8010E9488828823C1
:10F7700039F0E0909008F0909108E114F10491F4D0
:10F780006DE576E0C8010E948882811107C08091F2
:10F79000900890919108009709F0BBCEE090F20696
:10F7A000F090F30620E048EC50E2B40186E99DE0D9
:10F7B0000E94D18BC4010E942C851C821B8282E294
:10F7C00093E09A8389839E828D828FEF9FEF988743
:10F7D0008F83B701C5010E94C68CEACD0895FC0154
:10F7E000248135816217730748F4808191810097E5
:10F7F00029F0860F971FFC018081089580E008950D
:10F800000895AF92BF92CF92DF92EF92FF920F9343
:10F810001F93CF93DF936C017B018B01040F151FA6
:10F82000EB015E01AE18BF08C017D10759F069910E
:10F83000D601ED91FC910190F081E02DC601199562
:10F84000892B79F7C501DF91CF911F910F91FF901F
:10F85000EF90DF90CF90BF90AF900895FC01A0890A
:10F86000B1898C91A689B78982FD0FC09C91818D49
:10F870008F5F8F77228D821749F0A18DAE0FBF2F3A
:10F88000B11D5D969C93818F08958C910895FC0124
:10F89000538D448D252F30E0842F90E0821B930BF5
:10F8A000541718F081589F4F089501970895FC014F
:10F8B000918D828D981761F0A28DAE0FBF2FB11D73
:10F8C0005D968C91928D9F5F9F77928F90E00895C7
:10F8D0008FEF9FEF0895FC01918D828D981731F085
:10F8E000828DE80FF11D858D90E008958FEF9FEFD9
:10F8F0000895FC01918D228D892F90E080589F4FB3
:10F90000821B91098F779927089582EE99E00E94D2
:10F91000797C21E0892B09F420E0822F08958FEF74
:10F920009AE00E94797C21E0892B09F420E0822F63
:10F9300008958CE19CE00E94797C21E0892B09F4F8
:10F9400020E0822F08958EEF9DE00E94797C21E0D7
:10F95000892B09F420E0822F0895FC01A48DA80FC3
:10F96000B92FB11DA356BF4F2C91848D90E0019605
:10F970008F779927848FA689B7892C93A089B1891D
:10F980008C9180648C93938D848D981306C002882B
:10F99000F389E02D80818F7D80830895EF92FF921F
:10F9A0000F931F93CF93DF93EC0181E0888F9B8DA2
:10F9B0008C8D981316C0E889F989808185FF11C064
:10F9C000EE89FF896083E889F9898081806480837A
:10F9D00081E090E0DF91CF911F910F91FF90EF9028
:10F9E0000895F62E0B8D10E00F5F1F4F0F77112734
:10F9F000E02E8C8D8E110CC00FB607FCFACFE88973
:10FA0000F989808185FFF5CFCE010E94AD7CF1CFD1
:10FA1000EB8DEC0FFD2FF11DE356FF4FF0820B8FA6
:10FA2000EA89FB8980818062D2CFCF93DF93EC019A
:10FA3000888D8823B9F0AA89BB89E889F9898C91D6
:10FA400085FD03C0808186FD0DC00FB607FCF7CF92
:10FA50008C9185FFF2CF808185FFEDCFCE010E9492
:10FA6000AD7CE9CFDF91CF91089580E090E0892BC4
:10FA700029F00E94A37C81110E94000080E090E0A8
:10FA8000892B29F00E94997C81110E94000080E05E
:10FA900090E0892B29F00E948F7C81110E94000048
:10FAA00080E090E0892B29F00E94857C81110C94E4
:10FAB000000008950F931F93FC0162857385848570
:10FAC00095850281138124813581601B710B820B26
:10FAD000930B0685178520893189601B710B820B7A
:10FAE000930B1F910F910895DC01ED91FC91019012
:10FAF000F081E02D19948FEF9FEF0895FC0162894A
:10FB00007389848995890895EF920F931F93CF93FA
:10FB1000DF93FC01248D222341F0213051F1DF914C
:10FB2000CF911F910F91EF900895228933894489D5
:10FB3000558986899789A08DB18D821B930BA40B63
:10FB4000B50B892F9A2FAB2FBB278C010F5F1F4F4F
:10FB50006281738184819581CFB7F894DCB7E1E04D
:10FB6000ECBFEE24E394E2E0FEEF1995DCBFCFBFDB
:10FB7000D6CFF0E0E0E0DF91CF911F910F91EF90B1
:10FB80001994FC01138E128E41110CC08289938945
:10FB9000A489B589868B978BA08FB18F148E81E055
:10FBA00090E0089590E080E00895CF92DF92EF9288
:10FBB000FF92CF93DF93DC01CB01642FCFB7F89492
:10FBC0006D01EE24FF24CBBEDCB741E04CBFA901A0
:10FBD000E1E0FEEF1995DCBFCFBFDF91CF91FF9041
:10FBE000EF90DF90CF900895CF93DF93FC01248DA9
:10FBF000211110C0EC01828D938D892B49F066890B
:10FC00007789808D918D30E020E045E00E94D57DA0
:10FC10001B8E1A8EDF91CF9108951F93CF93DF93A0
:10FC2000FC01248D211145C0162FEC01828D938D8E
:10FC3000892B49F466897789808D918D30E020E0A9
:10FC400043E00E94D57D4A8D5B8DCA018170992762
:10FC5000FE01E80FF91F158F892B69F02D8D3E8D60
:10FC60006E897F89888D998D640F751F811D911D07
:10FC700041E00E94D57D8A8D9B8D01969B8F8A8F56
:10FC800081159140B1F46E897F89888D998D30E01E
:10FC900020E045E00E94D57D1B8E1A8E8E899F89BB
:10FCA000A88DB98D9F5FAF4FBF4F8E8B9F8BA88F55
:10FCB000B98F81E090E0DF91CF911F910895DC0131
:10FCC000ED91FC910280F381E02D40E01994FB015D
:10FCD00024813581428153812417350750F4A08156
:10FCE000B181A20FB31F8C93848195810196958376
:10FCF000848380E00895CF93DF93EC01E881F9815C
:10FD00000284F385E02DCE0119950196B9F7DF91B4
:10FD1000CF910895CF92DF92EF92FF920F931F93AE
:10FD2000CF93DF937C016A018B01D0E0C0E0CC155A
:10FD3000DD0581F0D701ED91FC910284F385E02D82
:10FD4000C70119958F3F980729F0F80181938F011A
:10FD50002196EDCFCE01DF91CF911F910F91FF90B2
:10FD6000EF90DF90CF900895CF93C62FDC01ED91F7
:10FD7000FC910088F189E02D1995DC01ED91FC9151
:10FD80000190F081E02D6C2FCF911994062E000C7C
:10FD9000770BFC01778366830895CF93DF93EC01A3
:10FDA0008E819F81019611F5E881F9810088F189A2
:10FDB000E02DCE011995DC01ED91FC910084F185D7
:10FDC000E02D1995892BB1F0E881F9810284F38542
:10FDD000E02DCE0119958132910534F3E881F98146
:10FDE0000684F785E02D682FCE01199581E0DF911B
:10FDF000CF91089580E0FBCFFC0120812EBD9B01B7
:10FE00002150310941F051810DB407FEFDCF4EB5AF
:10FE10005EBD4193F5CF61507109860F971F0DB4F8
:10FE200007FEFDCF2EB5FC0120830895E0919308D5
:10FE3000F0919408808190919208892B8083089595
:10FE4000E0919308F09194089081809192088095B8
:10FE50008923808308958EBD00000DB407FEFDCF79
:10FE60008EB5089590E02091CF09233339F40C9694
:10FE7000982F990F990F990F80E008954896F8CF21
:10FE8000EF92FF920F931F93CF93DF93EC018B01BF
:10FE90007A010E9414A7688B798B8A8B9B8B8C814B
:10FEA0009D81DC01ED91FC910280F381E02DA701A1
:10FEB000B801DF91CF911F910F91FF90EF901994AE
:10FEC0001F93CF93DF93EC01162F0E9414A7688B2A
:10FED000798B8A8B9B8B8C819D81DC01ED91FC91D0
:10FEE0000190F081E02D612FDF91CF911F91199446
:10FEF000CF92DF92EF92FF92CF93DF93EC018E814E
:10FF00009F818F3F980759F02FEF3FEF3F832E835C
:10FF1000DF91CF91FF90EF90DF90CF9008950E94F6
:10FF200014A76B017C01A4EFCA0EA1E0DA1EE11C4C
:10FF3000F11CE881F9810088F189E02DCE01199545
:10FF4000DC01ED91FC910084F185E02D1995892B60
:10FF500039F40E9414A76C157D058E059F0548F3A2
:10FF6000E881F9810088F189E02DCE011995DC0145
:10FF7000ED91FC910284F385E02DDF91CF91FF900C
:10FF8000EF90DF90CF9019940E940ADA0F931F939D
:10FF9000CF93DF93EC0188819981009759F02A81F2
:10FFA0003B812617370730F081E0DF91CF911F9119
:10FFB0000F9108958B016F5F7F4F0E9429D90097A1
:10FFC00059F0998388831B830A832C813D81232BDD
:10FFD00059F7FC011082E8CF80E0E7CFCF92DF92A3
:10FFE000EF92FF920F931F93CF93DF936C018B01DE
:10FFF00086E090E00E9442C8EC019093140980933F
:020000021000EC
:100000001309F60101900020E9F7CF018C199D0931
:100010000E9442C87C01B6010E9493DAF601019069
:100020000020E9F73197EC19FD09EE0DFF1D108254
:10003000F982E8821B830A8380911609909117093F
:100040009D838C83D0931709C0931609DF91CF91BC
:100050001F910F91FF90EF90DF90CF900895FC01DA
:10006000868197818F3F980729F02FEF3FEF3783E5
:1000700026830895808591850C94B1CC7F928F92D0
:100080009F92AF92BF92CF92DF92EF92FF920F9327
:100090001F93CF93DF93CDB7DEB7A6970FB6F89433
:1000A000DEBF0FBECDBF8C01762E942E852E20E2B2
:1000B000A22ECE0101967C01DC01EA2D1D92EA956B
:1000C000E9F76801F3E4CF0ED11C82E394E09AA330
:1000D00089A38FEF8BA38CA38DA38EA343E450E061
:1000E000BE016F5D7F4FC6010E94A828019609F4EA
:1000F000BFC081E089838A8386E0B82EBB821C82E0
:10010000D80114966D917D918D919C9117970E94C5
:1001100031D66D837E838F83988789869A8680E81F
:1001200090E09C878B874CE150E0B701C6010E94AC
:100130003D28FE0137968AE1DF011D928A95E9F795
:100140004801B8E08B0E911CF401D70101900D928B
:10015000BA94E1F740E150E0B701C6010E943D28A2
:10016000F7011192AA94E9F796E0A92EB12C40E28A
:1001700050E0B701C6010E943D28F1E0AF1AB10876
:10018000B1F783E6898392E89A8393E59B838C8316
:1001900085E38D8381E08E837F829DE3988797E05E
:1001A00099878A8786E0F401DE011B9601900D9203
:1001B0008A95E1F78CE0898B8A8B64E576E0CE0145
:1001C00043960E9493DAD8011B966C91CE01499612
:1001D0000E9494A2F8016485CE014B960E9494A2DD
:1001E000D8011D966C91CE014D960E9494A24EE1CD
:1001F00050E0B701C6010E943D28B3E07B121EC04B
:1002000082E3898384E08A83F80196859B839785BE
:100210009C8390899D8391899E8396E39F838887A1
:10022000828D8987838D8A87848D8B87858D8C8746
:100230004CE050E0B701C6010E943D2887E3898366
:1002400086E08A8391E09B8393E09C838D838FE09B
:100250008E838AE38F838BE388878FEF898749E0DA
:1002600050E0B701C6010E943D28C6010E947728D0
:10027000A6960FB6F894DEBF0FBECDBFDF91CF912B
:100280001F910F91FF90EF90DF90CF90BF90AF90B4
:100290009F908F907F90089590E080E00C941527B8
:1002A000CF93DF93C4E1D0E00E944C81882361F0BA
:1002B00061E070E080E090E00E94E2A62197A1F763
:1002C00080E0DF91CF91089581E0FBCFFF920F9303
:1002D0001F93CF93DF931F921F92CDB7DEB7F82EF7
:1002E00022E030E0AE014F5F5F4F66E270E00E94B7
:1002F000162809811A8110270127102722E030E0F3
:10030000AE014F5F5F4F66E270E08F2D0E941628AE
:1003100089819A819827892798270817190749F40E
:10032000C8010F900F90DF91CF911F910F91FF9017
:1003300008958C01E3CFAF92BF92CF92DF92EF92FC
:10034000FF920F931F93CF93DF93DC01CD90DC904E
:100350001197C114D10439F01496CD91DC918C0120
:100360007601209761F4DF91CF911F910F91FF905B
:10037000EF90DF90CF90BF90AF9008957501570137
:10038000BFEFAB1ABB0AF7018081082E000C990B56
:100390000E9457CB892B91F72197CC0DDD1D8881C9
:1003A000082E000C990B0E9457CB892B29F0CE15F3
:1003B000DF0510F02197F3CFAE014F5F5F4F4E196D
:1003C0005F09D80115965C934E931497CE14DF0401
:1003D00020F4B701C6010E9446DAD801ED91FC91E4
:1003E000119714968D919C91E80FF91F1082BBCF45
:1003F000CF93DF93DC011496ED91FC916E177F078C
:1004000028F54115510511F19F01261B370B4217A5
:10041000530708F49A01DB01EC0188819981E21B02
:10042000F30BFD83EC83AF01461B570B260F371FE1
:10043000BC01620F731F8A0F9B1F0E94B8DAE8810C
:10044000F9818C819D81E80FF91F1082DF91CF9196
:100450000895DF92EF92FF920F931F93CF93DF9354
:10046000FC01E480F580E114F10451F48FEF9FEF7B
:10047000DF91CF911F910F91FF90EF90DF90089542
:10048000EC010190F081E02DEE0DFF1DD080108277
:1004900008811981062E000C770BC8010E94C7DA6B
:1004A0000E0D1F1DF801D082009701F328813981BC
:1004B000821B930BDDCFFC0124813581621773070A
:1004C00020F480819181009729F41092150985E12B
:1004D00099E00895860F971F0895FB014481558187
:1004E000FC01248135812417350778F080819181C2
:1004F000009759F0FB01608171816115710529F048
:100500000E94AADA21E0892B09F020E0822F0895C9
:10051000FC0124813581232B39F421E0FB0180810A
:10052000882349F020E007C0808191810E948ADA07
:1005300021E0892BB9F7822F0895FC0124813581B0
:10054000FB014481558124173507E1F4FC018081CA
:100550009181FB01608171810097D1F06115710576
:10056000A1F4232BC1F0FC01808190E008C0232B73
:1005700091F0FB01808190E091958195910921E0B6
:10058000892B09F020E0822F08950E948ADAF7CFA4
:100590006115710561F721E0F6CFEF92FF920F939D
:1005A0001F93CF93DF936115710541F480E0DF91D4
:1005B000CF911F910F91FF90EF9008954115510534
:1005C000B1F07B01EC010C811D81040F151FB801F6
:1005D0000E94C67F882351F3288139818C819D81B7
:1005E000B701820F931F0E9493DA1D830C8381E071
:1005F000DECFCF93DF931F921F92CDB7DEB7698313
:100600001A8241E050E0BE016F5F7F4F0E94CD82B1
:100610000F900F90DF91CF9108950F931F93CF9379
:10062000DF938C01EB01FC01808191810097E1F067
:100630006881798161157105A9F0428153812C810E
:100640003D814217530770F00E9493DA8C819D819F
:10065000F801958384831D821C82DF91CF911F91C5
:100660000F9108950E94DEC888819981F8019183D5
:1006700080838A819B81938382838C819D819583F2
:100680008483198218821B821A82E5CFCF93DF936D
:10069000EC0188819981009711F00E94DEC81982CF
:1006A00018821D821C821B821A82DF91CF910895CD
:1006B000EF92FF920F931F93CF93DF9300D01F927F
:1006C000CDB7DEB77C01862F4AE08E010F5F1F4F4A
:1006D000B80190E00E94FACBF80101900020E9F700
:1006E0003197AF01401B510BB801C7010E94CD8269
:1006F000811103C0C7010E944683C7010F900F906C
:100700000F900F90DF91CF911F910F91FF90EF907D
:100710000895CF93DF93EC016115710539F4CE0193
:100720000E944683CE01DF91CF910895FB01019095
:100730000020E9F73197AF01461B570B0E94CD828D
:10074000882369F3EFCFCF93DF93EC01FB01448162
:100750005581608171810E94CD82811103C0CE01DB
:100760000E944683CE01DF91CF910895EF92FF92D0
:100770000F931F93CF93DF93EC017B018A01BA01A2
:100780000E94C67F81110BC0CE010E944683CE011C
:10079000DF91CF911F910F91FF90EF9008951D83EE
:1007A0000C83B701888199810E9493DAF0CFFB0115
:1007B00001900020E9F73197AF01461B570B0C94CD
:1007C000B683CF93DF93EC016115710531F00E9480
:1007D000D783CE01DF91CF9108950E944683F9CF50
:1007E000CF93DF93EC01FB018617970749F06081F7
:1007F00071816115710541F0448155810E94B68374
:10080000CE01DF91CF9108950E944683F9CFFC017C
:10081000808191810C94DEC8EF92FF920F931F9319
:10082000CF93DF93EC018B01198218821B821A820D
:100830001D821C82CB010E948ECB7C01BC01CE01AB
:100840000E94C67F811109C0CE01DF91CF911F9117
:100850000F91FF90EF900C944683FD82EC82B801DB
:1008600088819981DF91CF911F910F91FF90EF9037
:100870000C9487CBFC0111821082138212821582A4
:1008800014820C94F083FC01118210821382128274
:10089000158214826115710551F0FB010190002051
:1008A000E9F73197AF01461B570B0C94B6830895B7
:1008B0000F931F93CF93DF93EC010E9414A76887D7
:1008C00079878A879B87E881F9810284F385E02D07
:1008D000CE01199597FF15C00E9414A708851985A8
:1008E0002A853B85601B710B820B930B0C811D814C
:1008F0002E813F81601771078207930720F38FEFE6
:100900009FEFDF91CF911F910F910895EF92FF928A
:100910000F931F93CF93DF93EC017B01042F6DE5C1
:1009200076E00E944384C7010E945884002E000C88
:10093000110B97FD0BC00817190741F0682FCE0166
:100940000E94F982C7010E945884F3CFCE01DF9143
:10095000CF911F910F91FF90EF900895CF92DF926A
:10096000EF92FF920F931F93CF93DF936C017A0165
:100970008B01D0E0C0E0C6010E94588497FD07C0FB
:10098000F80181938F012196EC16FD06A1F7CE01A7
:10099000DF91CF911F910F91FF90EF90DF90CF905B
:1009A0000895FB0101900020E9F73197AF01461B44
:1009B000570BDC01ED91FC910280F381E02D19943D
:1009C0008F929F92AF92BF92EF92FF920F931F93DD
:1009D000CF93DF93CDB7DEB7A1970FB6F894DEBF04
:1009E0000FBECDBF7C01FA01CB0119A2223008F461
:1009F0002AE08E010F5D1F4F822E912CB12CA12C6D
:100A0000BF01A50194010E949ED5F901CA016A3077
:100A10000CF5605DD8016E938D01232B242B252BC3
:100A200079F790E080E0109721F0BD01C7010E94A6
:100A3000D184A1960FB6F894DEBF0FBECDBFDF9173
:100A4000CF911F910F91FF90EF90BF90AF909F902B
:100A50008F900895695CDECF6BE576E00C94D184CD
:100A6000242F462F50E070E060E00C94E084EF9279
:100A7000FF920F931F93CF93DF93009751F4CFEF23
:100A8000DFEFCE01DF91CF911F910F91FF90EF909B
:100A90000895DC011C96ED90FC90F7010081118116
:100AA000D801ED91FC910688F789E02DC8011995D0
:100AB000882329F3D801ED91FC910084F185E02D84
:100AC000C8011995D801ED91FC91892B61F302843D
:100AD000F385E02DC8011995EC01019681F2F8012A
:100AE000818D882339F04AE050E06C2F8EEF9DE035
:100AF0000E943085D70112968C91882311F2C5325D
:100B0000D10509F0BECFD801ED91FC910084F185AB
:100B1000E02DC801199502975CF0D801ED91FC9188
:100B20000688F789E02DC80119958111ECCFA7CF70
:100B3000D1E0C0E0D801ED91FC910284F385E02D75
:100B4000C80119958F3F980709F499CF9C0121544A
:100B500031092A31310570F48D2F8295807F829F73
:100B6000C00D1124D11104C00C2E000CDD0B89CF57
:100B7000D0E0E0CF9C01215631092A31310560F3E4
:100B8000C0978A30910570F79D2F9295907F989F1E
:100B9000C00D1124E7CFDC01ED91FC910190F081B3
:100BA000E02D1994CF92DF92EF92FF920F931F9353
:100BB000CF93DF932115310581F4DC01ED91FC9198
:100BC0000190F081E02D642FDF91CF911F910F9163
:100BD000FF90EF90DF90CF9019942A30310501F506
:100BE0002AE077FF1DC06A017B01EC016DE20E94E3
:100BF000CB858C0144275527BA014C195D096E0934
:100C00007F092AE0CE010E94E084800F911FDF91CE
:100C1000CF911F910F91FF90EF90DF90CF900895AB
:100C2000DF91CF911F910F91FF90EF90DF90CF90C8
:100C30000C94E0848F929F92AF92BF92CF92DF92FA
:100C4000EF92FF920F931F93CF93DF937C018B0161
:100C50004C0182E0880E911C5701E5E0AE0EB11CFC
:100C6000D0E0C0E0F40161914F014AE050E0C801DA
:100C70000E9430856C016EE2C8010E94CB858C0D0C
:100C80009D1DC80FD91F8A149B0461F74AE050E0EC
:100C9000F7016581C8010E9430858C0F9D1FDF918F
:100CA000CF911F910F91FF90EF90DF90CF90BF9069
:100CB000AF909F908F9008956115710511F00C947D
:100CC000D18490E080E008950F931F93CF93DF933A
:100CD000EC018B0169EF75E00E945C86011511053E
:100CE000C1F1F80161918F01662399F1603240F002
:100CF000623231F06C3521F0CE010E94CB85F1CF0C
:100D00006CE5CE010E94CB85F801319780818C3053
:100D1000D1F044F48930D9F08A30B9F0883009F73D
:100D200062E6EACF823259F024F462E78D3021F393
:100D3000D8CF8F3231F06CE58C35F1F2D2CF62E250
:100D4000DBCF6FE2D9CF66E6D7CF6EE6D5CF64E7CB
:100D5000D3CF62E2CE010E94CB8590E080E0DF91AC
:100D6000CF911F910F910895DB0114964D915C91E5
:100D700015976D917C91DC01ED91FC910280F381DE
:100D8000E02D1994EF92FF920F931F93CF93DF936F
:100D90008C017B01D0E0C0E0F701EC0FFD1F6491F6
:100DA000662361F0D801ED91FC910190F081E02D76
:100DB000C8011995892B11F02196EECFCE01DF9154
:100DC000CF911F910F91FF90EF9008950F931F9374
:100DD000CF93DF93EC010E94C2868C01CE010E946A
:100DE0002C85800F911FDF91CF911F910F91089556
:100DF000DC0182E394E08D939D9384E0FB010190FC
:100E00000D928A95E1F708953F924F925F926F920B
:100E10007F928F929F92AF92BF92CF92DF92EF928A
:100E2000FF920F931F93CF93DF93CDB7DEB7EA976F
:100E30000FB6F894DEBF0FBECDBF7C012A013B0187
:100E400069010E9414A74B015C0187010D5B1F4FD4
:100E5000C8010E941D1618161906ACF00E9414A7AE
:100E6000681979098A099B094616570668067906A2
:100E700008F468C10E94906961E070E080E090E051
:100E80000E94E2A6E5CF42E250E0BE016F5F7F4FD5
:100E9000C8010E94A81589818230D1F0312C832DA0
:100EA000EA960FB6F894DEBF0FBECDBFDF91CF91AB
:100EB0001F910F91FF90EF90DF90CF90BF90AF9078
:100EC0009F908F907F906F905F904F903F9008958C
:100ED000F801848995898334910501F76D817E81BC
:100EE0008F8198850E9431D64B015C01F60180828A
:100EF0009182A282B38246E050E0B701685F7F4FE3
:100F0000CE014D960E9439DA892B41F6F701808196
:100F10009181A281B38188169906AA06BB0608F4BE
:100F2000BDCF84819581A681B78188159905AA05D1
:100F3000BB0508F4B3CF89899A89AB89BC898687B8
:100F40009787A08BB18B4EEC50E070E060E0C80159
:100F50000E94A815312CC701829698AB8FA7F70184
:100F6000B696FAABE9AB08969CAB8BAB67019AE1FE
:100F7000C90ED11CBD96FEABEDABC701429698AF32
:100F80008FABFD97FAAFE9AF4701FEE18F0E911CE1
:100F9000F801818D928D181619060CF080CFC801CA
:100FA0000E94C7158333910509F4B2C014F581304E
:100FB000910509F464C044F4892B51F3C8010E94DF
:100FC000C715AC01552775C08330910509F462C07F
:100FD0000697A1F7C8010E94C715B82E44E050E05B
:100FE000B401C8010E94A815EB2DE450FF0BAF011E
:100FF00060C08A33910509F45FC084F5853391059B
:10100000B1F1C697D9F6C8010E94C7155C01B601B7
:10101000CE0189960E94F8868BA59CA5ADA5BEA59C
:10102000892B8A2B8B2BB1F0EDA9FEA94080518032
:1010300062807380B601CE0183960E94F8868DA1EE
:101040009EA1AFA1B8A5A501481659066A067B0660
:1010500009F0B8CF44E050E0B60118C08B339105D9
:1010600009F440C08F3F910509F492CFA7CFC80182
:101070000E94C715C8010E94C715382E89CFC80124
:101080000E94C71544E050E06FA978ADC8010E94E6
:10109000A8157ECFC8010E94C715B82E44E050E0C5
:1010A00069AD7AADC8010E94A8158B2D8450990BAB
:1010B000AC0170E060E0EACFC8010E94C71544E0CF
:1010C00050E069A97AA9C8010E94A815F70166A194
:1010D00077A180A591A50E9431D666A377A380A7AA
:1010E00091A756CFC8010E94C71544E050E06BA9F4
:1010F0007CA9C8010E94A815F70162A573A584A563
:1011000095A50E9431D662A773A784A795A740CF63
:10111000C8010E94C71544E050E06FA578A9C80136
:101120000E94A815F70162A173A184A195A10E9454
:1011300031D662A373A384A395A366A777A780ABD8
:1011400091AB26CF33243A94AACE2F923F924F925E
:101150005F926F927F928F929F92AF92BF92CF9247
:10116000DF92EF92FF920F931F93CF93DF9300D004
:1011700000D0CDB7DEB78C010E94B3C92FEC37E0A9
:1011800040E050E00E94C0D5DC01CB010196A11DDA
:10119000B11DF80184839583A683B78380839183EF
:1011A000A283B3835801F3E4AF0EB11CC5010E94C2
:1011B000721564E470E0C5010E94EC16882309F4FE
:1011C00045C10E9414A72B013C01480182E4880E0E
:1011D000911C48EEC42E43E0D42EE12CF12C52E0B9
:1011E000252E1E821D82D4018C918330B1F1811194
:1011F00066C0F80184819581A681B7810196A11D01
:10120000B11D84839583A683B7830E9414A76419B4
:10121000750986099709A70196010E949ED5A90123
:1012200061E0C8010E943E8081E0D4018C938D81F1
:101230009E810197C1F20E9414A76419750986095D
:101240009709D801D6962D913D914D915C91D997F2
:10125000261737074807590720F6C5010E9472155F
:10126000F80184819581A681B7810196A11DB11DE8
:1012700084839583A683B7830E9414A7F801FE9602
:1012800060837183828393838D819E8126960FB6BE
:10129000F894DEBF0FBECDBFDF91CF911F910F91AC
:1012A000FF90EF90DF90CF90BF90AF909F908F9086
:1012B0007F906F905F904F903F902F900895843073
:1012C000F1F4F80184819581A681B7810196A11D71
:1012D000B11D84839583A683B7830E9414A76419E4
:1012E000750986099709A70196010E949ED5A90153
:1012F00063E0C8010E943E80D4012C9298CF8130D7
:1013000051F5F80142AD53AD64AD75AD9E012F5F4F
:101310003F4FC8010E940487382EF2E08F1390C01F
:1013200089819A81AB81BC81F80184839583A683EE
:10133000B7830E9414A76419750986099709A70144
:1013400096010E949ED5A90163E0C8010E943E80DB
:10135000D4013C926CCF823009F069CFF80142ADE4
:1013600053AD64AD75AD9E012F5F3F4FC8010E9424
:101370000487382EF5E08F135DC0E3E0D401EC93D1
:10138000F80182A193A1A4A1B5A1892B8A2B8B2B53
:1013900041F484E893E0A0E0B0E082A393A3A4A387
:1013A000B5A3F80186A197A1A0A5B1A5892B8A2B89
:1013B0008B2B61F482A193A1A4A1B5A1B695A795A9
:1013C0009795879586A397A3A0A7B1A7F80182A5B3
:1013D00093A5A4A5B5A5892B8A2B8B2BA9F482A153
:1013E00093A1A4A1B5A1AC01BD0123E076956795B9
:1013F000579547952A95D1F7841B950BA60BB70BEC
:1014000082A793A7A4A7B5A7F80186A197A1A0A535
:10141000B1A586A797A7A0ABB1AB82A593A5A4A5BC
:10142000B5A582AB93ABA4ABB5AB81E090E09E8356
:101430008D83FDCE96E0891303C0D4011C92F7CEB4
:10144000BFEF3B12F4CEF4011082F1CE1E821D825A
:101450001BCF1F920F920FB60F9211240BB60F9253
:101460002F933F934F935F936F937F938F939F93AC
:10147000AF93BF93EF93FF9382EE99E00E94AD7C10
:10148000FF91EF91BF91AF919F918F917F916F915C
:101490005F914F913F912F910F900BBE0F900FBE18
:1014A0000F901F9018951F920F920FB60F92112454
:1014B0000BB60F922F933F934F935F936F937F934E
:1014C0008F939F93AF93BF93EF93FF9382EE99E037
:1014D0000E942E7CFF91EF91BF91AF919F918F91D0
:1014E0007F916F915F914F913F912F910F900BBE24
:1014F0000F900FBE0F901F9018951F920F920FB66E
:101500000F9211240BB60F922F933F934F935F933B
:101510006F937F938F939F93AF93BF93EF93FF93BB
:101520008FEF9AE00E94AD7CFF91EF91BF91AF9158
:101530009F918F917F916F915F914F913F912F91EB
:101540000F900BBE0F900FBE0F901F9018951F921B
:101550000F920FB60F9211240BB60F922F933F9359
:101560004F935F936F937F938F939F93AF93BF93AB
:10157000EF93FF938FEF9AE00E942E7CFF91EF9103
:10158000BF91AF919F918F917F916F915F914F919B
:101590003F912F910F900BBE0F900FBE0F901F9099
:1015A00018951F920F920FB60F9211240BB60F923F
:1015B0002F933F934F935F936F937F938F939F935B
:1015C000AF93BF93EF93FF938CE19CE00E94AD7CBF
:1015D000FF91EF91BF91AF919F918F917F916F910B
:1015E0005F914F913F912F910F900BBE0F900FBEC7
:1015F0000F901F9018951F920F920FB60F92112403
:101600000BB60F922F933F934F935F936F937F93FC
:101610008F939F93AF93BF93EF93FF938CE19CE0E5
:101620000E942E7CFF91EF91BF91AF919F918F917E
:101630007F916F915F914F913F912F910F900BBED2
:101640000F900FBE0F901F9018951F920F920FB61C
:101650000F9211240BB60F922F933F934F935F93EA
:101660006F937F938F939F93AF93BF93EF93FF936A
:101670008EEF9DE00E94AD7CFF91EF91BF91AF9105
:101680009F918F917F916F915F914F913F912F919A
:101690000F900BBE0F900FBE0F901F9018951F92CA
:1016A0000F920FB60F9211240BB60F922F933F9308
:1016B0004F935F936F937F938F939F93AF93BF935A
:1016C000EF93FF938EEF9DE00E942E7CFF91EF91B0
:1016D000BF91AF919F918F917F916F915F914F914A
:1016E0003F912F910F900BBE0F900FBE0F901F9048
:1016F0001895CF92DF92EF92FF921F93CF93DF93D3
:10170000EC016A017B01122FE889F98982E080836C
:10171000C11481EED806E104F104A1F060E079E0A3
:101720008DE390E0A70196010E949ED521503109DA
:10173000410951095695479537952795211580E11F
:10174000380798F0E889F989108260E874E88EE13A
:1017500090E0A70196010E949ED5215031094109D0
:1017600051095695479537952795EC85FD8530832A
:10177000EE85FF852083188EEC89FD891083EA8928
:10178000FB89808188698083EA89FB8980818F7DDC
:101790008083DF91CF911F91FF90EF90DF90CF90EA
:1017A0000895DF92EF92FF920F931F93CF93DF93F1
:1017B00000D000D0CDB7DEB78B017A01D22E6DE517
:1017C00076E0CE0101960E9443849E012F5F3F4F39
:1017D0004D2DB701C8010E946CAECE0101960E944A
:1017E000078426960FB6F894DEBF0FBECDBFDF91FB
:1017F000CF911F910F91FF90EF90DF900895CF92BE
:10180000DF92EF92FF920F931F93CF93DF93CDB7A9
:10181000DEB7EC970FB6F894DEBF0FBECDBFDC018C
:101820002C91222309F469C069E474E00E94C4CBBE
:101830009A8389837E01B3E0EB0EF11C01E010E096
:1018400069E474E090E080E00E94C4CBD02EC12E09
:10185000F701819391937F010E31110521F00F5F04
:101860001F4F892B69F70091130910911409E98022
:10187000FA800115110589F1D8016D917C91C7019C
:101880000E948ADA892B29F5D8011296ED91FC91F4
:10189000BE016F5F7F4F8D2D9C2D19958C018EEFB2
:1018A0009DE00E942C856BEA77E18EEF9DE00E941F
:1018B000C286C801EC960FB6F894DEBF0FBECDBF4E
:1018C000DF91CF911F910F91FF90EF90DF90CF901C
:1018D0000895F80104811581CCCF6FEA77E18EEF8E
:1018E0009DE00E94E6868EEF9DE00E942C856BEACB
:1018F00077E18EEF9DE00E94C28610E000E0D9CF34
:10190000CF938EEF9DE00E94797C892BE9F18EEFD9
:101910009DE00E94577CC82F8A3089F08D3079F085
:10192000883001F568E08EEF9DE00E94CB858091C4
:101930001809882331F3815080931809E2CFE09190
:101940001809F0E0E952F74F10826BE576E08EEF70
:101950009DE00E945C8687ED98E00E94FF8B1092CC
:101960001809CFCF682F8EEF9DE00E94CB85E091C4
:101970001809EB3330F681E08E0F80931809F0E000
:10198000E952F74FC083BDCFCF9108958F929F92B8
:10199000AF92BF92CF92DF92EF92FF920F931F937D
:1019A000CF93DF936115710509F497C0DB01189699
:1019B000EC911897E295E07FE595E595E595E5953D
:1019C000E73008F08AC0EC010E2E000CFF0B8827D0
:1019D000E351F3478F4F0C9429D6F48C058D0E8D6F
:1019E000258D708D828DBB8D6EE576E0CE01DF9109
:1019F000CF911F910F91FF90EF90DF90CF90BF900C
:101A0000AF909F908F900C94D18419968C9168E63A
:101A100076E0882359F363E676E0E8CF19964D9196
:101A20005D916D917C911C972AE030E0CE01DF91B1
:101A3000CF911F910F91FF90EF90DF90CF90BF90CB
:101A4000AF909F908F900C94D2851996CD90DD9099
:101A5000ED90FC901C9720E030E0A901C701B60191
:101A60000E9454D487FF09C06CEF74E0CE010E943D
:101A70005C86F7FAF094F7F8F094C701B6010E947B
:101A80002DD74B015C012AE0BC01A401CE010E94CC
:101A9000E08462E576E0CE010E945C86C501B40177
:101AA0000E9459D49B01AC01C701B6010E9447D6E0
:101AB0002DEC3CEC4CE45DE30E9448D620E030E0A5
:101AC00040E251E40E94BAD40E942DD7AB0170E0ED
:101AD00060E02AE0CE010E94E08490E080E01DC03A
:101AE00019966D917C91CE01DF91CF911F910F914D
:101AF000FF90EF90DF90CF90BF90AF909F908F902E
:101B00000C94648616960D911C916BE5CE010E9493
:101B1000CB85019679F48FEF9FEFDF91CF911F91E5
:101B20000F91FF90EF90DF90CF90BF90AF909F907C
:101B30008F9008950115110579F0B801CE010E942A
:101B4000C68C019641F3D80112960D911C91011596
:101B5000110511F06CE2DACF6DE5CE010E94CB8564
:101B600021E030E0019611F030E020E0882799274D
:101B7000821B930BD2CF16960D911C916BE7CE0171
:101B80000E94CB85019639F20115110529F1D80182
:101B90006D917C91CE010E946486019609F4BBCFC1
:101BA0006AE3CE010E94CB85019609F4B4CFB80157
:101BB000CE010E94C68C019609F4ADCFD8011296D1
:101BC0000D911C910115110539F06CE2CE010E94B6
:101BD000CB850196C9F69FCF6DE7BFCFCF93DF933B
:101BE000EC01E881F9810284F385E02DCE0119959D
:101BF0008F3F980769F0E881F981813291059CF364
:101C00000684F785E02D682FCE01199590E080E0DD
